:020000040800F2
:100000000000012095460008B92C0008BB2C000810
:10001000BD2C0008BF2C0008C12C00080000000007
:10002000000000000000000000000000C32C0008D9
:10003000C52C000800000000C72C0008C92C0008CF
:10004000E5460008E5460008CD2C0008E546000816
:10005000E5460008E5460008D92C0008DF2C00081A
:10006000E5460008E5460008072D0008E5460008BB
:10007000E52C0008E72C0008E92C0008F52C000806
:10008000012D0008032D0008E5460008E54600089C
:1000900000000000E5460008092D0008E5460008BC
:1000A000E5460008E5460008E5460008E546000884
:1000B000E5460008E5460008E5460008E546000874
:1000C000E5460008E5460008E5460008E546000864
:1000D000E5460008112D0008E5460008E546000841
:1000E000E54600080F2D00081D2D0008E546000814
:1000F000E54600080000000000000000E54600089A
:10010000E5460008E5460008292D0008E5460008F8
:10011000E5460008E5460008E5460008E546000813
:10012000E5460008E5460008E5460008E546000803
:08013000E5460008E546000861
:1001400010B5054C237833B9044B13B10448AFF311
:1001500000800123237010BD840A002000000000ED
:10016000C06E010808B5034B1BB103490348AFF348
:10017000008008BD00000000880A0020C06E010851
:1001800014214160704714207047406A7047000096
:1001900081010008870100088B010008A101000807
:1001A00010B5044604F1100000F05CFCC4F8F8003F
:1001B0000148C4F87C0110BD90010008F8B5E6B014
:1001C00004460D4616461F460A4906A800F0CAFE18
:1001D00070996F9A05910492009733466E996D9AC3
:1001E000039102922A466C990191214600F060F831
:1001F00067B0F0BD9C010008F8B5E6B004460D46B6
:1002000016461F46094906A800F0ACFE6F996E9A83
:100210000491039200976D996C9A02910192334672
:100220002A46214600F087F867B0F0BD9C0100081F
:1002300038B500281CBF01680029184A23D1184B83
:100240001C684FF6F0710C404CF24025AC421FBFC9
:100250001B6819404CF27024A14212D1114D29683B
:1002600079B911490B68C3F30B03B3F58A6F1FBF4C
:100270000968C1F30B0140F28343994204BF012195
:10028000117028B905E0094B994204BF0121117092
:100290004068BDE8324002F01BB900BFA00A002050
:1002A00000ED00E0002004E00010005C0000374892
:1002B0002DE9F04104460D46216816464A681F465E
:1002C00090478046B8F5403F2ED122680A9993683E
:1002D000204698478046B8F5403F25D12368089AC4
:1002E0000799D3F80CC02046E0478046B8F5403F58
:1002F0001AD12368069A39461F692046B8478046B6
:10030000B8F5403F10D1236829465D693246204642
:10031000A8478046B8F5403F06D123680B9A099953
:100320009D692046A847804621680A682046904774
:100330004046BDE8F0812DE9F04104460D462168B4
:1003400016464A681F4690478046B8F5403F2ED172
:1003500022680A999368204698478046B8F5403F3E
:1003600025D12368089A0799D3F80CC02046E047A6
:100370008046B8F5403F1AD12368069A39461F696E
:100380002046B8478046B8F5403F10D1236829463B
:100390005D6932462046A8478046B8F5403F06D101
:1003A00023680999DD6900222046A8478046216814
:1003B0000A68204690474046BDE8F0814FF440303F
:1003C00070470000F0B50C4685B0114600281A466B
:1003D0001CBF0568002D0B4B11D082B104B971B957
:1003E0000D9860B10F9E0E9F0A9B02900496039792
:1003F0000B980C9E009001962046A847034618468D
:1004000005B0F0BD020003002DE9F04F0646D0B064
:100410000868F56DD6F860E0726EB76EF36E00BADC
:1004200000906C46486800BA60600DF1400888682A
:1004300000BAA060C86800BAE060086900BA20612C
:10044000486900BA6061886900BAA061C86900BAE9
:10045000E061086A00BA2062486A00BA6062886A8D
:1004600000BAA062C86A00BAE062086B00BA2063F2
:10047000486B00BA6063886B00BAA063C86B00BAAF
:10048000E063402058F80C1C58F820CC58F838ACE1
:100490008CEA010158F840CC8AEA01018CEA010992
:1004A0004FEAF979401E48F8049BEBD187EA020035
:1004B00000EA0E00784010EBF5610098DFF824C4E4
:1004C00041186144C81882EABE032B404FEAF0612C
:1004D00053405918636859186144CF194FEAB5035E
:1004E00083EABE01014081EABE0111EBF765A16814
:1004F0004D196544A91883EAB0023A404FEAF16504
:100500005A405519E26855194FEAB70282EAB00716
:1005100065440F4005EBBE0E97EAB00717EBFE658A
:1005200027697D194FEAB10782EA0701654401EAAC
:100530000E01EB18514011EBF36561694D194FEA5B
:10054000BE0187EA010E65440EEA030E15EBB0000A
:100550008EEA070E0EEBF065D4F818E0754465449A
:10056000AA1881EAB30505404FEAF26E4D40AE4449
:10057000E569AE44E64477444FEAB00080EAB30E42
:100580000EEA020E8EEAB30E0EEBF765D4F820E009
:1005900075446544691880EAB2053D404FEAF16E42
:1005A0004540AE44656AAE44E6440EEBB3034FEA01
:1005B000B70787EAB20E0EEA010E8EEAB20E0EEB14
:1005C000F365D4F828E075446544281887EAB10536
:1005D0001D404FEAF06E7D40AE44E56AAE44E6440D
:1005E0000EEBB2024FEAB30383EAB10E0EEA000E3D
:1005F0008EEAB10E0EEBF265D4F830E07544654436
:10060000EF1983EAB00515404FEAF76E5D40AE443E
:10061000656BAE44E6440EEBB1014FEAB20282EAEA
:10062000B00E0EEA070E8EEAB00E0EEBF165D4F8AE
:1006300038E075446544EB1882EAB7050D404FEA8F
:10064000F36E5540AE44E56BAE44E6440EEBB000AD
:100650004FEAB10181EAB70E0EEA030E8EEAB70E39
:100660000EEBF065D4F840E07544654481EAB30EC2
:10067000AA180EEA000E4FEAF2658EEA010E7544E2
:10068000DDF844E04FEAB000754480EAB30E6544FB
:100690000EEA020E15EBB7078EEAB30E0EEBF76506
:1006A000DDF848E04FEAB202754480EA020E654484
:1006B0000EEA070E69188EEA000E0EEBF165DDF802
:1006C0004CE07544654405EBB3034FEAB70E1427BD
:1006D0000DF1500CDFF810528EEA010B82EA0B0B81
:1006E0000BEBF36A5CF804BBDA44AA44504483EA97
:1006F000B10B4FEAF06A8EEA0B0BDA445CF804BBEC
:10070000DA44AA44524480EAB30B4FEAF26A8BEA15
:10071000B10BDA445CF804BBDA444FEAB000AA44F7
:1007200080EA020BD6448BEAB30B0BEBFE6A5CF853
:1007300004BBDA444FEAB202AA4482EA0E0B0AEB87
:10074000B10180EA0B0B0BEBF16A5CF804BBDA44F5
:100750007F1DAA44282F0AEBB3034FEABE0EBBD37A
:100760003C2F61D3502F4DD204EB870CC7F15407B7
:100770005E4CA7FB04A504465D4FA8088EEA010A5B
:1007800082EA0A0A5CF804BB0AEBF3655D447D1952
:100790002C1983EAB10A4FEAF4658EEA0A0A554435
:1007A0005CF804AB5CF804BB55447D19AA1884EAD4
:1007B000B30A4FEAF2658AEAB10A55445D444FEA4A
:1007C000B4047D1984EA020AAE448AEAB30A0AEB49
:1007D000FE655CF804AB55444FEAB2027D1982EA2B
:1007E0000E0A15EBB10184EA0A0A5CF804BB0AEBB5
:1007F000F1655D447D1915EBB303401E4FEABE0E53
:10080000BCD12046F46D1B19F365336EC9183166EF
:10081000716E71447166B36ED218B266F16E401893
:10082000F06650B0BDE8F08F4EEA010B0EEA010A07
:100830000BEA020B4BEA0A0A0AEBF36554F827A00D
:10084000DFF8B0C0554443EAB10B654403EAB10A8E
:100850000BEA0E0B28184BEA0A0A7F1C0AEBF0651C
:1008600054F827A0554440EAB30B654400EAB30AA4
:100870000BEAB10BAA184BEA0A0A7F1C0AEBF265D5
:1008800054F827A055444FEAB00040EA020B6544F3
:1008900000EA020A0BEAB30BAE444BEA0A0A7F1CD9
:1008A0000AEBFE6554F827A055444FEAB20242EA2B
:1008B0000E0B654402EA0E0A0BEA000B15EBB101C0
:1008C0004BEA0A0A7F1C0AEBF16554F827A055444D
:1008D0007F1C65443C2F05EBB3034FEABE0EA3D348
:1008E00040E700BF9979825AA1EBD96ECDCCCCCC30
:1008F000D6C162CADCBC1B8F00B581B00168074A53
:10090000914200D110B9064801B000BD7C2114F01D
:100910009EFB4FF4003001B000BD00BF040A000888
:10092000030002002DE9F0410B4A92E8F85188B02B
:10093000694681E8F8510268084B9A4200D118B91B
:10094000074808B0BDE8F0811422083000F04FFBE2
:1009500008B0BDE8F08100BFE4090008040A0008FF
:1009600003000200152904D20268044B9A4200D108
:1009700008B903487047083000F048BB040A000873
:100980000300020010B481B013460268074CA24273
:1009900000D118B901B010BC0548704701B000F192
:1009A000240210BC083000F035BB00BF040A000868
:1009B0000300020010B481B013460268074CA24243
:1009C00000D118B901B010BC054870470A4601B003
:1009D00000F1240110BC083000F070BB040A0008CC
:1009E000030002000123456789ABCDEFFEDCBA9816
:1009F00076543210F0E1D2C3000000000000000085
:100A000000000000F9080008250900086509000831
:100A100085090008B509000809040008810F0008CD
:100A2000CD0F0008890F0008F0B5A3B004460B48AD
:100A300002900D4616461F46094B0822402104A885
:100A400000F0D1FA28980190009733462A462146B3
:100A500002A800F01BF823B0F0BD00BF040A000894
:100A6000180A000810B5040008BF002408D0054883
:100A7000054B20600822402104F1080000F0B3FA81
:100A8000204610BD040A0008180A00082DE9F041AC
:100A900004460E46216817464A681D469047804620
:100AA000B8F5003F19D12268069993682046984707
:100AB0008046B8F5003F10D123683146DE683A46DB
:100AC0002046B0478046B8F5003F06D12368079A14
:100AD00029461D692046A847804621680A682046A5
:100AE00090474046BDE8F08110B500F033FA4FF46E
:100AF000403400280EBF034C4FF4C07114F0A7FA25
:100B0000204610BD0200030010B5044600F022FA92
:100B100008B9054810BD0021A160D0F87C211168FA
:100B200088474FF4403010BD0200030070B5044602
:100B30000D4600F00FFA064E40B1D0F87C01416836
:100B40008847A84224BF65604FF44036304670BDE8
:100B5000020003002DE9FF4715000C4600D02CB120
:100B6000064600F0F7F95FEA000801D16448C3E0E7
:100B7000D8F8F80001684A689047B0F5003F17D1EF
:100B8000D8F87C118A68404690478146B9F1810FB8
:100B900080F09E80A94508F1FC0A17D2D8F8F80029
:100BA0000368D3F80CC02A462146E047B0F5003F61
:100BB00040F08E80D8F8F8000368D3F810C06A4679
:100BC0005146E047B0F5003F76D10AE0002004E04E
:100BD000215C0AF800100098401C00900098A84280
:100BE000F6D34FF0000C4749474A484B01AC0098F8
:100BF000844558D2D3E9007001ADC5E90070107882
:100C000000281ABF042086464FF0000E085854F8FA
:100C10000E5028443E4D05600127D0F800E0876063
:100C2000019D4F681AF80C007D408EEA050585F09D
:100C3000040E65680F687D4085F0FC05754485F0FD
:100C4000A30568400AF80C000CF1010CCFE7D3E9CA
:100C5000004501A8C0E9004510782E4D002814BFBA
:100C60004FF0040E4FF0000E01A8744651F80EE04C
:100C70000459A6440127CEF80050DEF80040CEF813
:100C800008704D68019F40687D406C400D68684069
:100C900084F0040480F0FC00041984F057040AF87E
:100CA0000C400CF1010CCC45D1D3D8F8F800016808
:100CB0004A689047B0F5003F0AD1D8F8F8000368B9
:100CC000D3F80C804A465146C047B0F5003F01D0EA
:100CD000114811E0002006E05AF8201081F06A3136
:100CE0004AF82010401CB0EB990FF5D3B06840F0E3
:100CF0000100B0604FF4403004B0BDE8F08700BFA1
:100D000002000300586F0108A00A00202C0F000801
:100D1000ADBE4ED70DBE75A10100030038B50C461F
:100D2000017A1546CA0702D500F014F908B9084837
:100D300032BDD0F8F80003682146DC682A46A04797
:100D4000B0F5003F01D0034832BD4FF4403032BD12
:100D500002000300010003002DE9F84191B00546AF
:100D60000E461746402101A814F071F9297AC807E8
:100D700004D5284600F0EEF8040002D1DFF8A48084
:100D80004BE0D4F8F800DFF8A0800368D3F810C077
:100D90006A4601A9E047B0F5003F3ED1D4F8F8001B
:100DA00001684A689047B0F5003F36D1D4F87C110D
:100DB0008A6820469047D4F8F830024618461B68E7
:100DC000D3F80CC004F1FC01E047B0F5003F24D19A
:100DD000D4F87C0141688847D4F8F83002461846B8
:100DE0001B68D3F80CC001A9E047B0F5003F14D14F
:100DF000D4F8F8000268696893689847B0F5003F36
:100E00000BD1D4F8F80003681C693A463146A04774
:100E1000B0F5003F08BF4FF44038404612B0BDE87F
:100E2000F08100BF02000300010003002DE9F8413A
:100E3000A5B0074688461646402115A814F007F9C4
:100E400000220492402105A814F001F9387AC10764
:100E50005ED5384600F07EF8050059D0D5F8F80088
:100E60002D4C0368D3F810C06A4605A9E047B0F5D9
:100E7000003F3CD1D5F8F80001684A689047B0F5CA
:100E8000003F34D1D5F87C118A6828469047D5F8C0
:100E9000F830024618461B68D3F80CC005F1FC0177
:100EA000E047B0F5003F22D1D5F87C014168884782
:100EB000D5F8F830024618461B68D3F80CC005A9CF
:100EC000E047B0F5003F12D1D5F8F8000268796824
:100ED00093689847B0F5003F09D1D5F8F80003684A
:100EE0001D6904AA15A9A847B0F5003F01D0204606
:100EF0000FE00A4B0A490B4A0396029101924046C1
:100F00001C68049B009415AA796800F0E5F900E0DC
:100F1000054826B0BDE8F08101000300606F0108BC
:100F2000936E030026C703000200030004B0010112
:100F300000170145E90A0008090B00082D0B0008FD
:100F4000BD030008550B00081D0D0008590D0008D1
:100F50002D0E00080168024A914218BF0020704718
:100F6000340F000810B5040008BF002404D0034863
:100F70002060204609688847204610BD340F0008CD
:100F800020225C3014F061B8F0B58468A308002218
:100F900004F0030407E000F15C0555F8226035BA5F
:100FA00041F82250521C9A42F5D300220BE000F186
:100FB0005C0502EB830755F82360D500C5F11805E1
:100FC000EE40CE55521CA242F1D3F0BD30B5C468FC
:100FD00003690022E31AD5188C5C0544521C082AC8
:100FE0002C77F8D330BD0360C1600261704738B51B
:100FF000044615460022626023685A689047002024
:101000006061A061A5604FF4003032BD81604FF493
:10101000003070472DE9F84304462079D4F80C805D
:10102000450748BF244845D466691D46A8F101001C
:1010300000EAD60306EBC506B6EBC50F666102D221
:10104000A669761CA6611746A66906EB5576A661C9
:101050000E46E918884225D2A8EB03094A463146D4
:10106000F81813F0F2FF2268136839460FE0424681
:10107000384613F0EAFF23681A683946204690473D
:1010800007E0311811F00300F1D1226813682046FF
:101090009847484600EB0809A9F10101A942F0D39D
:1010A000002300E000202A1A3118F81813F0CDFFB1
:1010B0004FF40030BDE8F283040002002DE9FC4F3C
:1010C000024685B0D0681369DFF86CC1DFF86C8127
:1010D000A0EB030A506840F004005060002703A80A
:1010E00002900DF10C0ED8E9003403A8544DC0E96C
:1010F00000342878534D00280CBF00230423994660
:101100005CF803305EF80940234401261D601C682A
:101110009E60DCF80430039DDCF80090DEF804608B
:101120005D406540484C654089EA0606474C66408C
:101130007519474C6540D8E9006B03AC0028C4E939
:10114000006B0EBF002404200424029E5CF8000003
:10115000345920183F4C04600126046886600398C7
:10116000029E43406340384C7068634089EA000047
:10117000364C6040034438484340280018BF0120E3
:101180005B1E9B41042F2CBFC0B2D80F02F1140389
:1011900053F8200007F00303C3F10303DB00D8403A
:1011A0000DF807007F1C082F9DD315460C466A6971
:1011B000AB69E868D20842EA4372401E00EA0207BF
:1011C000002302409B420AD8524508D28020E055B5
:1011D0007F1C574516D2AAEB0701E01910E08020CA
:1011E000E05500E0E355E8687F1C8742FAD32A689F
:1011F000136828469847BAF1000F03D0514620469D
:1012000013F025FF2A68069E059F936869462846C5
:1012100098472A68D2F8009021462846C8472B688C
:10122000DA683946284690470EB1A86830604FF416
:10123000003007B0BDE8F08F586F01085C1200085D
:10124000A00A00205FC5109304850012FC68017A93
:10125000C0F524FF24AF33D426AF698B04B001015D
:1012600000170145F8B501240094002300240DE087
:10127000009D065D0F5D7E40F643761CF60F86F0FE
:10128000010635400095641C009DEB189442EFD395
:101290001846F2BDF8B5002301240094002A11E09D
:1012A000009C85188F1815F8016C17F8015C6E40CA
:1012B000F643761CF60F86F0010634400094009C3D
:1012C000E318521EECD11846F2BD0000651200086A
:1012D00095120008010000002DE9F84F1D46DDF8C9
:1012E00028900B9F0D9C4FF0FF3300930E469246C3
:1012F000D9F800B0804632465146D847834664B399
:10130000D9F8043032465146404698476FEA0B02FE
:10131000521C42EA0B0200996FEAD2735B1C19401F
:10132000C2430091521C024300996FEAD2735B1CC6
:101330001940009186F05531484087EA000181F05C
:101340005531216080F05531C943491C0843009A4A
:101350006FEAD070401C82430092D9F8080001283F
:1013600009D17540E943491C0D4300986FEAD572D5
:10137000521C90430AE0F11C85EA9102D243521CB0
:10138000154300986FEAD5735B1C984386F0AA3624
:10139000009086EA0B0686F0AA33F243DB430C98F2
:1013A000C2F3C0725B1C42EAD3720099D243521C52
:1013B00091430091774000998843009987F0AA37BC
:1013C0000F403843BDE8F28F00000000000000002D
:1013D00001F0FF01102A2BDB10F0070F08D010F8E6
:1013E000013B013A8B422DD010F0070F42B3F6D1EA
:1013F000F0B441EA012141EA014122F007047FF003
:1014000000070023F0E80256083C85EA010586EA59
:10141000010685FA47F5A3FA87F586FA47F6A5FA95
:1014200087F68EB9EED1F0BC01F0FF0102F00702A1
:1014300032B110F8013B013A83EA010313B1F8D14C
:101440000020704701387047002D06BF354603382D
:10145000073815F0010F07D1013015F4807F02BF66
:10146000013015F4C03F0130F0BC0138704700BFB7
:10147000034613F8012B002AFBD1181A01387047D4
:1014800081F0004102E000BF83F0004330B54FEA35
:1014900041044FEA430594EA050F08BF90EA020FA2
:1014A0001FBF54EA000C55EA020C7FEA645C7FEA35
:1014B000655C00F0E2804FEA5454D4EB5555B8BF58
:1014C0006D420CDD2C4480EA020281EA030382EAC9
:1014D000000083EA010180EA020281EA0303362D5B
:1014E00088BF30BD11F0004F4FEA01314FF4801C2E
:1014F0004CEA113102D0404261EB410113F0004F40
:101500004FEA03334CEA133302D0524263EB4303F6
:1015100094EA050F00F0A780A4F10104D5F1200E94
:101520000DDB02FA0EFC22FA05F2801841F10001EF
:1015300003FA0EF2801843FA05F359410EE0A5F1C3
:1015400020050EF1200E012A03FA0EFC28BF4CF0F4
:10155000020C43FA05F3C01851EBE37101F00045AA
:1015600007D54FF0000EDCF1000C7EEB00006EEBB7
:101570000101B1F5801F1BD3B1F5001F0CD3490841
:101580005FEA30004FEA3C0C04F101044FEA445298
:1015900012F5800F80F09A80BCF1004F08BF5FEA1F
:1015A000500C50F1000041EB045141EA050130BDFF
:1015B0005FEA4C0C404141EB0101013C28BFB1F511
:1015C000801FE9D291F0000F04BF01460020B1FA5C
:1015D00081F308BF2033A3F10B03B3F120020CDA2F
:1015E0000C3208DD02F1140CC2F10C0201FA0CF00D
:1015F00021FA02F10CE002F11402D8BFC2F1200C72
:1016000001FA02F120FA0CFCDCBF41EA0C01904027
:10161000E41AA2BF01EB0451294330BD6FEA040470
:101620001F3C1CDA0C340EDC04F11404C4F120025B
:1016300020FA04F001FA02F340EA030021FA04F36D
:1016400045EA030130BDC4F10C04C4F1200220FAC4
:1016500002F001FA04F340EA0300294630BD21FA02
:1016600004F0294630BD94F0000F83F4801306BFC8
:1016700081F480110134013D4EE77FEA645C18BFBC
:101680007FEA655C29D094EA050F08BF90EA020F53
:1016900005D054EA000C04BF1946104630BD91EA4B
:1016A000030F1EBF0021002030BD5FEA545C05D14E
:1016B0004000494128BF41F0004130BD14F580048D
:1016C0003CBF01F5801130BD01F0004545F0FE4101
:1016D00041F470014FF0000030BD7FEA645C1ABF36
:1016E000194610467FEA655C1CBF0B46024650EA6D
:1016F000013406BF52EA033591EA030F41F4002199
:1017000030BD00BF90F0000F04BF0021704730B51E
:101710004FF4806404F132044FF000054FF00001F3
:1017200050E700BF90F0000F04BF0021704730B5B4
:101730004FF4806404F1320410F0004548BF404289
:101740004FF000013EE700BF42004FEAE2014FEADE
:1017500031014FEA02701FBF12F07F4393F07F4FB9
:1017600081F06051704732F07F4208BF704793F0BC
:101770007F4F04BF41F40021704730B54FF46074CF
:1017800001F0004521F000411CE700BF50EA0102D2
:1017900008BF704730B54FF000050AE050EA01027B
:1017A00008BF704730B511F0004502D5404261EBEB
:1017B00041014FF4806404F132045FEA915C3FF42C
:1017C000D8AE4FF003025FEADC0C18BF03325FEAC9
:1017D000DC0C18BF033202EBDC02C2F1200300FA7A
:1017E00003FC20FA02F001FA03FE40EA0E0021FA9F
:1017F00002F11444BDE600BF70B54FF0FF0C4CF48D
:10180000E06C1CEA11541DBF1CEA135594EA0C0F3E
:1018100095EA0C0F00F0DEF82C4481EA030621EA79
:101820004C5123EA4C5350EA013518BF52EA0335B4
:1018300041F4801143F4801338D0A0FB02CE4FF066
:101840000005E1FB02E506F00042E0FB03E54FF096
:101850000006E1FB03569CF0000F18BF4EF0010E8E
:10186000A4F1FF04B6F5007F64F5407404D25FEA8A
:101870004E0E6D4146EB060642EAC62141EA55513D
:101880004FEAC52040EA5E504FEACE2EB4F1FD0C7F
:1018900088BFBCF5E06F1ED8BEF1004F08BF5FEAFD
:1018A000500E50F1000041EB045170BD06F00046AF
:1018B00046EA010140EA020081EA0301B4EB5C045C
:1018C000C2BFD4EB0C0541EA045170BD41F4801154
:1018D0004FF0000E013C00F3AB8014F1360FDEBF79
:1018E000002001F0004170BDC4F10004203C35DA55
:1018F0000C341BDC04F11404C4F1200500FA05F3D8
:1019000020FA04F001FA05F240EA020001F0004278
:1019100021F0004110EBD37021FA04F642EB0601EE
:101920005EEA430E08BF20EAD37070BDC4F10C0418
:10193000C4F1200500FA04F320FA05F001FA04F2DC
:1019400040EA020001F0004110EBD37041F10001C8
:101950005EEA430E08BF20EAD37070BDC4F12005D3
:1019600000FA05F24EEA020E20FA04F301FA05F23B
:1019700043EA020321FA04F001F0004121FA04F2E3
:1019800020EA020000EBD3705EEA430E08BF20EAB3
:10199000D37070BD94F0000F0FD101F000464000ED
:1019A00041EB010111F4801F08BF013CF7D041EA6F
:1019B000060195F0000F18BF704703F00046520073
:1019C00043EB030313F4801F08BF013DF7D043EA44
:1019D0000603704794EA0C0F0CEA135518BF95EAFA
:1019E0000C0F0CD050EA410618BF52EA4306D1D181
:1019F00081EA030101F000414FF0000070BD50EAA0
:101A0000410606BF1046194652EA430619D094EA29
:101A10000C0F02D150EA013613D195EA0C0F05D113
:101A200052EA03361CBF104619460AD181EA030167
:101A300001F0004141F0FE4141F470014FF000001F
:101A400070BD41F0FE4141F4780170BD70B54FF0BA
:101A5000FF0C4CF4E06C1CEA11541DBF1CEA13553A
:101A600094EA0C0F95EA0C0F00F0A7F8A4EB05041C
:101A700081EA030E52EA03354FEA013100F0888013
:101A80004FEA03334FF0805545EA131343EA1263DC
:101A90004FEA022245EA111545EA10654FEA002691
:101AA0000EF000419D4208BF964244F1FD0404F54A
:101AB000407402D25B084FEA3202B61A65EB0305A6
:101AC0005B084FEA32024FF480104FF4002CB6EB63
:101AD000020E75EB030E22BFB61A754640EA0C00E3
:101AE0005B084FEA3202B6EB020E75EB030E22BF23
:101AF000B61A754640EA5C005B084FEA3202B6EB64
:101B0000020E75EB030E22BFB61A754640EA9C0022
:101B10005B084FEA3202B6EB020E75EB030E22BFF2
:101B2000B61A754640EADC0055EA060E18D04FEAB0
:101B3000051545EA16754FEA06164FEAC30343EA50
:101B400052734FEAC2025FEA1C1CC0D111F4801F1D
:101B50000BD141EA00014FF000004FF0004CB6E716
:101B600011F4801F04BF01430020B4F1FD0C88BFB5
:101B7000BCF5E06F3FF6AFAEB5EB030C04BFB6EBC0
:101B8000020C5FEA500C50F1000041EB045170BDB3
:101B90000EF0004E4EEA113114EB5C04C2BFD4EBE0
:101BA0000C0541EA045170BD41F480114FF0000E64
:101BB000013C90E645EA060E8DE60CEA135594EAE0
:101BC0000C0F08BF95EA0C0F3FF43BAF94EA0C0FE3
:101BD0000AD150EA01347FF434AF95EA0C0F7FF458
:101BE00025AF104619462CE795EA0C0F06D152EAAC
:101BF00003353FF4FDAE1046194622E750EA410690
:101C000018BF52EA43067FF4C5AE50EA41047FF4A0
:101C10000DAF52EA43057FF4EBAE12E74FF0FF3C05
:101C200006E000BF4FF0010C02E000BF4FF0010CD6
:101C30004DF804CD4FEA410C7FEA6C5C4FEA430C4F
:101C400018BF7FEA6C5C1BD001B050EA410C0CBF9E
:101C500052EA430C91EA030F02BF90EA020F002000
:101C6000704710F1000F91EA030F58BF994208BF67
:101C700090422CBFD8176FEAE37040F00100704724
:101C80004FEA410C7FEA6C5C02D150EA013C07D17B
:101C90004FEA430C7FEA6C5CD6D152EA033CD3D0C6
:101CA0005DF8040B704700BF8446104662468C46C0
:101CB0001946634600E000BF01B5FFF7B7FF0028F3
:101CC00048BF10F1000F01BD4DF808EDFFF7F4FF1C
:101CD0000CBF012000205DF808FB00BF4DF808EDA7
:101CE000FFF7EAFF34BF012000205DF808FB00BFCA
:101CF0004DF808EDFFF7E0FF94BF012000205DF8EC
:101D000008FB00BF4DF808EDFFF7CEFF94BF0120A0
:101D100000205DF808FB00BF4DF808EDFFF7C4FF99
:101D200034BF012000205DF808FB00BF4FEA410CE2
:101D30007FEA6C5C02D150EA013C0AD14FEA430CC5
:101D40007FEA6C5C02D152EA033C02D14FF0000002
:101D500070474FF0010070474FEA410212F5001240
:101D600015D211D56FF47873B3EB625212D94FEAE2
:101D7000C12343F0004343EA505311F0004F23FACC
:101D800002F018BF404270474FF00000704750EA21
:101D9000013005D111F0004008BF6FF000407047DE
:101DA0004FF00000704700BF80F0004002E000BF2D
:101DB00081F0004142001FBF5FEA410392EA030F36
:101DC0007FEA226C7FEA236C6AD04FEA1262D2EB80
:101DD0001363C1BFD218414048404140B8BF5B4285
:101DE000192B88BF704710F0004F40F4000020F01E
:101DF0007F4018BF404211F0004F41F4000121F034
:101E00007F4118BF494292EA030F3FD0A2F101027D
:101E100041FA03FC10EB0C00C3F1200301FA03F1BB
:101E200000F0004302D5494260EB4000B0F5000FDE
:101E300013D3B0F1807F06D340084FEA310102F19D
:101E40000102FE2A51D2B1F1004F40EBC25008BF4F
:101E500020F0010040EA03007047490040EB000019
:101E6000013A28BFB0F5000FEDD2B0FA80FCACF11A
:101E7000080CB2EB0C0200FA0CF0AABF00EBC25047
:101E800052421843BCBFD0401843704792F0000F35
:101E900081F4000106BF80F400000132013BB5E788
:101EA0004FEA41037FEA226C18BF7FEA236C21D0FE
:101EB00092EA030F04D092F0000F08BF0846704763
:101EC00090EA010F1CBF0020704712F07F4F04D131
:101ED000400028BF40F00040704712F100723CBF44
:101EE00000F50000704700F0004343F0FE4040F46E
:101EF000000070477FEA226216BF08467FEA23632C
:101F00000146420206BF5FEA412390EA010F40F416
:101F1000800070474FF0000304E000BF10F0004362
:101F200048BF40425FEA000C08BF704743F0964349
:101F300001464FF000001CE050EA010208BF704764
:101F40004FF000030AE000BF50EA010208BF7047EB
:101F500011F0004302D5404261EB41015FEA010C00
:101F600002BF84460146002043F0B64308BFA3F1F8
:101F70008053A3F50003BCFA8CF2083AA3EBC253DA
:101F800010DB01FA02FC634400FA02FCC2F12002F9
:101F9000BCF1004F20FA02F243EB020008BF20F030
:101FA0000100704702F1200201FA02FCC2F1200296
:101FB00050EA4C0021FA02F243EB020008BF20EA8B
:101FC000DC7070474FEA4002B2F1FE4F0FD34FF082
:101FD0009E03B3EB12620DD94FEA002343F0004396
:101FE00010F0004F23FA02F018BF404270474FF044
:101FF0000000704712F1610F01D1420205D110F0CB
:10200000004008BF6FF0004070474FF0000070477D
:1020100053B94AB9002908BF00281CBF4FF0FF314F
:102020004FF0FF3000F070B9ADF1080C6DE904CE4F
:1020300000F006F8DDF804E0DDE9022304B07047A3
:102040002DE9F047089E0D4604460F46002B4AD165
:102050008A42944665D9B2FA82F343B102FA03FC8C
:10206000C3F120029F4020FA02F217439C404FEA3E
:102070001C4E1FFA8CF5B7FBFEF1220C0EFB1177FC
:1020800042EA074201FB05F090420AD91CEB02022A
:1020900001F1FF3780F01B81904240F21881023934
:1020A0006244121AA4B2B2FBFEF00EFB102244EA04
:1020B000024400FB05F5A5420AD91CEB040400F11B
:1020C000FF3280F00681A54240F203816444023869
:1020D00040EA0140641B00211EB1DC400023C6E938
:1020E0000043BDE8F0878B4208D9002E00F0EC8059
:1020F0000021C6E900050846BDE8F087B3FA83F180
:10210000002949D1AB4202D3824200F2F780841AFF
:1021100065EB030201201746002EE2D0C6E9004716
:10212000DFE702B9FFDEB2FA82F3002B40F08F80C6
:102130008A1A4FEA1C471FFA8CFE0121B2FBF7F501
:1021400007FB1520220C42EA00420EFB05F09042EC
:1021500008D91CEB020205F1FF3802D2904200F2CE
:10216000CA804546121AA4B2B2FBF7F007FB102250
:1021700044EA02440EFB00FEA64508D91CEB040409
:1021800000F1FF3202D2A64500F2BA801046A4EB5D
:102190000E0440EA05409FE7C1F120078B4022FA78
:1021A00007FC4CEA030C05FA01F420FA07F3FD40A2
:1021B000234300FA01F94FEA1C401FFA8CFEB5FBDD
:1021C000F0F81C0C00FB185544EA054408FB0EF51A
:1021D000A54202FA01F20BD91CEB040408F1FF3A04
:1021E00080F08780A54240F28480A8F10208644410
:1021F000641B9DB2B4FBF0F300FB134445EA0444B6
:1022000003FB0EFEA64508D91CEB040403F1FF30C6
:102210006BD2A64569D9023B644443EA0840A0FB5F
:102220000283A4EB0E049C42C6461D4655D352D0F1
:1022300056B1B9EB0E0364EB050404FA07F7CB4083
:10224000CC401F43C6E900740021BDE8F087C3F10C
:10225000200102FA03FC20FA01F225FA01F19D4067
:102260002A434FEA1C471FFA8CFEB1FBF7F007FB2D
:102270001015110C41EA054100FB0EF58D4204FAE0
:1022800003F408D91CEB010100F1FF382FD28D4275
:102290002DD902386144491B92B2B1FBF7F507FB17
:1022A000151142EA014205FB0EF1914208D91CEBDF
:1022B000020205F1FF3816D2914214D9023D624460
:1022C000521A45EA004139E73146304609E73946B6
:1022D000E7E61046FCE6C145AAD2B8EB020E63EB76
:1022E0000C050138A4E74546EAE7034695E7404672
:1022F000D1E7D0467CE7023D624433E708460BE76E
:102300006444023843E700BF704700BF1348144AD3
:1023100008B54FF00043C0E90023042200234261C6
:102320000122C2614FF4805107220383C0E90233C6
:10233000C0E90933C0E90C120361837680F82030CC
:1023400080F82C30826380F83C30C36404F0CCFF0A
:1023500018B1BDE8084000F00BBC08BDA40A00207D
:10236000002401400268084B9A4282B00AD14FF023
:10237000B0431A6E42F400721A661B6E03F40073C7
:102380000193019B02B07047002401400268054B95
:102390009A4201BF4FF0B042136E23F400731366EC
:1023A000704700BF0024014030B585B000240546C9
:1023B000CDE901440394FFF7A9FF144805F02CFB75
:1023C00008B100F0D5FB1148039401A9CDE90154EF
:1023D00005F0E8F808B100F0CBFB0C4805F046FA30
:1023E00008B100F0C5FB4FF0FF31084805F07CF85C
:1023F000064805F0F3FA054805F0D0F8044603480E
:1024000005F096FA204605B030BD00BFA40A0020B2
:10241000014B024A1A607047A40A002000240140C0
:1024200008B50948FFF7C0FF68B1084BB3F8AA30F8
:102430004FF6FF72934216BF40F6E442044B5343FB
:10244000B3FBF0F398B208BD002000B40075FF1F85
:10245000D8084C0013B50023ADF80630FFF7E0FFB5
:1024600004461948FFF7A0FF184BB3F8C820B3F88B
:10247000A8108A4204FB00F018D040F6E443B0FBF9
:10248000F3F364205B1A4343521A93FBF2F31E33B7
:102490001BB2ADF80630BDF806305BB21B02ADF8DA
:1024A0000630BDF8060000B202B010BD4FF47A72DB
:1024B00040F6FF73B0FBF3F35343A3F53923A3F5C1
:1024C0000C6340F6C412E0E7001000B00075FF1F77
:1024D0004FF0B04382B09A6A22F480529A629A6CAA
:1024E00042F480529A649B6C03F480530193019BE5
:1024F000002002B070474FF0B04382B09A6C0243A4
:102500009A649B6C03400193019B02B0704708B52D
:102510000420FFF7F0FF0120FFF7EDFF0220FFF797
:10252000EAFF002211460B2005F014FB0B2005F0FA
:1025300043FB002211460C2005F00CFB0C2005F09B
:102540003BFB002211460D2005F004FB0D2005F099
:1025500033FB002211460E2005F0FCFA0E2005F098
:102560002BFB002211460F2005F0F4FA0F2005F096
:1025700023FB00221146112005F0ECFA112005F092
:102580001BFB00223620114605F0E4FABDE80840A6
:10259000362005F011BB000008B505F055FD10B15F
:1025A0006FF0040008BD064B9A6942F040429A6100
:1025B0004CF2FA321A6105F059FD0028F2D0EFE72B
:1025C00000400058F0B585B000230C460093064645
:1025D000A8B3FFF7E1FF054670BB05F035FD88BBEA
:1025E0001A481B4A02230193D0F8E01506F17843FC
:1025F00002EA8121B3FBF1F701FB1733DB0A0293F7
:10260000D0F8E00504F178410139314402EA802232
:10261000B1FBF2F002FB1011C3EBD1230133694689
:1026200001A8039305F0A2FD20B102280CBF0125EB
:102630006FF0010505F01AFD284605B0F0BD6FF0FA
:102640000505F9E76FF00405F6E700BF0070FF1F0E
:1026500000FCFF03014B186000207047080B0020AE
:102660002DE9F04F89B0B0F1006F06460F46009299
:10267000C0F0C580DFF89881664DD8F8E03505EAEE
:10268000832303F10063013B984200F2B8800028E5
:1026900000F0B880002900F0B58040EA02035B0733
:1026A00040F0B080FFF778FF0446A0BB05F0CCFCFB
:1026B000002840F0AA80D8F8E01506F1784205EA33
:1026C0008121B2FBF1F301FB1322009B03F178435C
:1026D000013B3344B3FBF1F001FB1033DB0A013360
:1026E0004FEAD22AA3EBD222012A039388BFC6F372
:1026F0000A050AF58038C6F1080398BF009D0693C5
:1027000088BFC5F500654FEAC828B346039B9A45C4
:1027100005D305F0ABFC204609B0BDE8F08FA6F16B
:102720000803069A1A44954219D804950197CDF8E2
:1027300014B04FF00009059B09EB0301049B994578
:102740003ED3009BAB442F445D1BB5F5006F28BF03
:102750004FF400650AF1010A08F50068D6E753F85E
:10276000081F5A68B2F1FF3F08BFB1F1FF3FD8D050
:10277000294B186810B96FF00504CAE7B8F1000FCB
:1027800004D04FF40062414611F040FADFF888901F
:10279000D9F80030CBF30A0039461844AAB211F038
:1027A00035FA4FF400614046FFF70CFF08BBD9F83B
:1027B000003001934FF40063CDF814800493B8E720
:1027C000019B07914B4402930120D3E9002305F0BC
:1027D00087FC88B90799019BD1E9000259F80310D9
:1027E000029B5B689A4208BF884205D109F108093B
:1027F000A1E76FF001048CE76FF0030489E74FF065
:10280000FF3488E76FF0050485E76FF0040482E782
:102810000070FF1F00FCFF03080B0020B1F1006FE8
:1028200070B511D30B4BD3F8E0650B4B03EA86234D
:1028300003F10063013B994206D840B139B192B22D
:1028400011F0E4F9002070BD4FF0FF30FBE76FF0AE
:102850000500F8E70070FF1F00FCFF03B0F1006FF8
:1028600010B40DD3084BD3F8E045084B03EA84239A
:1028700003F10063013B984202D810BCFFF7A2BEEF
:102880004FF0FF3010BC70470070FF1F00FCFF03CB
:102890004FF0B04382B0DA6C0243DA64DB6C034081
:1028A0000193019B02B0704770B586B014220021DD
:1028B00001A812F042FB0120FFF7EAFF0220FFF718
:1028C000E7FF0420FFF7E4FF4FF4007101224FF00F
:1028D000904005F0BFFD012502234FF4041401A927
:1028E0004FF09040CDE90134224E039505F08CFC69
:1028F0004FF4441301A94FF09040CDE90235019502
:1029000005F082FC2023CDE9013401A900243046E2
:10291000039405F079FC4FF4007301A94FF0904047
:10292000CDE90135CDE9035405F06EFC04230DEB30
:1029300003013046CDE90135CDE9034405F064FCDF
:1029400022462146062005F005F9062005F034F957
:1029500022462146072005F0FDF8072005F02CF956
:1029600022462146162005F0F5F8162005F024F938
:1029700006B070BD0004004808B51248124A134B57
:10298000C0E9002300230122C0E90232C0E9043378
:10299000C0E90633036205F0D1FE08B100F0E8F8A3
:1029A0000848002106F04AF808B100F0E1F80548AF
:1029B000002106F069F818B1BDE8084000F0D8B869
:1029C00008BD00BFCC0B0020005800405D3E302009
:1029D00070B596B005461422002103A812F0ADFA96
:1029E0003822002108A812F0A8FA2A68304B9A422F
:1029F0005BD18023089308A84FF440230E9306F080
:102A00009FFD08B100F0B4F84FF0B0444FF4C0504F
:102A1000E36C43F00103E364E36C03F0010302930E
:102A2000029B12230026CDE903030323CDE90563AE
:102A30004FF09040042303A9079305F0E5FBA36D35
:102A4000DFF870C043F48003A365A36D1A4C03F450
:102A500080030193019B26620D23C4E900C3204635
:102A60008023C4E90266C4E90436C4E9066605F0B9
:102A700003F908B100F07CF8104AEC63A562104C31
:102A80000E23C4E900231021002380222046C4E93C
:102A90000213C4E90423C4E90633236205F0ECF809
:102AA00008B100F065F8AC63A56216B070BD00BF58
:102AB00000580040440002400C0B00205800024027
:102AC0006C0B002000B59BB04822002108A812F032
:102AD00034FA1822002102A812F02FFA05F0FAFFAA
:102AE0004FF0B0420120D2F8903023F01803C2F822
:102AF0009030D2F8003423F4C06343F40073C2F87A
:102B00000034D2F8003403F4C0630193019B242302
:102B1000089381230B930023CDE91003B02208A86A
:102B2000CDE9122306F04EF908B172B6FEE74F2345
:102B3000CDE90230CDE90400CDE90600022102A86A
:102B400006F0DAFB08B172B6FEE71BB05DF804FBD5
:102B500008B504F077FBFFF7B5FFFFF7A5FEFFF719
:102B6000D6FCFFF709FF00F0ECFD00F0F1FDFCE7FB
:102B700072B6FEE700B58DB02C22002101A812F03C
:102B8000DCF91748174B03601F2383604FF0804226
:102B90000023C0E90433C0E9072383614FF4807345
:102BA000436206F053FE08B1FFF7E2FF0C4806F05F
:102BB00079FF08B1FFF7DCFF4FF0005300220793C5
:102BC000074808924FF4807301A9029206920B9372
:102BD00006F09CFE08B1FFF7CBFF0DB05DF804FBDB
:102BE000200C00200028004010B5044690B0382288
:102BF000002102A812F0A1F92268194B9A422CD1A7
:102C00004FF48033029302A84FF480730F9306F0C1
:102C100097FC08B1FFF7ACFF4FF0B0430220D3F8A8
:102C2000902042F40042C3F890209A6D42F48062F2
:102C30009A659B6D002203F4806311460193019B0A
:102C400004F088FF022004F0B7FF00222A2011467A
:102C500004F080FF2A2004F0AFFF10B010BD00BFC9
:102C6000002800407047000008B504F001FB044B49
:102C70000120C3F88800BDE8084005F083BF00BF0D
:102C80000004005804F0FBBA08B504F0F8FA00F0AC
:102C90008BFCFFF709FEFFF73AFCBDE80840FFF7A1
:102CA0006BBE08B504F0E4FABDE80840012100203D
:102CB00005F018BF70477047FEE7FEE7FEE7FEE746
:102CC000FEE770477047704770470000014806F004
:102CD0000FBF00BF200C0020012005F0C1BB022067
:102CE00005F0BEBB70477047014805F03FB900BF13
:102CF0000C0B0020014805F039B900BFA00C0020E2
:102D00007047FFF7F7BF7047202005F0A9BB704759
:102D1000014807F0B1BA00BF000D0020014806F0DD
:102D200019BD00BF200C0020014807F00CB900BFFE
:102D3000840C00202DE9F04389B080460020109ECD
:102D40000790894615461F46FDF772FAF0B9104CF8
:102D5000CDE90090CDE9020407AB0E48059314239A
:102D600004933A46434629460068FDF72BFB234669
:102D7000324604F1140153F8044B42F8044B8B42E1
:102D8000F9D1079B337509B0BDE8F0830120FAE75C
:102D9000580C0020546F01081FB50E4C00233C2234
:102DA00002A8CDE902336275237500F0B9F8042357
:102DB00003AA009412210848FFF7BCFF0749142218
:102DC000204612F0AAF8B0FA80F35B09637504B0EC
:102DD00010BD00BF6C0C00207C6F0108AE0F0020FE
:102DE000054808B50823036006F0C8FE18B1BDE821
:102DF0000840FFF7BDBE08BD840C00204FF0B04373
:102E000007B55A6E42F001025A665B6E002203F06B
:102E10000103019311463220019B04F09BFE3220F6
:102E200003B05DF804EB04F0C7BE00000CB407B5B6
:102E3000054A05AB1021019311F0F2F903B05DF8DA
:102E400004EB02B0704700BF8E6F010830B585B04B
:102E5000044602A80D4611F00FF8BDF90C30064AE1
:102E600000931021029B2046FFF7E0FF2046FEF76B
:102E7000FFFA288005B030BD8E6F01084FF0B042D8
:102E800010B5936823F40043936011F07DF80E4B66
:102E900001241C7000F0B6F810F046FD0B4810F04D
:102EA0005DFD0B4B4FF400421A61002010F05CFDF9
:102EB000FFF7AEFA00F012F910F052FE20460021A2
:102EC000BDE8104010F06CBE900C00204D2E0008A4
:102ED0000040005810F07ABE08B5FFF7A1FA40F69E
:102EE000B83398420CD8B0F5E16F0BD3FE23A0F5B0
:102EF000E16058434FF49663B0FBF3F0C0B208BDF5
:102F0000FE20FCE70020FAE77FB5684600F0CAF82B
:102F10000198FFF757F800B207B05DF804FB000016
:102F2000194A38B5D2F88035591C044619D104F035
:102F3000ADF9054604F0B6F9054404F0ADF92B0EE1
:102F4000E3712B0CA3712B0A6371030EE370C0F3C2
:102F50000742C0F307232571C0B2A27063702070CE
:102F600038BD190AC3718171190C1B0E41710371AF
:102F7000D2F88435C370D2F88405C0F30722C0F3B9
:102F80000743000EE9E700BF0070FF1F38B5094B8B
:102F9000D3F8803503600133054609D104F076F992
:102FA000044604F079F9444004F07CF944402C6074
:102FB00038BD00BF0070FF1F0121022010F0DABDF4
:102FC0000021022010F0D6BD00207047024B187877
:102FD00008B100F013B97047900C002082B0019046
:102FE000019802B000F0A6B94FF0B04382B0DA6C9D
:102FF00042F00202DA64DB6C03F002030193019BEE
:1030000002B070472DE9F043254C87B004F050F929
:1030100004F056F904F05CF90123002502934FF403
:103020008059032301A9204604934FF400580395C7
:103030000595FFF7D9FFFFF7D7FFFFF7D5FFFFF79C
:10304000D3FFCDF8049005F0DFF801A920464FF436
:103050000067CDF8048005F0D7F801A920464FF4A9
:103060000046019705F0D0F801A92046019605F029
:10307000CBF82A464946204605F0ECF92A46414657
:10308000204605F0E7F92A463946204605F0E2F9E0
:103090002A463146204605F0DDF907B0BDE8F08349
:1030A0000004004810B50446FFF7D4F9074BA360AD
:1030B00040F30F20FEF732FF054B064A2360064B14
:1030C0006060C4E90323002010BD00BF0000484237
:1030D00000007A440D093E00AB0305000020704754
:1030E0000120704708B511F07BFF162303604FF0F5
:1030F000FF3008BD08B511F073FF16230360FEE72B
:1031000070B50D4614460E46731B9C4201DC2046EA
:1031100070BDAFF3008006F8010BF5E770B50D4602
:1031200014460E46731B9C4201DC204670BD16F807
:10313000010B04F06FF8F5E74FF0FF3070474FF4E4
:1031400000534B60002070470120704700207047FB
:103150000B4A116810B5034609B90A491160106895
:1031600009490A4C0344091B8B4206D911F038FF68
:103170000C2303604FF0FF3010BD1360FCE700BF6D
:10318000940C0020103000200000012000080000F6
:10319000014B1868704700BF9C0C0020032070474B
:1031A00008B501464FF47A7200238002890DFEF7BC
:1031B0002FFF08BD4FF47A73A0FB0303800A40EA97
:1031C00083507047034B98689A689042FBD1C04384
:1031D000704700BF0028004008B5FFF7F3FF014B20
:1031E000186008BD9C0C002008B5FFF7EBFF024BF0
:1031F0001B68C01A08BD00BF9C0C0020024B187849
:1032000008B1FFF7DFBF7047980C002010B5074BDF
:10321000074C0122DA654FF48071204606F060FA0F
:103220004FF0FF332363002010BD00BF0028004093
:10323000200C002002460021014806F06ABC00BFB5
:10324000200C002002460121014806F062BC00BFAC
:10325000200C002010B58CB02C220021044601A8BF
:1032600011F06BFEFFF7D2FF0C4B0D481B681C449E
:103270000023089306934FF00053E4430793012281
:103280004FF4807301A902940B9306F03FFB08B141
:10329000FFF76EFC00200CB010BD00BF9C0C00209E
:1032A000200C002038B50546FFF78CFF02210446AC
:1032B000074806F035FCC4F309024FF47A71A2FB0B
:1032C0000121920AA30A2A8043EA805038BD00BF38
:1032D000200C00200148002106F022BC200C002018
:1032E0000148012106F01CBC200C0020F8B50F4D50
:1032F0002E78CEB90E4C4FF0FF372763FFF73AFC1C
:10330000FFF784FF4FF48071204606F0E9F920466C
:10331000276306F0A9FB32462046022106F0F9FB9E
:10332000FFF75AFF01232B700020F8BD980C0020F6
:10333000200C0020014610B54FF47A720023800261
:10334000890DFEF765FE0146FFF73CFF0446FFF7D7
:1033500039FF031B8B4200D310BD00BFF7E710F00D
:103360001BBF000010B5064C0221204606F0D8FB1A
:103370000221421C2046BDE8104006F0CABB00BF37
:10338000200C00201648174A08B54FF4E133C0E975
:10339000002300230C22C0E90233C0E90523C0E961
:1033A0000733C0E90933036107F099FD08B1FFF75E
:1033B000DFFB0B48002107F00EFF08B1FFF7D8FB39
:1033C0000748002107F027FF08B1FFF7D1FB0448A9
:1033D00007F0E1FE18B1BDE80840FFF7C9BB08BD22
:1033E000000D00200044004070B596B0064614223F
:1033F000002103A811F0A1FD3822002108A811F036
:103400009CFD3268274B9A424AD10223089308A8B0
:10341000254B0A9306F094F808B1FFF7A9FB4FF08B
:10342000B04300259A6D214C42F400329A659A6DA2
:1034300002F400320292029ADA6C42F00102DA647B
:10344000DB6C03F001030193019B0C220223CDE905
:1034500003230323CDE9055303A907234FF090402D
:10346000079304F0D1FE124925621423C4E9001326
:103470001023C4E9023520468023C4E90435C4E999
:10348000065504F0F9FB08B1FFF772FB2520F4673D
:1034900000220221A66204F05DFB252004F08CFBD3
:1034A00016B070BD0044004004000C00A00C0020C9
:1034B0008000024002680C4B9A4210B5044612D1BB
:1034C0004FF0B0420C21936D23F4003393654FF01D
:1034D000904004F045FFE06F04F042FCBDE810406E
:1034E000252004F077BB10BD0044004008B50A4613
:1034F0000146024806F024FE002008BD000D002011
:1035000013B5114B114C18604FF40013009302AB2C
:1035100013E90600204607F0E2FD2368DA69D103CB
:10352000FCD4DA695202FCD59A68084842F4800259
:103530009A6007F01AFE06490448012207F088FD48
:10354000002002B010BD00BF940D0020000D00202F
:103550009C0D002008B5074B1860FEF7D8FFFFF759
:1035600011FF054AD2F8803043F00063C2F8803082
:10357000002008BD980D00200008005808B54FF045
:10358000B04308489A6B42F400329A639A6B22F473
:1035900000329A63FFF78EFF0F2004F01BFB002020
:1035A00008BD00BF000D002008B5074807F097FCD4
:1035B00008B1FFF7DDFA054804F05EFB18B1BDE87D
:1035C0000840FFF7D5BA08BD000D0020A00C002070
:1035D0000268044B9A4203D1034B00201B68184732
:1035E000704700BF00440040980D002002680B4B5C
:1035F0009A4210B504460FD1094B1B682BB1D0F885
:10360000902012B907480121984720460549BDE896
:103610001040012207F01CBD10BD00BF0044004057
:10362000940D00209C0D002002480122102104F07E
:1036300011BF00BF0004004802480022102104F01E
:1036400009BF00BF0004004810B50A4C23780BB92D
:10365000E37C6BB1FFF7A0FB0038074B18BF0120DC
:10366000400018701B78022B02BF00232370E37404
:1036700010BD00BFAE0F0020A40D002038B5114CC6
:103680002378F3B9E37CE3B90F4D2B68012B07D9FD
:103690002B68042B04D80D4A0421012000F014FAF1
:1036A0002B68042B0DD9FFF777FB0038084B18BFA8
:1036B0000120400018701B78022B02BF00232370EA
:1036C000E37438BDAE0F0020A00D0020E86F0108A4
:1036D000A40D002008B5FFF7A7FF01F0F7F9BDE83A
:1036E0000840FFF7A9BF022801D8FFF79DBF704728
:1036F000022801D8FFF7A0BF70470000022808B5D4
:103700001BD8012210210D4804F0A4FE3220FFF73F
:1037100065FC0A480022102104F09CFE01221021C1
:10372000064804F097FE3220FFF758FCBDE8084039
:1037300002480022102104F08DBE08BD000400489C
:10374000704708B5FFF79AFBBDE8084000F062BB80
:103750004FF0FF3010F09EBA70477047704700007E
:10376000014BD870704700BF5C000020014B1874FB
:10377000704700BF5C00002020B1037813B10248FD
:1037800010F0B8BC704700BFE40E002008B502205E
:10379000002110F047FABDE80840014810F0AABC2B
:1037A000FC0E00200021012010F03CBA10B5094C9D
:1037B00060B12060084810F04FFC2168064810F006
:1037C000D3FCBDE81040044810F094BC42F21073E2
:1037D0002360EFE774000020FC0E002010B5094CB8
:1037E000206023680BB9084B2360084810F034FCB4
:1037F0002168064810F0B8FCBDE81040034810F0FE
:1038000079BC00BF0C000020A0860100140F00202E
:1038100038B504460D4607484FF40061FFF71EF81F
:1038200030B92A4621460348BDE83840FEF718BFA4
:1038300038BD00BF00F003080A460149FEF7EEBF9D
:1038400000F0030838B50C4810F006FC08F048F901
:1038500060B90A4C0A480125257007F0D3FF20788B
:10386000294607F025FD044810F044FCBDE8384027
:10387000044810F03FBC00BFFC0E002000000020F8
:103880005C000020CC0E002008F0C6B930B585B031
:10389000FFF722FB044607F001FE054680B1002435
:1038A000354810F0D9FB354B33481968A14238BF71
:1038B000214610F059FC304810F01CFC05B030BD1A
:1038C000684600F0E5FF23B203EB4303FE2203EB5F
:1038D0004313B3FBF2F32A4A0B21117029495068B4
:1038E0000978DBB28DF80C30017050684570506873
:1038F0001A24847050680124C47050680371224BEC
:10390000187840B11D700C231370536861F07F016B
:103910001970052314E01D4B1D48197811B9017861
:103920000029F6D0002101701970536802215971E5
:10393000BDF800305168180A88715168CB710823AE
:103940001449154C0978012988BF00235370637A04
:1039500033B107F08FFD012802D1204610F07CFB27
:103960000E4B0748D978002207F0AEFD063096D1FD
:1039700007F07AFD044693E7FC0E00207400002057
:1039800004000020970E00202C0F0020C30F002001
:10399000AD0F0020A40D0020980E00205C00002038
:1039A00008B5104B0122002102201A7010F03AF9DC
:1039B0000D4810F09FFB0D4B1B788BB10C4B1A7808
:1039C00072B9DB7C63B90B4B1A68042A9EBF1A6874
:1039D00001321A600021BDE80840102010F022B921
:1039E00008BD00BF2C0F0020140F0020C80E0020BF
:1039F000AE0F0020A00D0020044B1B78022B03D13A
:103A00000021082010F00EB9704700BF0000002010
:103A100008B508F06EF880B907F02CFD01280CD12C
:103A2000BFF34F8F0549064BCA6802F4E0621343A7
:103A3000CB60BFF34F8F00BFFDE708BD00ED00E096
:103A40000400FA0510B5044690B190F906307BB930
:103A5000084810F001FB084BE2791A70074B186810
:103A6000FFF7BCFE064BBDE810401868FFF79EBE8E
:103A700010BD00BF980E0020C80E00200C000020D2
:103A8000740000207047704770477047022808B5DF
:103A900001460FD0202810D0012811D14FF09040BE
:103AA00004F0D2FC01280BD100210220BDE808401F
:103AB00010F0B8B800210820F8E7024B01221A7074
:103AC00008BD00BF2810002070B505460C461646FC
:103AD00007F0E4FC0346002834D000241A4810F014
:103AE000BBFA1A4B18481968A14238BF214610F09A
:103AF0003BFBBDE87040144810F0FCBA4A68F05C2B
:103B0000D0540133DAB29442F8D8114B0D701B78BF
:103B1000012B88BF00244C700E4C637A33B107F040
:103B2000A9FC012802D1204610F096FA0A4B0B4856
:103B3000D978002207F0C8FC0630CED107F094FCFB
:103B40000446CBE70549DDE7FC0E002074000020A9
:103B5000A40D0020980E00205C000020040000202E
:103B6000044B1B7823B9044A05210120FFF7ACBFA1
:103B7000704700BFA40D0020ED6F010810B50024B0
:103B800090B03C22214601A8009411F0D6F92F4BA9
:103B90002022DA7219788DF8001059788DF801100A
:103BA00099788DF80210D9788DF8031019798DF86D
:103BB000041059798DF8051099798DF80610D97986
:103BC0008DF80710197A8DF80810597A8DF80910B8
:103BD000997A8DF80A108DF80B2021460DF10B0211
:103BE00058180131007B02F8010F1C29F8D193F815
:103BF00028208DF8282093F829208DF8292093F883
:103C00002A208DF82A2093F82B208DF82B2093F86A
:103C10002C206AB193F83F2052B10DF12B01002204
:103C20009818013290F82C0001F8010F142AF7D1EE
:103C300007484FF40061FEF711FE20B90448402206
:103C40006946FEF70DFD10B010BD00BF78000020E2
:103C500000F80308014940220FF0D8BF00F803081C
:103C600070B52A4D28796B794D2BC0B233D1C0EB9A
:103C7000001080000A2838BF0A204FF47A73584396
:103C8000234BAC791860EB794D2BE4B22BD1C4EB0C
:103C90000414A40095F82C301E4E63BB95F83F30F9
:103CA0004BBB42F21070FFF781FD3068FFF796FDC5
:103CB0002B7A194A1949DBB213706B7A184ADBB2B6
:103CC00013700023EA1892F82C20D2B2CA540133A0
:103CD000142BF7D170BD6B79482B0ABF4FF4616389
:103CE0006B795843C6E7EB79482B0ABF4FF4616301
:103CF000EB795C43CEE7FFF759FD012C38BF012477
:103D00004FF47A735C433460CFE700BF7800002043
:103D1000740000200C000020C20F0020AE0F002015
:103D2000A40D002010B590B000213C2201A8009104
:103D300011F003F94022344968460FF067FF9DF8FF
:103D400000203AB99DF801001A2803D19DF802100D
:103D500001290ED0FFF712FF2C48142200210FF08A
:103D60005FFF4FF47A70FFF739F9FFF779FF10B072
:103D700010BD274B1A70587099709DF80310D970B8
:103D80009DF8041019719DF8051059719DF80610E1
:103D900099719DF80710D9719DF8081019729DF856
:103DA000091059729DF80A1099729DF80B1001F0D4
:103DB0003F01D972D87AD1B288421BD89DF8282009
:103DC00083F828209DF8292083F829209DF82A20AF
:103DD00083F82A209DF82B2083F82B200DF12B014E
:103DE00000229818013211F8014F80F82C40142A53
:103DF000F7D1BAE701F140006844194410F8340CD7
:103E000008730132D6E700BF00F80308AE0F0020A8
:103E1000780000201FB5002403A92046039407F072
:103E20004BFE03A9012007F047FE384B38480094A9
:103E300022464FF4FA7110F0B1F8364B3648009430
:103E400022464FF4FA7110F0A9F8344B344800942C
:103E500001224FF4FA7110F0A1F82046FEF7FAFBA8
:103E600008B1FEF785FE2F4B009400224FF4FA6153
:103E70002D4810F093F82D4A002101200FF08EFFFD
:103E80002B4A002102200FF089FF2A4A002104203A
:103E90000FF084FF284A002108200FF07FFF00F078
:103EA0007DFB2649264807F0BDFD264807F0AAFC01
:103EB0001B4810F01FF9244B0021187807F0F8F97F
:103EC00022490094224B09682248002210F066F82B
:103ED000204810F00FF9FFF725FF1F4A002110209E
:103EE0000FF05CFF1D4A00214FF480700FF056FF69
:103EF0001B4B1C4819681C4B0094002210F04EF814
:103F0000184810F0F7F804B010BD00BF893A000857
:103F1000E40E00208B3A0008B00E0020853A00081D
:103F2000980E0020F9390008CC0E0020FDB50008DD
:103F30008D38000889380008453800080000030162
:103F4000100000205C000020000000207400002011
:103F50008D370008FC0E00207D360008D53600089D
:103F60000C000020140F0020A139000810B5002417
:103F7000A2B021467C2203A8029410F0DEFF532356
:103F80008DF808304FF48D73ADF80A300123ADF889
:103F900004408DF80C30FEF79FFF00B200EB4000AC
:103FA000FE2300EB4010B0FBF3F08DF80D0001A8EC
:103FB00000F07EFC072498B958238DF80E3030228B
:103FC0008021164810F0B9FF224602A9134811F0CB
:103FD00041F8124A21460120FFF776FD22B010BDBC
:103FE0008DF80E408DF80F0000F070FD0C4B1A6834
:103FF00012128DF810201A688DF811205A681212CA
:104000008DF812205A688DF813209A689B688DF8F5
:10401000153012128DF814200E24D0E72D0F002039
:104020005410002030B50378592B91B0044640F06D
:10403000E881052959D84378443B162B55D8DFE849
:1040400013F026015400160154001E0154005400C0
:1040500054005400880054000101540054005400DE
:104060008F0154005400A400540054005400170061
:104070008578482D11D1B14A14210120FFF724FD84
:1040800041F28830FEF7AAFF40F6B830FEF7A6FFEF
:1040900011B0BDE83040FFF7BBBC532D0ED130222C
:1040A0008021A74810F049FFFFF760FF41F28830F8
:1040B000FEF794FFA24A152101207BE0432D16D183
:1040C000002468468DF8004007F014FB9C4A4C23FE
:1040D00013701A2393709DF80030547001204133FF
:1040E000D07013710521FFF7EFFC11B030BD442DE6
:1040F000FBD1934C592323705A236370A57000F0B1
:10410000B8FB2C228021201D10F017FF0023257002
:10411000637001251A23A370E5702571FEF7DCFE9C
:104120008849FE23B0FBF3F04B6864229BB2B3FBDB
:10413000F2F3A3714B6800EB40009BB200EB401020
:10414000B3FBF2F102FB11336071E37122460821E7
:10415000B2E78378303BDBB2092BC6D87A497B4A79
:104160000B700B78DBB25372754A592313704D23D1
:1041700053700B783033937003210120FFF7A4FCB8
:1041800011B0BDE83040FFF7F9BC8578482D16D155
:104190006B4A56231370002353701A239370032322
:1041A0001371182353710223012093711523D070CA
:1041B000D371082111B0BDE83040FFF785BC432D15
:1041C00093D15F4C00213C2201A8009110F0B5FE74
:1041D0006846FFF73FFD2422802104F10C0010F017
:1041E000ACFE9DF8003063709DF80130A3709DF81F
:1041F0000230E3709DF8033023719DF80430637141
:104200009DF80530A3719DF80630E3719DF80730E5
:1042100023729DF80830257063729DF80B509DF84D
:104220000930A3729DF80A30E3722A4603A9257368
:1042300004F10D0010F00EFF05F10D012246C9B288
:10424000012050E7807839280CD83038C0B2FFF709
:104250004AFA3B4A2378137063785370A3789370BB
:10426000032129E711B0BDE83040FFF779BC807821
:104270003928F7D83038C0B2FFF73AFAE9E7807842
:104280003928EFD83038C0B2FFF738FAE1E7837841
:10429000303BDAB2092AE5D8C0783038C2B2092AF0
:1042A000E0D82179A1F14802D2B20B2ADAD8284D00
:1042B00045FA02F2D507D5D40A224D2902FB0300A4
:1042C00036D13C2358434FF47A735843214B18603E
:1042D000214B1860FFF76AFA194A23781370637844
:1042E0005370A3789370E378D37023791371052109
:1042F0000120FFF7E9FB154B00221A701A225A70B1
:1043000001229A70DA70A278303A02EB8201E278E8
:10431000303A02EB4102D2B21A7122795A710F4A35
:104320001278D2B21A72084A1278D2B25A7227E7B9
:104330004829C8D14FF46163C4E700BFF36F010897
:104340002D0F002054100020A40D00207800002024
:10435000DEF7FFFF740000200C000020C20F0020D9
:104360008278303AD3B2092B3FF67CAFC378303B2A
:10437000D9B209293FF676AF0079A0F14801C9B258
:104380000B293FF66FAF624D45FA01F1C9073FF5C2
:1043900069AF0A214D2801FB02332DD13C22534342
:1043A0004FF47A7253435B4A13601068FFF716FAB2
:1043B000594A2378137063785370A3789370E37825
:1043C000D3702379137105210120FFF77DFB534B37
:1043D00000221A701A225A7001229A70DA70A2789A
:1043E000303A02EB8201E278303A02EB4102D2B27B
:1043F0009A712279DA7192E74828D1D14FF461623B
:10440000CDE7502B48D102297FF66FAE4378303B81
:10441000012B3FF66AAE8378312B7FF466AE0B2911
:1044200004D8FFF79DFB00213B4A45E63B4D023493
:10443000002214F8013FA918303B0132DBB20C2AEC
:104440000B73F6D1FFF77CF9334B50221A211A7007
:104450009970002201215A70D97003F8041FA9181D
:104460000132097B0C2A01F1300103F8011FF6D15A
:1044700000232B701A236B700123AB70EB70284B59
:104480001B78DBB22B72274B1B78DBB26B72EA72A4
:10449000FFF774FB1121C7E7412B7FF426AE437869
:1044A000432B7FF422AE16297FF41FAE1E4D421C13
:1044B000002312F8011FE9540133142BF9D1FFF73F
:1044C000C3F81A4B5B7D012B19D114490023EA5C18
:1044D000C8180133D2B2142B80F82C20F7D1114B1D
:1044E00000221A701B78DBB24B72FFF747FB0A4AB7
:1044F000631E1534A34206D1074A1621DCE5094B99
:1045000002221A70F3E713F8011F02F8011BF1E70A
:10451000DEF7FFFF0C0000202D0F002078000020A8
:10452000C20F0020A40D0020AE0F00206C0C002054
:1045300038B504460D4661B316480FF0DBFD2B7805
:104540003BB334B36068237818B3032B0CD00B2B28
:1045500017D0022B1DD1617801291AD00B0618D46F
:10456000BDE83840FFF75EBD6378012B11D10078BC
:10457000012802D0022800D058B9BDE8384007F021
:104580006FB86378012B04D10378034A03F0010369
:10459000137038BDB00E0020970E0020034B002290
:1045A000C3E902220122C3E900227047C40F0020A0
:1045B00000487047C40F00204FF0B04382B0DA6C5F
:1045C0000243DA64DB6C03400193019B02B0704745
:1045D0002DE9F04186B000240220154D0594FFF727
:1045E000EBFF0420FFF7E8FF124F03944FF48076AF
:1045F00001230DEB0001CDE9016328460323049359
:104600004FF4005803F000FE01A93846CDF80480AD
:1046100003F0FAFD22464146384603F01BFF2846C8
:104620002246314603F016FF204606B0BDE8F08171
:104630000004004800080048032810B50ED80128DF
:1046400010D868B902460B484FF4807103F002FF9E
:10465000002209484FF4005103F0FCFE002010BD79
:104660000122F0E7002203484FF4807103F0F2FECC
:104670000122EEE7000400480008004802207047CD
:10468000002070470120704700280CBF0F20162023
:10469000704700000D48854602F0D2FD0C480D49D8
:1046A0000D4A002302E0D458C4500433C4188C428D
:1046B000F9D30A4A0A4C002301E013600432A242F3
:1046C000FBD310F093FCFEF743FAFEE70000012055
:1046D00000000020840A00208C7E0108840A00204B
:1046E00010300020FEE74FF0B04382B0DA6C42F0A9
:1046F0000102DA64DB6C03F001030193019B02B059
:104700007047000030B587B0FFF7EDFF4FF48051E0
:1047100001224FF0904003F09DFE01224FF4006112
:104720004FF0904003F096FE4FF4C0551123CDE9B1
:10473000015301A901234FF09040039303F064FD5E
:1047400008240A2500224FF480514FF0904003F0D6
:1047500081FE0120FEF742FC01224FF480514FF010
:10476000904003F077FE0120FEF738FC013DE9D1CF
:104770004FF400614FF0904003F066FE08B9013C31
:10478000DFD14FF400614FF0904003F05DFE68BB55
:10479000FFF7A9FF04240123039001A92A48CDE9CA
:1047A000014303F031FD284C01220421204603F08F
:1047B00051FE2120FEF712FC00220421204603F0C6
:1047C00049FE2120FEF70AFC01220421204603F0C5
:1047D00041FE2120FEF702FC20460022042103F0C6
:1047E00039FE4FF42570FEF7F9FBDDE7FFF77BFF9D
:1047F0004FF0B04300249A6D42F480029A659B6D9D
:1048000003F4800300934FF4C052009B1223CDE9C0
:1048100001230323CDE9034304230DEB03014FF0F0
:104820009040059303F0F0FC08480949094B846067
:10483000C0E900130123C0E90334C0E9074444611F
:1048400003F07CFF07B030BD00040048D40F002007
:10485000005800401A091020FFF754BF40B94B1E02
:104860005A425A414FF400714FF0904003F0F2BDAC
:10487000704708B50120FEF736FF6420FEF7AEFB57
:1048800000F024F9BDE808400120FEF731BF000028
:10489000054B1A6802805A689B684381034B02816A
:1048A00001221A70704700BF54100020AD0F002085
:1048B00010B5044600F008F810F0FF001FBFEE230B
:1048C0002370AA23637010BD2DE9F3470024304EF6
:1048D000304D346021462046FFF7C0FF21460120BD
:1048E000FFF7BCFF21460220FFF7B8FF2A4F4FF029
:1048F0005208A146012195F8640185F86081C5F848
:104900006891FFF7ABFF0320FEF768FB00228821C8
:10491000284602F0E5FB0DF10602C021284602F010
:104920002DFC80BBBDF806204EF6AA639A422AD120
:104930004FEA440A0AF1540A5FFA8AFA51462846B5
:1049400000F034F9F8B90DF10602C021284685F8C7
:1049500060A102F013FCB0B9284600F0EBFA90B960
:10496000326801231A4432603A68C5F86831A340BE
:1049700013433B600134032C05F5C875BAD1306888
:1049800002B0BDE8F0870021E0B2FFF767FFF1E772
:104990004C100020BC000020481000202DE9F74FEB
:1049A000354C834604F5966A4FF00A094FF00E081D
:1049B00048F2E8074FF490164FF48045D4F8682188
:1049C000002A51D0204600F0A9FD0DF102020DF1A0
:1049D0000101204600F05CFB0DF1030201A9204615
:1049E00000F0A1FE0021204600F0E4F801220021A1
:1049F000204600F0A3F901221146204600F09EF95E
:104A0000BBF1020F0ED81D4B1D4A33F81B501D4B36
:104A100012F80B8053F82B601B4A1C4B12F80B90BA
:104A200053F82B702A460121204600F0D2F9324675
:104A30000021204600F0CDF93946204600F0D4F898
:104A400042460021204600F0D1F84A460121204686
:104A500000F0CCF80DF102020DF10101204600F04A
:104A600017FB0122C4F87C2104F5C8745445A5D174
:104A700003B0BDE8F08F00BFBC0000200870010843
:104A800028700108107001082B7001081C700108C3
:104A900010B50B7E9BB9D0F87C21098912B1C0E911
:104AA0005E1310BD084BD0F878411A68C2F58073C8
:104AB0004B4304FB02331B12C0F87831F1E70123AA
:104AC000C0F87C31EDE700BFB80000202DE9F84FB9
:104AD000DFF8C0A0304DFFF7BFFEDAF800300BB1B1
:104AE0002B6813B9FFF7F0FE28602B682B4E0024CB
:104AF000A34234607460B46049DDDFF8A480294DBE
:104B0000DFF8A4B02046FFF749FF88F80040D5F849
:104B10006831012B31D103FA04F90A2722492846CA
:104B200000F05CFCB0B959462846FFF7B1FF9BF88E
:104B300018307BB9D5F8783146F82430DAF80030EF
:104B400043EA0903CAF8003098F8003043F0010343
:104B500088F800300120FEF741FA9BF818301BB1AD
:104B6000013F17F0FF07D9D1D5F8783140F6C412CC
:104B7000002B08BF134646F8243005200134FEF709
:104B80002DFA032C05F5C875C1D198F80030BDE8A1
:104B9000F88F00BF48100020501000205410002053
:104BA000AD0F0020BC0000202C1000204A088A21F4
:104BB00002F096BA152906D8044BCB40DB0702D584
:104BC0000174002070476FF0070070470B00300041
:104BD00010B50A460C46092102F0A4FA18B9237848
:104BE00003F00103237010BD01F06BBE01F053BD53
:104BF00001F04DBEF7B500230C46174601210DF11B
:104C0000070206468DF8073002F08CFA0546D8B93F
:104C1000012F9DF8073026D1042C3AD8DFE804F0A4
:104C200003171A1D200043F01004A3420CD02246A3
:104C30000121304602F054FA054628B9716986F818
:104C400030413046FFF7D0FF284603B0F0BD43F0B7
:104C50002804EAE743F00404E7E743F04004E4E70C
:104C600043F08004E1E7042C13D8DFE804F00306E6
:104C7000090C0F0003F0EF04D7E703F0D704D4E7E3
:104C800003F0FB04D1E703F0BF04CEE703F07F0499
:104C9000CBE76FF00305D7E713B500230C460DF102
:104CA000070201218DF8073002F03CFA78B99DF82F
:104CB0000730C3F300122270C3F3C002A270C3F323
:104CC00080026270C3F38012DB09E270237102B0CC
:104CD00010BD37B50D460DF10202F821044602F071
:104CE0004DFA70B901AA0421204602F067FA40B9D2
:104CF000BDF802201AB1019BB3FBF2F32B602B68C5
:104D0000A36103B030BD037F0B700020704737B53F
:104D10000D460DF106022021044602F02FFA28B9B3
:104D2000BDF8063023B9236A2B60207703B030BD6D
:104D3000DB002B60236201232377F7E70529F8B511
:104D400004460E46154635D862B100EB81030121B9
:104D50005A6B0023701E042807D8DFE800F00E17F6
:104D60001A1D240011460123F4E784F82810344466
:104D7000E5B984F82850002007E0C2F34F2244210F
:104D8000204602F0BDF90028F1D0F8BD84F82A10C1
:104D9000EDE784F82B10EAE75B00FE226021204655
:104DA00002F0D5F9EFE71B01EF22F7E7012384F8C2
:104DB0002830E0E76FF00300E7E7052996BF4018C9
:104DC000002390F82830137094BF00206FF0030088
:104DD000704770B54318044693F828000E461546F0
:104DE00018B904EB8106726370BD05291BD8DFE892
:104DF00001F0030912141616626304EB8604002006
:104E00006563F1E7C2F34F224421204602F078F9AE
:104E10000028E9D1F1E7E263EFE72264EDE7C2F3AE
:104E20004F226421F1E76FF00300DDE737B5044658
:104E3000154605292CD8DFE801F0030717191B1BBD
:104E4000436B2B60002021E00DF10602442102F0AB
:104E500095F9D8B9BDF8062053029AB12B60A36327
:104E6000012384F8293011E0C36BEAE7036CE8E71B
:104E70000DF10602642102F081F938B9BDF806305F
:104E80005B02DEE7A36B2B6084F8290003B030BD22
:104E90006FF00300FAE737B50D460DF10702012167
:104EA000044602F03FF938B99DF8073084F83031F4
:104EB000DB092B7084F84C3003B030BD2DE9F8438A
:104EC000037C0C4601F8083B0546FFF702FF40BB98
:104ED000207304F110012846FFF719FF08BB04F105
:104EE0001401284600F021FCD8B904F1240705F18B
:104EF000270904F1170806463A46B1B22846FFF7DB
:104F000095FF70B9013619F8013F08F8013F062EE8
:104F100007F10407F0D104F13C012846FFF7BBFF7D
:104F200008B1BDE8F883211D2846BDE8F84301F02B
:104F300030BD0000F0B50022054693B0882102F094
:104F4000CFF84FF47A72A5F852214FF4C872A5F841
:104F500054214C4AC5F8582100234B4A85F8F030BB
:104F6000C5F8D4202B6202A92846FFF7A7FF044604
:104F700070B9ADF8080002AE0FCE05F110070FC7EB
:104F80000FCE0FC70FCE0FC796E80F0087E80F00B0
:104F90003E4BC5F834314FF4FA730126A5F8383189
:104FA0004FF42063A5F83C313246802185F85061EA
:104FB000284602F095F832460746FF21284602F0BF
:104FC0008FF8002211460743284602F089F83C4337
:104FD00064B204430DF107029121284602F0A2F8C1
:104FE00064B29DF8073085F83A3104433246002117
:104FF000284602F075F864B204430022FF212846D7
:1050000002F06EF864B2044300228021284602F0C8
:1050100067F864B2204340B2002488BBA1B20122E9
:1050200028460134FFF78AFE062CF6D140BB044621
:105030006885024604212846FFF780FE00BB024631
:1050400005212846FFF77AFED0B94FF490136B6321
:105050004FF4804201212846FFF7BBFE80B94FF490
:105060000C13FF22C5E90F3085F8302101212846B5
:1050700002F036F8012385F8323108B985F8154178
:1050800013B0F0BD856B0100A470090064008403B7
:10509000012300F079BD2DE9F0428EB00C460C23BF
:1050A00004AA1421054602F005F8844600286CD1B4
:1050B0009DF81A309DF81B609DF817209DF8181078
:1050C000A07506EB03269DF81630206002EB032244
:1050D0009DF81930606003EB01239BB25B029DF8E1
:1050E000121023619DF81330B5F8520103EB012330
:1050F00092B252029BB2E260A382B0F57A7F9DF831
:10510000101095F83171B6B20AD0704300F5FA70FC
:105110004FF47A76B0FBF6F02E7F002E39D186B2AE
:10512000002F40D0B001C0B2B608E0750DF10F00FD
:105130002681CDE90040284601F086FE844620BB4A
:105140009DF80FE084F818E005F150060FCE07AF88
:105150000FC796E80700E37D87E80700D4E903015D
:10516000A28AADF83020D4E90149CDE90A01CDE9A0
:10517000084907AC8DF833308DF834E00FCC50354A
:105180000FC597E8070086E8070060460EB0BDE847
:10519000F0822E8C5E43B2EB262F4FEA262C04D1F0
:1051A00057B948F6E0260020BFE780B25043A2EB93
:1051B0000C06B0FBF6F0B2E742F2B826B2E7000008
:1051C000F7B517460E210DF106021D460B4C06469B
:1051D00001F0D4FFBDF8063004EA43433B6050B908
:1051E0000DF106020C21304601F0C8FFBDF8063073
:1051F00004EA43442C6003B0F0BD00BF0000FE1F72
:1052000073B590F8DA30013B022B06460C4634D8D1
:1052100001AB6A460121FFF7D3FF009BB3F57F0F77
:10522000054603D8019BB3F57F0F23D915BB34B1D5
:105230001349304602B0BDE8704001F00FBC0422B3
:10524000FF21304601F04CFF2A46044670213046CB
:1052500001F046FF2A460443FF21304601F040FF9B
:1052600064B204432A468021304601F039FF64B21B
:10527000044365B2284602B070BD0025FAE700BFBE
:105280005F06002037B5044601228021057C01F02D
:1052900027FF0122FF21204601F022FF00221146B4
:1052A000204601F01DFF94F83A219121204601F09B
:1052B00017FF01220021204601F012FF0022FF21EA
:1052C000204601F00DFF00228021204601F008FF5A
:1052D000012D29D0032D37D0002D3CD101222946A4
:1052E000204601F0FDFE01238DF80730A0B103B088
:1052F00030BD01460DF10702204601F013FF9DF875
:105300000730DB0705F1010508D538B9B5F5FA6FA7
:10531000EFD16FF00600EAE70546F0E7B5F5FA6F62
:1053200008BF6FF00600E2E718B929462046FFF7EC
:1053300067FF02220021204601F0D2FE0028D6D1CC
:10534000042384F83231D2E718B901212046FFF74F
:1053500057FF0422EEE76FF00700C8E738B5057C79
:10536000044625B1204600F054FD28B138BDFFF7B2
:1053700089FF0028F6D0F9E7002DF7D1032384F840
:105380003231F3E773B50646002501220B21304682
:1053900001F0A6FE002204460B21304601F0A0FEDB
:1053A0000DF1070204431321304601F0BBFE9DF8C6
:1053B000073064B2044301355B0760B2EDB205D03B
:1053C000032D08D00028E0D002B070BD032D08BF27
:1053D0006FF00B00F8E76FF00B00F5E738B500232E
:1053E000037404460D46FFF7B9FF50B9294620461D
:1053F000FFF751FE28B901462046BDE83840FFF7C7
:10540000C1BF38BD152970B5054616461C4667D183
:105410000122FF2101F064FE0022114604462846C5
:1054200001F05EFE00220443FF21284601F058FEF1
:1054300064B2044301228021284601F051FE64B287
:10544000044302228521284601F04AFE64B2044347
:105450000422FF21284601F043FE64B204430022E7
:10546000CD21284601F03CFE64B204431122CC2138
:10547000284601F035FE64B204430722FF21284686
:1054800001F02EFE64B204430022BE21284601F042
:1054900027FE64B204430622FF21284601F020FEC5
:1054A00064B204430922CC21284601F019FE64B2FB
:1054B00004430022FF21284601F012FE64B2044397
:1054C0000122FF21284601F00BFE64B200220443B2
:1054D0001146284601F004FE64B2204340B270BD7C
:1054E000042A17D80A2101F0FBFD0028F7D1231E5A
:1054F00018BF01231B01EF228421284601F027FE5B
:105500000028ECD185F8DA6001462846BDE87040F5
:10551000FFF738BF6FF00A00E1E7000070B594B004
:1055200005464022002104A80FF007FD00230121B9
:105530002846ADF806308DF803308DF8043002931C
:1055400000F0B8FC95F8142195F81311012A04D83D
:1055500040F0AD80202940F2AC8001AA02A9284683
:1055600000F02DFB0446002840F09E8095F8503155
:10557000002B40F0A280D5F84C11284601F06EFABD
:105580000446002840F09080234621460422284605
:10559000FFF738FF0446002840F086800122FF21F3
:1055A000284601F09DFD0DF106020646842128469D
:1055B00001F0E4FD22460643FF21284601F090FD5C
:1055C00076B2064374B2002C6ED1BDF806301B01D2
:1055D000C5F8D43004A92846FFF770FC044600281B
:1055E00062D10DF103012846FFF7F2FA04460028C4
:1055F0005AD19DF8033085F8313104AE0FCE05F154
:1056000010040FC40FCE0FC40FCE0FC496E80F00C6
:1056100084E80F000DF103020121284601F082FD0C
:105620000446002840D19DF8033085F83031024609
:1056300001462846FFF7DEFA0446A8BB02460221CF
:105640002846FFF7D7FA044670BB0323014685F8C6
:1056500032310DF10502284601F019F9044618BB54
:105660009DF8053085F8E8300DF105020121284646
:1056700001F00DF90446B8B99DF8053085F8E03021
:1056800003AA0321284600F001FF044660B9039BEA
:10569000C5F8E43003AA0421284600F0F7FE0446CA
:1056A00010B9039BC5F8DC30204614B070BD0C293E
:1056B00051E7284600F010F954E701495DE700BFC3
:1056C0006C05002013B50C460DF10702132101F003
:1056D00029FD9DF8073013F0180F03F0070218BFDB
:1056E0006FF00500226002B010BD13B590F8DA30FB
:1056F000042B0C460BD101A9FFF7E4FF019B042BFF
:1057000001D1012300E00023237002B010BD01AAE3
:10571000142101F007FD0028F7D19DF80430DB07C4
:10572000EFD42070F1E700F04ABA13B50C460DF142
:105730000602282101F022FD78B9BDF80620C2F347
:105740000B0312F4006F18BFA3F580534FF0FA0259
:1057500014BF13FB02F35343236002B010BDF0B536
:105760004FEAD20C4FF0FF341C6002F0070266468D
:1057700000278E4200D207B1F0BD845D664503BFAD
:105780001441E4B215463D4614F0010704D005EB80
:10579000C6051D600136ECE70135082D4FEA5404BB
:1057A000F2D1F7E7034B800953F82000003818BF07
:1057B000012070471808002010B5B1EBD20F4FEA56
:1057C000D20402F0070381BF01229A40035D134314
:1057D0008ABF03556FF03100002010BD0A46062332
:1057E000B02101F049BC0A460623B02101F062BC99
:1057F0002DE9F04F85B08046109E0E9D01968A4699
:1058000093461C464FF00009119B994508D100238F
:10581000129A1660F3B16FF0310005B0BDE8F08F59
:1058200001AB324629465846FFF799FF019F7B1C82
:105830000DD00F9BF818FFF7B5FF504507D13A463A
:105840002046FFF7B9FF7E1C09F10109DCE76FF084
:105850003103DDE721464046FFF7C0FF0028DCD1D9
:1058600002A94046FFF7BFFF2544234602AAAB42E8
:10587000D3D013F8014B12F8011B8C42F7D0CAE7C2
:1058800070B5C02288B00E46012190F8304105461F
:1058900001F026FCF0B901A92846FFF79FFDC8B921
:1058A0000122FF21284601F01BFC98B93246B6219F
:1058B000284601F063FC68B90246FF21284601F042
:1058C0000FFC38B922460121284601F009FC08B92D
:1058D00085F8304108B070BDF0B50F4689B0164666
:1058E000FF210122044601F0FBFB0246A8B94F212B
:1058F000204601F0F5FB80B92C224E21204601F014
:10590000EFFB024648B9FF21204601F0E9FB20B930
:10591000B422B621204601F0E3FB0025C4F824514F
:10592000A4F82851DEB9354607ABB422CDE903739C
:105930000623CDE90032029504F5927304F59572C1
:1059400031462046FFF754FF30B9012384F8153162
:1059500084F8137184F8146109B0F0BD013505F1C4
:10596000B400FFF71FFF0028DED12C2DF6D1DBE7B6
:1059700010B541F001020021044601F0B1FB78B9F5
:10598000204600F046FA58B901462046FFF7FAFCD7
:1059900030B9024601462046BDE8104001F0A0BBE8
:1059A00010BD2DE9F74F4FF0000B88461746FF2139
:1059B000012205461E469DF838A09DF83C908DF8C2
:1059C00007B001F08DFB5A4604465946284601F0BF
:1059D00087FB5A460443FF21284601F081FB64B24D
:1059E000044364B2B8F1000F32D0BAF1000F06D010
:1059F0000C9ACB21284601F095FB204344B2B9F123
:105A0000000F07D00DF10702EE21284601F08AFBB6
:105A1000204344B20122FF21284601F061FB01220C
:105A200004430021284601F05BFB64B204430022DA
:105A3000FF21284601F054FB64B29DF807300D9A0F
:105A4000204323F0100340B2137003B0BDE8F08F81
:105A5000BAF1000F06D03A46CB21284601F040FBB0
:105A6000204344B2B9F1000FD4D033468022EE2156
:105A7000284601F06CFBCBE72DE9F04387B0914657
:105A80000022054688468DF817201E461BB390F865
:105A9000307101221146284601F022FB044658BB12
:105AA00040212846FFF764FF044628BBB9F1010FE7
:105AB00013D10DF11703CDE90290CDE90083024621
:105AC000034649462846FFF76CFF40B1044620468E
:105AD00007B0BDE8F0831F46DBE788F80000002E22
:105AE000F5D03A460121284601F0FAFA044600288A
:105AF000EDD185F83071EAE7002388F800302046C0
:105B0000E4E72DE9F043054687B0884691461E46F6
:105B100023B390F8307102220121284601F0E0FA07
:105B2000044660BB01462846FFF722FF044630BB0F
:105B3000B9F1010F14D10DF11703CDE9020900935A
:105B400002460346CDF8048049462846FFF729FF60
:105B500040B10446204607B0BDE8F0831F46DAE7AF
:105B600088F80000002EF5D03A460121284601F0C1
:105B7000B7FA04460028EDD185F83071EAE7002332
:105B800088F800302046E4E7F8B51D4616460023A5
:105B90002A4690F830710446FFF76EFF70B903464D
:105BA0002A4631462046FFF7ACFF38B93A46012174
:105BB000204601F095FA08B984F83071F8BD2DE956
:105BC000F04F002393B0CDE90A12C0F82431A0F8B9
:105BD00028310122FF21CDE90E33B0F83C818DF848
:105BE000343005468DF8353001F07AFA0446002845
:105BF00040F0E38002464F21284601F071FA044646
:105C0000002840F0DA802C224E21284601F068FA64
:105C10000446002840F0D1800246FF21284601F0CA
:105C20005FFA0446002840F0C880B422B621284616
:105C300001F056FA0446002840F0BF800246802159
:105C4000284601F04DFA0446002840F0B68003468D
:105C50000DF135020DA92846FFF796FF04460028EE
:105C600040F0AB800323CDE90203B421062305F500
:105C7000957A05F592790EAECDE90031049601468C
:105C80004B4652462846FFF7B3FD0446002840F035
:105C900094800DF1360128460E9FFFF7F1FD044672
:105CA000002840F08A80BDF83630434540F2AA8093
:105CB000C5F82401A5F8280107F1B400FFF772FD2B
:105CC00008B92B2F7DD90623B4224FF0030BCDE961
:105CD0000032CDE9027B04964B465246012128460C
:105CE000FFF786FD002840F08B800DF13601284635
:105CF0000E9FFFF7C5FD064600287CD1BDF8363063
:105D0000434540F2828001260696BDF83630434571
:105D100060D2A3EB080383EAE372A2EBE3729DF87F
:105D20001860099205F592734FF0030B0793079BD8
:105D300018689B881090ADF844303A460FAB0621A6
:105D40005046FFF70CFD0F9F7B1C56D007F1B400A7
:105D5000FFF728FD069B98423CD10BF101033A4620
:105D600048460893FFF728FD002849D149462846B0
:105D7000FFF734FD002843D10DF136012846FFF727
:105D80007FFD00283CD1BDF83620A2EB0803002B94
:105D9000B8BF5B42424516D9099A934218D910A957
:105DA0002846FFF71BFD079A0799034610981060D5
:105DB000BDF844208A806BB11C46204613B0BDE874
:105DC000F08F013778E7DDF820B009930137AEE7AF
:105DD000DDF820B00A9BC3F800B00B9B1E700123B6
:105DE00085F815310A9B1B6885F813310B9B1B78CE
:105DF00085F81431E1E70446DFE76FF03104DCE7B2
:105E00000446DAE70026B3467EE70123834606937D
:105E10007BE737B5002304468DF807304FF4FA6569
:105E20000DF107012046FFF760FC58B99DF80730D7
:105E3000012B07D0013D03D0204601F0E5F9EFE743
:105E40006FF0060003B030BD02464FF0804393422E
:105E500002D8002013B970479B08F8E7C118914297
:105E60004FEA50009CBFC018521A9B08F2E773B566
:105E700000228321054601F033F9044688B94FF426
:105E8000FA660DF107028321284601F04BF99DF8CF
:105E900007300343DBB204461BB9013EF1D16FF07A
:105EA000060401228321284601F01AF9204340B25A
:105EB00002B070BD2DE9F04F90F8F06091B04FF056
:105EC0000009072ECDE9079904460F4600F0A2828B
:105ED0000122802101F004F901228046FF212046A1
:105EE00001F0FEF84A4648EA00084946204601F01B
:105EF000F7F84FFA88F848EA00080622FF21204602
:105F000001F0EEF84FFA88F848EA00080DF11502A2
:105F10008321204601F006F99DF815204FFA88F8F4
:105F200048EA000842F004028321204601F0D8F834
:105F30004FFA88F848EA00080722FF21204601F0BE
:105F4000CFF84FFA88F80122812148EA000820465C
:105F500001F0C6F84FFA88F848EA0008204601F038
:105F600053F94FFA88F848EA0008012280212046B8
:105F700001F0B6F84FFA88F848EA000517F0010B6F
:105F80006DB200F01E82F20700F11E826B22942196
:105F9000204601F0A5F880462046FFF768FF06AAD4
:105FA00048EA00089021204601F008F945EA080572
:105FB000069B6DB22422942105432046C3F3062A92
:105FC000C3F3C03901F08CF86DB205432046FFF7EA
:105FD0004EFF6DB2054306AA9021204601F0EEF86F
:105FE000069B6DB21BBA25229421054320460993D6
:105FF00001F076F86DB205432046FFF738FF6DB229
:10600000054306AA9021204601F0D8F8069B6DB200
:106010001A0E05431B0C6DB28DF828208DF829301F
:1060200017F00203029300F0DB8016F0020840F044
:10603000D78002229421204601F052F80190204698
:10604000FFF715FF019B0DF1160203439021204637
:106050001D4301F067F86DB27B2294210543204671
:1060600001F03EF86DB205432046FFF700FF6DB228
:1060700005430DF117029021204601F053F86DB24F
:10608000772294210543204601F02AF86DB205439A
:106090002046FFF7ECFE6DB2054306AA902120468C
:1060A00001F08CF8069B5A0E8DF82C20C3F3864223
:1060B0008DF82D20C3F3C6228DF82E206DB2C3F3C8
:1060C0000612DB0003F07803942105438DF82F209E
:1060D000204678228DF8153001F002F86DB20543A4
:1060E0002046FFF7C4FE6DB2054306AA9021204664
:1060F00001F064F8069B9DF8152002EB53728DF8B1
:106100003020C3F386528DF83120C3F3C6328DF8A8
:106110003220C3F306228DF833206DB2C3F346025A
:106120009B0103F04003942105438DF83420204661
:1061300079228DF8153000F0D3FF6DB2054320466B
:10614000FFF795FE6DB2054306AA9021204601F0A7
:1061500035F8069B9DF8152002EB93628DF83520EB
:10616000C3F3C6428DF83620C3F306328DF83720CC
:106170006DB2C3F346129B0003F07C0394210543E8
:106180008DF8382020467A228DF8153000F0A8FFCF
:106190006DB205432046FFF76AFE6DB2054306AABD
:1061A0009021204601F00AF8069B9DF815208DF8F5
:1061B0003E8002EB93728DF83920C3F3C6526DB264
:1061C0008DF83A20C3F3064205438DF83B20C3F314
:1061D0004622C3F386036DB28DF83C208DF83D3026
:1061E00017F00403019300F0F180730700F1EE80D3
:1061F0007B229421204600F073FF80462046FFF763
:1062000036FE07AA48EA00089021204600F0D6FF93
:1062100045EA08084FFA88F848EA00057C229421EC
:10622000204600F05DFF6DB205432046FFF71FFEDC
:106230006DB2054308AA9021204600F0BFFF6DB261
:10624000732294210543204600F04AFF6DB20543B6
:106250002046FFF70CFE6DB2054306AA90212046AA
:1062600000F0ACFF069B6DB21B0274229421054323
:1062700020461FFA83F800F033FF6DB20543204635
:10628000FFF7F5FD6DB2054306AA9021204600F008
:1062900095FF6DB29DF81B30752294210543204671
:1062A00043EA080800F01CFF6DB205432046FFF7E3
:1062B000DEFD6DB2054306AA9021204600F07EFF68
:1062C000069B6DB21B029BB27622942105432046A9
:1062D000039300F005FF6DB205432046FFF7C7FDAD
:1062E0006DB2054306AA9021204600F067FF6DB20B
:1062F0009DF81B20039B05436DB2134300228121AF
:106300002046039300F0ECFE06220543FF212046C1
:1063100000F0E6FE6DB205430DF115028321204623
:1063200000F000FF9DF815206DB2054302F0FB025E
:106330008321204600F0D4FE6DB205430122FF21E7
:10634000204600F0CDFE6DB205430122002120461B
:1063500000F0C6FE6DB205430022FF21204600F08A
:10636000BFFE6DB2054300228021204600F0B8FE3A
:106370006DB205436DB2039BFDB9BBF1000F29D18E
:10638000029AAABB019AAAB1720713D4079AC4F859
:106390001821089AC4F81C214FEA4822C4F8202189
:1063A0003BB1A3F5C8534FF47A7253431B095B42C8
:1063B0001BB2E3603E4384F8F060284611B0BDE8AC
:1063C000F08FD946DA462BE6CA4629E64FF0000898
:1063D000434693E7F007D3D40998BDF8282084F802
:1063E00013A184F81491C4F82A01A4F82E21C7E758
:1063F000B107C7D49DF8162084F8F1209DF8172026
:1064000084F8F2200BA904F1F30002930EF015FEBC
:10641000029BB7E74D46D0E750B10138002330F07A
:10642000FF019AB203F1010303D100EB022080B215
:1064300070474008F3E7C3B2000A03FA00F00130E6
:1064400070470000084B5A434FF47A7302F5FA7212
:106450004FF4FA60B2FBF0F0B2FBF3F203FB010081
:10646000B0FBF2F0704700BF002F3A00064B5A43D2
:106470004FF47A7002F5FA72B2FBF0F24A4302F579
:10648000FA72B2FBF0F07047002F3A002DE9FF419D
:1064900002294FF00005074616468DF80350ADF867
:1064A00004501CD80DF102022946FEF7A1FB044658
:1064B00030B90DF103024621384600F033FE0446A0
:1064C0009DF80300FFF7B7FF81B29DF80220384620
:1064D000FFF7CCFF3060204604B0BDE8F08103290F
:1064E00018D10DF102022946FEF782FB044600286E
:1064F00046D101460DF102023846FEF779FB04460B
:1065000028B901AA5121384600F038FE0446BDF8EA
:106510000400D7E7042935D102A9FEF7BDFB9DF899
:106520000B30ABB10DF1020229463846FEF760FB95
:10653000044658B901AA5121384600F01FFE04460E
:10654000BDF80400FFF777FF85B214B1002015E015
:106550001D460DF1020201213846FEF749FB0446B3
:106560000028F3D10DF106027121384600F006FE35
:106570000446BDF80600FFF75EFF80B2401BA3E7AC
:106580002846A7E728462C46A4E7F0B5022985B09F
:10659000054616461ED80DF105020021FEF728FB20
:1065A0000446A0B99DF8052031462846FFF74AFF6A
:1065B00083B2B3F5807F9ABF00F1FF32D2B2FF22DF
:1065C000A5F8D8204621284600F08AFD044620463A
:1065D00005B0F0BD03291FD10DF105020021FEF722
:1065E00007FB9DF80520314604462846FFF72AFFA1
:1065F00080B2FFF711FF0246ADF80600A5F8D800FB
:10660000002CE4D15121284600F07AFD04460028F0
:10661000DDD1C5F8E460DAE7042939D102A9FEF733
:106620003BFB9DF80B70B7B10DF105020021284628
:10663000FEF7DEFA04460028C9D10DF10602512109
:10664000284600F09BFD0446BDF80600FFF7F3FE68
:1066500087B2002CBBD10DF1050201212846FEF7BF
:10666000C7FA04460028B2D19DF8052031462846D5
:10667000FFF7E8FE3844FFF7CFFE712102462846B7
:1066800000F03EFD04460028A1D1C5F8DC609EE77D
:106690006FF003049BE7F0B585B000238DF803305D
:1066A000D30705460F46164605D439B9A2F10C03A7
:1066B000DAB2062A11D96FF00300E6E0012921D1F0
:1066C000A2F10803DAB2062AF5D8062B1AD8DFE8B9
:1066D00003F03B1969198A199D00062B12D8DFE8CF
:1066E00003F004112D112F113100182257212846D3
:1066F00000F0F6FC08225621284600F0F1FC0028A4
:1067000040F0C3807408013CE4B2002F00F0918097
:10671000012FD0D101AA04212846FFF7B7FE50B9B6
:1067200022467021284600F0DBFC20B9019A0421A2
:106730002846FFF72AFF85F8E06099E03022D5E788
:106740004022D3E75022D1E71022482100F0C8FCB4
:1067500008224721284600F0C3FC022204463221C9
:10676000284600F0BDFC0C2204433021284600F0EE
:10677000B7FC64B204430122FF21284600F0B0FCBC
:1067800064B2044364B230223021284600F0A8FCF1
:1067900000220443FF21284600F0A2FC64B22043FB
:1067A00040B2ACE72822482100F09AFC0822472199
:1067B000284600F095FC032204463221284600F0CA
:1067C0008FFC044364B209223021284600F088FC83
:1067D00001220443FF21284600F082FC64B20443F6
:1067E00064B22022D0E73822482100F079FC082248
:1067F0004721284600F074FC032204463221284633
:1068000000F06EFC044364B20822DDE74822114622
:1068100000F066FC08224721284600F061FC0322B4
:1068200004463221284600F05BFC044364B2072290
:10683000CAE702AA03212846FFF728FEB0B903AA37
:1068400002212846FFF722FE80B922465021284621
:1068500000F046FC50B9029A03212846FFF795FE46
:1068600020B9039A02212846FFF78FFE85F8E860D9
:1068700058B969692846FEF7B7F930B902460123CD
:106880000DF103012846FFF73CF905B0F0BD13B543
:10689000144629B1012910D06FF0030002B010BDD9
:1068A0000DF10702502100F03DFC0028F6D19DF8C3
:1068B000073001335B002370F0E70DF10702702110
:1068C000F1E7F0B5002385B04FF4FA62CDE900237B
:1068D00044F61F63994206460F4604D86FF003053D
:1068E000284605B0F0BD02A9FEF7D6F905460028F6
:1068F000F6D19DF809209DF8083013439DF80A2031
:106900001343A7F636341BD06A4602213046FFF700
:10691000BDFD00283BD19DF808302BB1009B03F250
:106920004E239C42DAD9E41A9DF80A3023B3009B27
:1069300003F2B223B4EB430F4FEA4302CED9A41AB9
:106940009DF80B305BB101AA03213046FFF79EFD95
:10695000019B03F52573A342C0D2C0B9E41A9DF888
:106960000C30002BBCD0A4F2262204213046FFF7C5
:106970000CFE77610546B3E79DF80930002BDFD0A8
:10698000009B03F525739C42A8D9E41AD8E7054675
:10699000A6E770B54FF4FA6286B00023CDE9022372
:1069A00040F636330B600C4604A90646FEF774F930
:1069B0000546002836D19DF811209DF8103013436C
:1069C0009DF81220134319D002AA02213046FFF786
:1069D0005DFD002840D19DF810302BB1029B03F2E1
:1069E0004E222368134423609DF81230EBB1029BC2
:1069F00003F2B222236803EB420323609DF81330B5
:106A0000EBB99DF814305BB101AA04213046FFF7C1
:106A10003DFD019B03F22622236813442360D8B96D
:106A200023687361284606B070BD9DF81130002BB5
:106A3000E4D0029B03F5257223681344DDE703AA23
:106A400003213046FFF722FD039B03F525722368DF
:106A5000134423600028D4D00546E3E72DE9F7432B
:106A6000002406460D46204615F80480B8F1000FB4
:106A700000D010B103B0BDE8F083671CB8F1FF0F80
:106A800015F8079029D1A71CEB5DB9F1030F36D893
:106A9000DFE809F0020B131B271D2C44E27802EB00
:106AA0000323A6F834313C46DEE7271D2C44E27868
:106AB00002EB0323A6F83631F5E7271D2C44E278D4
:106AC00002EB0323A6F83831EDE7271D2C44E278CA
:106AD00002EB0323A6F83C31E5E7B8F1040F0ED82A
:106AE00002344246291901A80EF0B4FA434601AA1D
:106AF0004946304604EB080700F0BEFAD3E76FF0D2
:106B00000300D0E773B500230E4613600DF10701B3
:106B100005461446FEF7F7F840B99DF807302BB14B
:106B2000B38A2A6A534380331B0A236002B070BDC4
:106B300013B5CB681360144601AAFFF7E3FF18B939
:106B40002368019A1344236002B010BDF8B5B0F871
:106B50005451D0F8580168438030000A0E4645432E
:106B6000DDE90717144652B1B60206EB5202B2FB3A
:106B7000F4F202EB4202524302F50042140C069A70
:106B8000534301F50042120C06200332B2FBF0F22F
:106B9000C2EBC202B2F5803F38BF033103F50043B8
:106BA0003EBFB1FBF0F1C1EBC10101F500414FEA7D
:106BB000134334BF090C1B4903FB03F338BF49439C
:106BC00003EB57030B44B3FBF7F39B03FE2205F1E2
:106BD00020007F33B3FBF2F35C434FF47A7704F584
:106BE000FA748009B4FBF7F42401FFF72DF904F5DA
:106BF000FA74BC4228BF4FF4FA63064629BFB4FBBF
:106C0000F3F300205B19B4FBF7F428BFB3FBF4F0F7
:106C1000FFF71AF9099B864294BF1E601860002096
:106C2000F8BD00BF0000F0FF2DE9F04F91B0CDE9B5
:106C30000723036A0E930B6909930546CB680B93F0
:106C40000F460FAAFFF774FF0EAA39462846FFF732
:106C500059FF58BB0F9C95F8E0B0D5F8DC30059390
:106C60004FF47A7606FB04F101F5004104910E9988
:106C70000A910499D5F8E4300693BBF1080F04F1AA
:106C800080040CBF0223032324F0FF0A090C95F8AB
:106C9000E820DFF8A081CDF83CA00C9109D1079B3A
:106CA000C3F80080089BC5F84081186011B0BDE8AA
:106CB000F08F06990D932846FFF7C4FB5A460599B5
:106CC00081462846FFF7BEFB0D9B5B490C9A814429
:106CD00003FB09F94FEAC92940F2776309F5FA790C
:106CE000240AB9FBF6F903FB09F909F5FA79B9FBAE
:106CF000F6F909FB04F404F18003099C74430C4089
:106D0000B4FBF2F44D4A1B0A944228BF1446012BEF
:106D100038BF01230C204FF4167258435443FFF739
:106D200093F83B7E3A894FEA400B002B7FD14249D2
:106D3000049B0B4003F5FA71414B5A4341F25C232B
:106D4000B2FBF3F20A9B7343B3F5481F28BF4FF41D
:106D50004813A1EB4303B1FBF6F1B3FBF6F31B02BF
:106D6000B3FBF1F63602C6F58036564306F500460B
:106D7000360C06F5803676087643B60B4FF448702D
:106D8000704304F5004300F500401B0C5B43000C0E
:106D900000FB0030FFF758F803046422323341F25D
:106DA0008837B3FBF2F340F6B532B3FBFBF302FBDB
:106DB0000377244B9F429CBF42F21073B7FBF3F75B
:106DC000DDE90532134403F5FA734FF47A7B4FF48F
:106DD000FA62B3FBFBF0B3FBF2F202F5C812B2FBAE
:106DE000F0F088BF4FF47047FFF72EF8000200F56F
:106DF000FA70B0FBFBF0404307FB0700FFF724F8F5
:106E00000BFB00F0079B0B9A404528BF40461860DB
:106E1000089BC5F84001CDE902934FF448730093F5
:106E20000194334651462846FFF790FE3EE74FF463
:106E30008036A3E7AE878F020000FFFF666666001C
:106E40009A9906000F279F242DE9F04F8BB0002759
:106E500011F0780FDDE914B80446019299468DF8D7
:106E60000E708DF80F708DF810708DF81170ADF8F0
:106E700012700997C1F3C30A00F0AF80AAF10503AD
:106E8000DBB20A2B01D86B4AD75C0DF10E02002150
:106E90002046FDF792FF9DF80E500646D5B100281A
:106EA00040F09D8009AB05AA59462046FFF7BCFE7D
:106EB000002840F09680099BABF80A30014606AAEC
:106EC0002046FDF7B3FF069D25B1059B9D422CBFD3
:106ED0000025012520B904AA02212046FDF76DFFF7
:106EE0009DF8106026B300287DD107AA0221204614
:106EF000FDF79CFF88B90122FF21204600F0F0F841
:106F000058B90DF11202B621204600F037F920B928
:106F10000246FF21204600F0E3F8BDF81230079E3C
:106F20005B02C4F848311EB19E422CBF00260126E8
:106F300028B90DF1110203212046FDF73EFF9DF80F
:106F4000113093B1002873D1B9F1000F03D0019B28
:106F50001B02B3FBF9F908AA03212046FDF766FFDF
:106F6000089B4B4594BF0023012320B9012F3CD13E
:106F7000FF2288F8002098F800200AB9ABF80A2010
:106F80000DF10F02012120460193FDF716FF08BB0A
:106F90009DF80E20019B002A08BF0125BAF1040FBD
:106FA00018BF9DF80F2084F82E501ABFB2FA82F253
:106FB0005209012284F82F209DF81020002A9DF804
:106FC000112008BF0126002A08BF012384F8306081
:106FD00084F831300BB0BDE8F08F012755E700256C
:106FE0007EE735467CE70026A9E70AF1FF32092A49
:106FF0000AD8DFE802F0050505090907090B070BA8
:107000000522B6E70422B4E7012E01D10322B0E73E
:10701000BAF1040F01D0012B01D10222A9E7012D01
:107020001BBF002388F8003088F800502B46A2E7E9
:107030000023A0E72E70010807B502F10A030093B0
:1070400093B20A4690F86011D0F85C0101F0C8FBD9
:1070500003B05DF804FB13B502F10A0390F8604138
:107060000093D0F85C0193B20A4644F0010101F0AC
:107070004DFC02B010BD00003F2BF8B50E46054692
:1070800011461C4611D80A4F38461A4600F8016BC3
:107090000DF0E0FF621C39462846FFF7CDFF0028BF
:1070A0000CBF00206FF01300F8BD6FF00300FBE78A
:1070B0006010002073B515468DF8071001220DF100
:1070C000070104461E46FFF7B7FF28B93246294696
:1070D0002046FFF7C0FF08B16FF0130002B070BD8B
:1070E00008B5064B19705A7019460222FFF7A4FF23
:1070F000002814BF6FF01300002008BD60100020AE
:1071000008B5074B1970110A59709A701946032275
:10711000FFF792FF002814BF6FF01300002008BD96
:107120006010002037B515468DF8071001220DF1CB
:1071300007010446FFF780FF28B9012229462046AF
:10714000FFF789FF08B16FF0130003B030BDF7B54A
:1071500015460DF1070206460F461C46FFF7E2FFF3
:1071600050B99DF807301D4044EA050239463046C3
:107170008DF80720FFF7B4FF03B0F0BD73B51446D8
:107180008DF8071001220DF107010646FFF754FFA5
:1071900018B16FF0130002B070BD074D02222946EE
:1071A0003046FFF758FF0028F3D12A786B7803EBBD
:1071B00002232380EFE700BF6010002073B5144660
:1071C0008DF8071001220DF107010646FFF734FF85
:1071D00018B16FF0130002B070BD0A4D04222946A9
:1071E0003046FFF738FF0028F3D16B782A781B046C
:1071F00003EB0263EA781344AA7803EB02232360CB
:10720000E9E700BF6010002008B50220FBF7E6FEAA
:10721000002008BD37B5084B0190084C187894251C
:107220004FF47A73012201A905FB004003F0D0FD61
:10723000019803B030BD00BFA0100020A4100020B2
:107240007047000010B5032000F072FC01F0AAFDA9
:10725000064B18600F20FBF7B7FE044618B9FBF782
:107260002AFD204610BD0124FBE700BF28080020AE
:107270004FF0E022136923F00203136170474FF0CF
:10728000E022136943F0020313617047014BD3F806
:10729000900570470070FF1F014BD3F894057047AD
:1072A0000070FF1F014BD3F8980570470070FF1F57
:1072B000024A536823F0010353607047002004E042
:1072C000024A536823F0020353607047002004E031
:1072D000024A536823F0040353607047002004E01F
:1072E0008068C0F380007047F7B50023019304461F
:1072F000002800F0E980856D25B9FBF733F8E565D6
:1073000084F8545023689A68D00040F1A1809A68AC
:10731000D10000F1B480A26D42F01002A265E26DCE
:1073200042F00102E26501251846FFF7D9FFA26D80
:1073300002F01002024340F0C980A26D206922F4DD
:10734000817242F00202A2659A68D2075DD4226B74
:10735000A67E94F82CC0003A18BF01221703D4E986
:1073600002120A43217E42EA8132617E42EAC13240
:1073700042EA4632002842EA4C02B4BF20F0004103
:107380004FF400113A430A4394F82010012903D125
:10739000002E76D142F48032616A21B1A66A01F4EE
:1073A000E07131430A43D968E66C21F4FE3121F4DF
:1073B000FF711143D96094F83C206168012A01F003
:1073C000404C4CEA060609D1D4E910273A4332432F
:1073D000A66C324342EA0C0242F001061F693E4AA3
:1073E0003A4032431A6121F00042B2F1804F0CD092
:1073F000B1F1004F09D0394ED6F8082701F47011C9
:1074000022F470120A43C6F808275A69666BA16B0A
:1074100022F0070232435A615A6922F0700242EAAE
:1074200001125A61002835D19A6A62F00F029A62FD
:107430005B6903F007039E423CD10023E365A36D23
:1074400023F0030343F00103A365284603B0F0BD16
:107450009A68234922F0104222F0170242F080522B
:107460009A60204A1268B2FBF1F201325200019296
:10747000019A002A3FF44BAF019A013AF7E7002541
:1074800052E7A16D41F02001A165E16D41F00101DC
:10749000E16581E7B0F5001FCAD19A6AE269013A55
:1074A00092006FF00F0102F01C0201FA02F2216E4D
:1074B0000A43BCE7A36D23F0120343F01003A36556
:1074C000E36D43F00103E3650125BEE7A36D43F0DF
:1074D0001003A365F8E700BF02FCFF1F0020014076
:1074E000400D030028080020F8B54569082D044622
:1074F0000E460AD00368DB68D80705D5A36D43F0B4
:107500002003A3650120F8BD0425FBF75FFD0746B6
:1075100023681A682A4221D0A26D42F40072A26543
:10752000DA6812F4406F14D1A27E92B91A68120779
:107530000FD51846FFF7D4FE28BB5A6822F00C027C
:107540005A60A26D22F4807222F0010242F0010220
:10755000A265207E00BB0C221A60D4E7711CD8D033
:10756000FBF734FDC01BB04201D8002ED0D12368F8
:107570001B682B40CCD1A26D84F8543042F0040239
:10758000A2650320BFE7A26D42F02002A265E26D72
:1075900042F00102E265DCE70020B4E70368186C02
:1075A00070470000F7B50023019390F85430012B89
:1075B000044600F0C58005680669012380F8543050
:1075C0002846FFF78DFE002840F0B480D1E9002066
:1075D000022826F0040300F08280B3F1004FC2F3CA
:1075E000110E13D1AB6A43EA0E03AB628B68686974
:1075F00003EA022323F07C4323F0FF0320EA022165
:107600000B43002A6B6126DB002055E0236E00F05F
:107610001F074FF00F0C0CFA07FC6FEA0C0623EA69
:107620000C0CBEF1000F11D1C2F38463BB4043EADE
:107630000C0323668008E36901309842D6D8A86A13
:10764000C2F38363BB4006403343CEE792FAA2F312
:10765000B3FA83F3EAE73B493B48D1F80837824263
:1076600003F0E07519D11B02CED4D1F8083723F00E
:10767000E0732B4343F40003C1F80837334B1A6817
:10768000334BB2FBF3F20C2302FB03330193019B58
:10769000002BB9D0019B013BF8E72E48824210D164
:1076A00013F08070B0D1D1F8083723F0E0732B438A
:1076B00043F08073C1F80837002384F8543003B0D6
:1076C000F0BD254882429FD113F480009CD1D1F8AF
:1076D000083723F0E0732B4343F48003EAE7B3F168
:1076E000004F01BFAB6AC2F311018B43AB62002AAA
:1076F0008ADA154813498242D1F8083709D1D1F8FE
:10770000082703F0A07322F0E0721343C1F8083792
:107710007AE71048824204D1D1F8082703F44003E5
:10772000F1E70D4882427FF46FAFD1F8082703F0EC
:10773000C073E8E7A26D42F02002A2651846BBE7DD
:107740000220BCE700200140001000B02808002003
:10775000400D0300004000B8002000B4026838B5B6
:1077600004461046FFF7BCFD08B9002038BD9368F9
:10777000990707D4936823F0004323F0170343F0DD
:1077800010039360FBF722FC054623689B685B07A8
:10779000EBD5FBF71BFC401B0228F6D923689B683E
:1077A0005A07F2D5A36D43F01003A365E36D43F0D0
:1077B0000103E3650120D9E773B500230268019353
:1077C0009368DD07044602D5002002B070BD9168C1
:1077D000214B194209D0A36D43F01003A365E36D5B
:1077E00043F00103E3650120EFE7936823F00043D2
:1077F00023F0170343F001039360184BD3F80837C5
:1078000018021CD4637E012BDED0FBF7DFFB144E85
:10781000054622681368DB07D6D49368D9075FBF93
:107820009368334043F001039360FBF7CFFB401BA9
:107830000228EED923681B68DA07EAD4CBE7094BA4
:10784000094A1B68B3FBF2F301330193019B002B40
:10785000D8D0019B013BF8E71700008000200140D1
:10786000E8FFFF7F28080020400D030038B50446DC
:107870000068FFF735FD054620BB94F85430012B16
:1078800020D0012384F854302046FFF795FFB0B98B
:10789000A36D226823F4706323F0010343F4807323
:1078A000A3651C23E065136084F85400936823F0FB
:1078B000004323F0170343F00403936038BD84F8BA
:1078C0005450FBE70220F9E7026838B593689168E5
:1078D0000446C80701D4002038BD9907FBD493683B
:1078E00003F00503012B19D1936823F0004323F023
:1078F000170343F00203936003231360FBF766FB57
:10790000054623689B68DB07E5D5FBF75FFB401B5B
:107910000228F6D923689B68DA07F2D5A36D43F0F5
:107920001003A365E36D43F00103E3650120D3E792
:1079300070B5044600284BD0836D43F00203836585
:10794000FFF70CFF054668B92046FFF7BDFF054667
:1079500008B90123A3652268936823F0104323F03C
:107960001703936023685A6822F4677222F00302B7
:107970005A6040F29F321A60D968164A0A40DA60AB
:107980001A6922F040421A615A6922F007025A61CC
:107990001A6A02F0F0221A625A6A02F0F0225A625F
:1079A000DA6A02F0F022DA629A6A0B4A00269E62D4
:1079B000D2F8083723F0FE73C2F808372046FAF7EA
:1079C000E5FCE6652666A66584F85460284670BD29
:1079D0000125FBE700023E830020014010B590F82E
:1079E0005430012B044615D0012380F85430FFF7A2
:1079F000B5FE58B92046FFF767FF38B9A36D23F4E9
:107A0000807323F0010343F00103A365002384F88E
:107A1000543010BD0220FCE7F7B50023019390F825
:107A20005430012B04467FD0012380F85430FFF7F7
:107A30004BFF23689A6812F00102054607D0A36D38
:107A400043F01003A365002384F854302DE0A16DAA
:107A5000364F21F4817141F00201A165DE68D968D9
:107A600026F4FF4626F07C0621F40041360421F07E
:107A70000301360CD96008209968394041F0004173
:107A800099609968002913DA0199013101910199EE
:107A9000B1F52E3FF5D3A36D23F0120343F010038D
:107AA000A365002384F854300125284603B0F0BDB7
:107AB000D3F8B410013801F07F010A44DCD1996891
:107AC0001A48014041F001019960D3F8B41021F047
:107AD0007F0141EAD202C3F8B4209A68024042F022
:107AE00002029A60FBF772FA074623689A68D20787
:107AF00008D4DA683243DA60A36D23F0030343F05D
:107B000001039FE7FBF762FAC01B0228EDD9236847
:107B10009B68D907E9D5A36D43F01003A365E36D16
:107B200043F00103E365BFE70225BEE7E8FFFF7FFF
:107B30000749CA6822F4E0620302120403F4E06316
:107B4000120C134343F0BF6343F40033CB60704720
:107B500000ED00E0164B30B5DC68C4F30224C4F13C
:107B60000703251D042B28BF0423062D4FF0FF35E6
:107B70008CBF033C002405FA03F321EA0303A5406C
:107B800022EA0502A340002843EA0203ACBF00F149
:107B90006040084A4FEA0313B8BF00F00F00DBB2A1
:107BA000AABF00F56140135480F8003330BD00BF18
:107BB00000ED00E014ED00E0002807DB044A410975
:107BC000012300F01F00834042F82130704700BFBE
:107BD00000E100E000280CDB4309064900F01F002B
:107BE00020330122824041F82320BFF34F8FBFF39F
:107BF0006F8F704700E100E070B5D0E91345656014
:107C0000446D14B1D0E916456560D0E9105404F014
:107C10001C060124B4406C60046863608368102B08
:107C20000BBFA260A160E160E26070BD0268416CC0
:107C3000D3B210B5083B1424B3FBF4F30B4CA242AF
:107C400088BF0B4A21F0030199BF01F1804202F580
:107C50000232521807338264064AC26403F01F03DB
:107C6000012202FA03F3036510BD00BF07040240BE
:107C70001C0802408008024038B500285ED0026827
:107C80002F4B9A424FF014014CD82E4B1344B3FBA8
:107C9000F1F32D499B00C0E91013022380F8253031
:107CA0001368056923F4FF4323F070031360D0E9E0
:107CB000024323432B43456911682B4385692B43BA
:107CC000C5692B43056A2B430B431360FFF7AEFFD7
:107CD000B4F5804F04BF002343604268816C02F01A
:107CE0007F030B60D0E91314013A032A4C6020D8BB
:107CF000164A174981651A44013B9200012103F09D
:107D0000030301FA03F300214265C3651160114AC0
:107D1000536400230122C36380F8243080F82520B7
:107D2000184638BD0C4B1344B3FBF1F30B499B00D1
:107D3000B1E70023C0E91533C365EAE70120F0E7A6
:107D400007040240F8FFFDBF000002403F82001020
:107D50004009024000090240F8FBFDBF0004024058
:107D600038B5002841D00268136823F0010313607E
:107D70001F4B9A424FF0140130D81E4B1344B3FBF3
:107D8000F1F31D499B00C0E91013012403F01C030B
:107D900004FA03F3002515604B60FFF747FF836C7F
:107DA00041681D60D0E913325A604A1E032A06D882
:107DB000124B0B449B0094401D60114B5C640023EC
:107DC000C363C0E91533C0E90B33C0E90D33C365A4
:107DD00080F8253080F82430184638BD094B13440C
:107DE000B3FBF1F308499B00CDE70120F5E700BFA5
:107DF00007040240F8FFFDBF000002403F82001070
:107E000000090240F8FBFDBF0004024070B590F885
:107E10002450012D04463BD090F825600125AE4248
:107E200080F824504FF000062CD1022580F8255010
:107E30000568C6632E6826F001062E60FFF7DCFE9B
:107E4000036BBBB12B6843F00E032B60A36C1A6865
:107E5000D20342BF1A6842F480721A60636D1BB18C
:107E60001A6842F480721A602B6843F001032B6099
:107E7000002070BD2B6823F004032B602B6843F0B7
:107E80000A03E2E78023C36380F824602846F0E712
:107E90000220EEE7034640B190F82520022A06D0E2
:107EA0000422C263002280F8242001207047026867
:107EB000806C116821F00E011160016821F480715D
:107EC0000160116821F001011160D3E9100202F094
:107ED0001C0101228A404260D3E9132151605A6D8E
:107EE00032B1116821F480711160D3E9162151601B
:107EF0000122002083F8252083F82400704710B564
:107F000090F82530022B03D00423C363012010BD59
:107F100003681A6822F00E021A601A6822F0010241
:107F20001A60826C136823F480731360D0E9101315
:107F300003F01C02012393404B60D0E913325A60D6
:107F4000436D33B11A6822F480721A60D0E9163298
:107F50005A60012380F82530836B002480F8244088
:107F600013B198472046D2E71846D0E770B4426C68
:107F7000046C036826681D6802F01C02042191400D
:107F800031420FD015F0040F0CD01A6892065EBF74
:107F90001A6822F004021A60036B6160002B33D070
:107FA00070BC184702219140314217D015F0020FE2
:107FB00014D01A68940606D41A6822F00A021A60CD
:107FC000012280F82520114A93428CBF104B114B9F
:107FD0005960002380F82430C36ADFE7082191400C
:107FE000314211D029070FD5196821F00E0119600F
:107FF000012303FA02F26260C36380F82530002394
:1080000080F82430436BC9E770BC704780000240A1
:1080100000040240000002400A4A536943F48023EE
:1080200030B55361EFF3108472B60023CD58C550BC
:108030000433B3F5807FF9D11369DB03FCD484F3F7
:10804000108830BD00400058064B5A69002ABFBF57
:10805000054A9A6002F188329A60BABF5869C00F27
:10806000002070470040005823016745044B5A69BF
:1080700042F000425A615869C043C00F704700BFC8
:108080000040005870B50546FAF7A0FF124E0446AE
:108090003369D90313D43369DA0744BF012232614B
:1080A0004CF2FA32134011D10B4E306910F480209B
:1080B0000BD0FAF78BFF001BA842F6D304E0FAF7C7
:1080C00085FF001BA842E3D3032070BD024A136161
:1080D000024A01205360F8E70040005838110020A0
:1080E0002DE9F041184D98462B78012B06460C4699
:1080F000174626D001232B704FF47A7000236B6053
:10810000FFF7C0FFA0B9012E16D1104A536943F002
:10811000010353612760BFF36F8FC4F804804FF4ED
:108120007A70FFF7AFFF094A536923EA06035361E8
:1081300000232B70BDE8F08139462046FFF76CFF25
:10814000EDE70220F6E700BF38110020004000589C
:10815000054A536923F47E7343EAC00040F480303B
:1081600040F0020050617047004000582DE9F04196
:10817000234F3B78012B054688463FD001233B70B7
:108180004FF47A7000237B60FFF77CFF044688B9C8
:108190002B68042B13D11B4A536943F4803343F0FB
:1081A000040353614FF47A70FFF76CFF0446154BDC
:1081B0001A681B6800233B702046BDE8F0814FF031
:1081C000FF33C8F800306E68D5E901321344B3427A
:1081D0000AD93046FFF7BCFF4FF47A70FFF752FF21
:1081E00050B1C8F800600446064A536923F47E7310
:1081F00023F002035361DAE70136E5E70224DBE707
:1082000038110020004000582DE9F04F524C002357
:108210004FF00F090A6832FA03F501D1BDE8F08F7B
:10822000012505FA03F818EA020200F08E804E6874
:10823000032706F003054FEA430E07FA0EFC6F1EF4
:10824000012F6FEA0C0C32D8876807EA0C0ACF6856
:1082500007FA0EF747EA0A078760476827EA08081F
:10826000C6F300179F4047EA08074760C76807EA58
:108270000C088F6807FA0EF747EA0807022DC76057
:1082800017D14FEAD30800EB880803F0070AD8F8A3
:1082900020704FEA8A0A09FA0AFB27EA0B0B0F69DA
:1082A00007FA0AF747EA0B07C8F8207001E0032D28
:1082B000DCD1076805FA0EF507EA0C073D4316F412
:1082C000403F056041D023F0030707F1804707F5E1
:1082D000803703F0030CBD684FEA8C0C4FF0070E9B
:1082E0000EFA0CFEB0F1904F25EA0E0E2FD01B4D6A
:1082F000A8422ED005F58065A8420CBF02250725AF
:1083000005FA0CF545EA0E05BD602568D74316F45D
:10831000801F0CBF3D4015432560656816F4001FA3
:108320000CBF3D4015436560D4F8805016F4803F83
:108330000CBF3D401543C4F88050D4F88450B603B8
:1083400054BF3D401543C4F88450013362E7002513
:10835000D6E70125D4E700BF000800580004004814
:10836000374A2DE9F04F00234FF0010A4FF0070B79
:108370004FF00F0931FA03F401D1BDE8F08F0AFA8A
:1083800003FC1CEA010654D023F0030404F18044EA
:1083900004F5803403F00307A568BF000BFA07F863
:1083A000B0F1904F08EA050E45D0264DA84244D0C2
:1083B00005F58065A8420CBF02250725BD4075451F
:1083C00017D1D2F8805025EA0605C2F88050D2F8BD
:1083D000845025EA0605C2F88450156825EA06058A
:1083E0001560556825EA06055560A56825EA080563
:1083F000A560056803265C0006FA04F423FA06F675
:10840000254300EB8606056003F00705376AAD00DB
:1084100009FA05F527EA05073762856825EA0405A4
:108420008560456825EA0C054560C56825EA0404B1
:10843000C46001339EE70025C0E70125BEE700BF09
:1084400000080058000400480369194214BF0120C5
:10845000002070470AB18161704781627047000057
:10846000044AD168014208B502D0D060FBF70EFB88
:1084700008BD00BF0008005803689A69910744BF0F
:1084800000229A629A69D2075EBF9A6942F001029D
:108490009A61704730B5039D04682B4343EA024359
:1084A000064A6068C1F309010B4342EA555223F0C2
:1084B000004320EA02000343636030BDFF63FF0313
:1084C00003682DE9F0419C6914F0100405460F463D
:1084D00016466FD010220024DA61A0462B689A69F4
:1084E000900661D4B8F1000F35D044F004040120A7
:1084F0002E68B369D90541BF4FF48072F26144F030
:10850000010401205A0541BF4FF4806244F0080481
:10851000F26101209B054FD54FF4007344F0020433
:10852000F3612846FFF7A8FF736823F0FF7323F475
:108530008B3323F4FF7323F0010373606B6C2343CD
:108540006B64202385F84130002385F8423085F89C
:108550004030012032E07A1CC1D0FAF737FD801B91
:10856000B84201D8002FB9D12B68596895F842203C
:1085700098690004D2B20AD5490408D4202A06D04A
:108580005A6842F480425A60FAF720FD06462B688A
:108590009B699B06A2D4FAF719FD801B1928F6D90E
:1085A00020244FF0010899E7B8F1000F9DD1202257
:1085B000DA619AE720469BE70028B2D1BDE8F08156
:1085C00070B504460D46164623689B699B0701D586
:1085D000002070BD324629462046FFF771FFA0B942
:1085E0006A1CF1D0FAF7F2FC801BA84201D8002DDA
:1085F000EAD1636C43F020036364202384F84130A4
:10860000002384F8423084F840300120E1E770B55F
:1086100004460D46164623689B695B070ED4324616
:1086200029462046FFF74CFF38BB23689A6991061C
:1086300025D59A69520703D5228D0AB1002070BD55
:108640009A6912F010021CBF1022DA614FF020016B
:1086500018BF04226264D9615A6822F0FF7222F4C2
:108660008B3222F4FF7222F001025A60002384F858
:10867000411084F8423084F840300120DFE7FAF7F7
:10868000A5FC801BA84201D8002DC4D1636C43F027
:1086900020036364202384F841300023EBE72DE9B5
:1086A000F041069F0446884616461D462268936997
:1086B00038EA03030CBF01230023B34201D000209A
:1086C00015E06B1CF3D0FAF781FCC01BA84201D85F
:1086D000002DEBD1636C43F020036364202384F806
:1086E0004130002384F8423084F840300120BDE856
:1086F000F08170B504460D46164623689B699B06BB
:1087000001D5002070BD324629462046FFF7D8FE2D
:1087100090B9FAF75BFC801BA84201D8002DECD180
:10872000636C43F020036364202384F8413000230A
:1087300084F8423084F840300120E3E710B5044665
:1087400000284AD090F8413003F0FF021BB980F8AE
:108750004020FAF73DF9242384F8413023681A6851
:1087600022F001021A60626822F070621A619A684F
:1087700022F400429A60D4E90221012924D142F472
:1087800000429A605A6842F0007242F400425A6015
:10879000DA6822F40042DA60D4E904210A43A169CC
:1087A00042EA0122DA60D4E907210A431A601A6812
:1087B00042F001021A6000202023606484F84130F6
:1087C000206384F8420010BD42F4044202299A60FA
:1087D00004BF4FF400625A60D4E70120F3E70000C1
:1087E0002DE9F347984690F841300A9F202B044624
:1087F0000E46914640F0868090F84030012B00F004
:1088000081804FF0010A80F840A0FAF7DFFB1923BE
:108810000546009052464FF400412046FFF73FFFC7
:1088200018B1012002B0BDE8F087212384F841305F
:10883000102384F842306064A4F82A80638DC4F861
:1088400024909BB2FF2B60632F4B26D9FF222285F9
:1088500000934FF0807331462046FFF71BFE638D77
:108860009BB22A4639462046FBB9FFF742FF002853
:10887000D7D123682021D9615A6822F0FF7222F4EF
:108880008B3222F4FF7222F001025A6084F8411008
:1088900084F8400084F84200C4E7628D009392B2ED
:1088A00022854FF00073D2B2D5E7FFF789FE00288A
:1088B000B7D1636A226813F8011B91626362638D0A
:1088C000228D013B9BB26385638D013A92B29BB2CC
:1088D0002285002BC3D0002AC1D100953B468021C0
:1088E0002046FFF7DCFE00289BD1638D9BB2FF2B57
:1088F00003D9FF2222850090ABE7628D009092B2EF
:108900002285CEE702208DE7002000802DE9F34785
:10891000984690F841300A9F202B04460E46914617
:1089200040F0878090F84030012B00F082804FF0BB
:10893000010A80F840A0FAF749FB19230546009088
:1089400052464FF400412046FFF7A9FE18B101201E
:1089500002B0BDE8F087222384F84130102384F868
:1089600042306064A4F82A80638DC4F824909BB2DE
:10897000FF2B6063304B26D9FF22228500934FF0F6
:10898000807331462046FFF785FD638D9BB22A46F2
:1089900039462046FBB9FFF7ACFE0028D7D1236843
:1089A0002021D9615A6822F0FF7222F48B3222F41E
:1089B000FF7222F001025A6084F8411084F84000EE
:1089C00084F84200C4E7628D009392B222854FF092
:1089D0000073D2B2D5E7FFF71AFE0028B7D123689B
:1089E0005A6A636A1A70636A228D01336362638D07
:1089F000013B9BB26385638D013A92B29BB22285A3
:108A0000002BC2D0002AC0D100953B4680212046D1
:108A1000FFF745FE00289AD1638D9BB2FF2B03D947
:108A2000FF2222850090AAE7628D009092B22285F3
:108A3000CDE702208CE700BF0024008010B590F83D
:108A40004120202A0346D4B21CD190F84020012AAC
:108A500018D0242280F841200268106820F001001C
:108A60001060106820F4805010601068014311609D
:108A70001168002041F00101116083F8414083F842
:108A8000400010BD0220FCE710B590F84120202ADC
:108A90000346D4B21BD190F84020012A17D02422DB
:108AA00080F841200268106820F001001060106812
:108AB00020F4706040EA012111601168002041F04B
:108AC0000101116083F8414083F8400010BD02208D
:108AD000FCE70000024A136843F480731360704798
:108AE000000400580D4B10B55B690C4628B99A0577
:108AF00007D500F027F820B110BD9B0501D400F088
:108B000019F8074A1369012C23F00403136101D1FA
:108B100030BFF1E740BF20BF20BFEDE700040058A1
:108B200000ED00E0024B186800F4C060704700BF21
:108B300000040058024A136843F4804313607047EE
:108B4000000400580C4A136823F4804313600B4B55
:108B50001B6832214B430A49B3FBF1F35169890584
:108B600000D533B9536913F4007F14BF03200020EC
:108B70007047013BF2E700BF0004005828080020BE
:108B800040420F000B4A136823F0070343F002032F
:108B90001360094B1A69012842F004021A6105D1D9
:108BA00030BF1A6922F004021A61704740BF20BF2B
:108BB00020BFF6E70004005800ED00E04FF0B0439E
:108BC0001868C0F3404070474FF0B0431868C0F3D6
:108BD000400070474FF0B042536823F47F4343EAAC
:108BE0000023536070474FF0B0431868C0F34060F3
:108BF000704700007FB54FF0B0432C4AD3F80831DE
:108C0000C0F3031003F00F0352F82040284A52F833
:108C10002330B4FBF3F4FFF785FF264B054693E8BA
:108C20000700B5F5007F04AB03E9070010D0224B25
:108C30009C4218D303F5B70303F67F539C4229D90E
:108C400003F5741303F510639C4225D802230BE04F
:108C50001A4B9C4207D91A4B9C421BD903F5370388
:108C600003F5D853F0E7002304AA02EB830353F87B
:108C70000C4C144D2B6823F0070323432B60FAF7A9
:108C8000A5F906462B6803F007039C4206D1002095
:108C900004B070BD0123E7E70024EAE7FAF796F98C
:108CA000801B0228EED90320F2E700BF9C70010868
:108CB0003C700108D86E0108C0CF6A00BFEA2101EC
:108CC0003F933402004000584FF0B04310B59A680B
:108CD000D96812F00C0205D00C2A4AD101F0030326
:108CE000012B50D14FF0B0412B480B6813F0080313
:108CF00006D00B6813F0080337D1D1F8941007E0C1
:108D00000C68240756BFD1F894300968C3F30323D5
:108D100050F82330002A0CBF184600204FF0B04115
:108D20008A6802F00C020C2A1ED1CA6802F0030203
:108D3000022A2ED0032A06D10B68184A13F4801F8A
:108D4000174B18BF13464FF0B042D068D168D268B5
:108D5000C0F306205843C1F302130133B0FBF3F014
:108D6000530F0133B0FBF3F010BD0B68C3F30313D3
:108D7000CEE7042A0AD0082A05D11B6813F4801311
:108D800004D10748CAE700231846C7E70348002371
:108D9000C4E7024BD7E700BF9C7001080024F40031
:108DA0000048E80108B5FFF78FFF4FF0B043044AD1
:108DB0009B68C3F3031352F82330B0FBF3F008BDF4
:108DC0003C7001082DE9F0410446002853D04FF0D3
:108DD000B0439D68DE6803689B0605F00C0506F04D
:108DE000030668D5026A1DB10C2D46D1012E44D16F
:108DF000002A40D04FF0B043A16A1A68170756BF47
:108E0000D3F894301B681B0903F0F00399421FD973
:108E10000846FFF7EFFE00282DD14FF0B04213684F
:108E200043F0080313601368A16A23F0F0030B43B7
:108E30001360606AFFF7CEFEFFF7B4FFAB4B18601C
:108E4000AB4B1868FAF7C0F8002834D0BDE8F081C1
:108E50004FF0B042136843F008031360136823F027
:108E6000F0030B431360606AFFF7B4FE0846FFF798
:108E7000C1FE0028E0D00120E8E74FF0B043002A0F
:108E800054D01A6842F001021A60FAF79FF80746B8
:108E9000FFF79AFE002842D04FF0B042136843F02B
:108EA000080313601368A16A23F0F0030B431360F7
:108EB000606AFFF78FFE2368D80748D423689907B4
:108EC00000F18C8023681E0740F1FA80A3694FF0FF
:108ED000B046002B00F0E180D6F89430E16903F051
:108EE0001002914200F0C48003F00302022AC2D0B3
:108EF000D80740F1B380D6F8943023F00103C6F8C8
:108F00009430FAF763F80746D6F89430990740F1A1
:108F1000A580FAF75BF8C31B112BF5D904E0FAF72B
:108F200055F8C01B0228B3D903208FE71A6822F036
:108F300001021A60FAF74AF80746FFF745FE0028D3
:108F4000B9D0FAF743F8C01B0228F6D9ECE7082D90
:108F500003D00C2D05D1032E03D16368002BADD1B6
:108F600089E74FF0B043A1681A6822F480120A43DF
:108F70001A606268B2F5803F10D11A6842F48032FC
:108F80001A60FAF723F80746FFF718FE002895D174
:108F9000FAF71CF8C01B6428F6D9C5E7B2F5041F20
:108FA00004D11A6842F400121A60E6E7196821F445
:108FB00080311960196821F400111960002AE0D18C
:108FC000FAF704F80746FFF7F9FD00283FF476AFFB
:108FD000F9F7FCFFC01B6428F5D9A5E7042D236928
:108FE00003D00C2D0ED1022E0CD1002B3FF443AF39
:108FF0004FF0B0426169536823F0FE4343EA0163D6
:1090000053605FE74FF0B046BBB1336843F4807301
:109010003360F9F7DBFF074633685A0507D57368F5
:10902000626923F0FE4343EA026373604AE7F9F79B
:10903000CDFFC31B022BEFD976E7336823F480738F
:109040003360F9F7C3FF074633685B057FF53AAF36
:10905000F9F7BCFFC31B022BF6D965E74FF0B0420E
:10906000E169D2F8943023F010030B43C2F8943036
:109070004FF0B047D7F8943043F00103C7F894306D
:10908000F9F7A4FF0646D7F894309A0718D4F9F7F1
:109090009DFF831B112BF6D946E7D6F8943023F0B9
:1090A0000103C6F89430F9F791FF0746D6F89430DB
:1090B0009B0705D5F9F78AFFC31B112BF6D933E7B8
:1090C0002368580754D50B4F3B68D90514D4FFF7D4
:1090D00001FDF9F77BFF06463B68DA050CD4F9F78A
:1090E00075FF831B022BF7D91EE700BF280800205D
:1090F0002C08002000040058E3684FF0B046002B15
:1091000058D023F08003052B02BFD6F8903043F0EF
:109110000403C6F890304FF0B046F9F757FFD6F881
:10912000903043F001030746C6F8903041F288388A
:10913000D6F890309B0705D4F9F748FFC31B434589
:10914000F6D9F1E6E36823F00403812B1BD1F9F78C
:109150003DFFD6F8903043F08003C6F890300746C4
:109160004FF0B04641F28838D6F89030180504D553
:10917000E06A00284AD1002068E6F9F727FFC01B03
:109180004045F1D9D0E6F9F721FFD6F8903023F029
:109190008003C6F8903007464FF0B04641F2883859
:1091A000D6F890301905E3D5F9F710FFC01B4045FC
:1091B000F6D9B9E6F9F70AFFD6F8903023F0800324
:1091C0000746C6F8903041F28838D6F890301A0534
:1091D00016D4F9F7FBFED6F8903023F00103C6F859
:1091E000903007464FF0B04841F28836D8F89030BA
:1091F0009B07BDD5F9F7EAFEC31BB342F6D993E648
:10920000F9F7E4FEC01B4045DFD98DE60C2D4ED0AA
:109210004FF0B04302281A6822F080721A6033D1EE
:10922000F9F7D4FE0546FFF7DEFC38BBD4E90C3174
:109230004FF0B0420B43D0682D4901400B43E16B26
:109240000B43216C0B43616C0B43A16B43EA01237D
:10925000D360136843F080731360D36843F0805386
:10926000D360F9F7B3FE0446FFF7BDFC002882D1B6
:10927000F9F7ACFE001B0A28F6D955E6F9F7A6FE69
:10928000401B0A28CFD94FE6F9F7A0FE0446FFF7A6
:10929000AAFC30B94FF0B042164BD1680B40D360F6
:1092A000D4E5F9F793FE001B0A28F0D93CE6012823
:1092B0003FF4CCAD4FF0B043226BDB6803F0030109
:1092C00091427FF4D8AD616B03F070028A427FF463
:1092D000D2ADA16B03F4FE42B2EB012F7FF4CBAD14
:1092E000626C03F0604393423FF445AFC3E500BFB7
:1092F0008C80C111FCFFFEEE2DE9F0410D460446C5
:1093000010B90120BDE8F081684E336803F007030F
:109310008B4216D323689A0727D54FF0B047A2682F
:10932000BB6823F0F0031343BB60F9F74FFE06461A
:10933000BB68DB0319D4F9F749FE831B022BF7D96D
:1093400011E0336823F007030B433360F9F73EFE67
:109350000746336803F00703AB42DBD0F9F736FE6C
:10936000C01B0228F5D90320CCE72368580617D57F
:109370004FF0B0476269D7F8083123F00F0343EA92
:109380001213C7F80831F9F721FE0646D7F808315D
:10939000D90305D4F9F71AFE831B022BF6D9E2E7AD
:1093A00023685A0713D54FF0B047E268BB6823F42F
:1093B000E0631343BB60F9F709FE0646BB689B03F5
:1093C00005D4F9F703FE831B022BF7D9CBE72368FB
:1093D000180714D54FF0B0472269BB6823F46053D7
:1093E00043EAC203BB60F9F7F1FD0646BB685903C7
:1093F00005D4F9F7EBFD831B022BF7D9B3E72368FC
:10940000DA070FD4294C236803F00703AB4239D89D
:10941000FFF7C8FC264B1860264BBDE8F0411868E2
:10942000F9F7D2BD6268022A1DD1FFF7C7FB0028F9
:109430003FF467AF4FF0B04641F28838B36823F08D
:1094400003031343B360F9F7C1FD0746B3686268CD
:1094500003F00C03B3EB820FD4D0F9F7B7FDC01BB8
:109460004045F3D97FE7032A02D1FFF7BCFBDEE7D3
:1094700012B9FFF7A9FBDAE74FF0B0431B685B05B1
:10948000D8D43EE7236823F007032B432360F9F782
:109490009DFD0646236803F00703AB42B8D0F9F7F9
:1094A00095FD801B0228F5D95DE700BF00400058FC
:1094B000280800202C08002008B5FFF773FC4FF0A7
:1094C000B043044A9B68C3F3022352F82330D840C8
:1094D00008BD00BF7C70010808B5FFF763FC4FF0C2
:1094E000B043044A9B68C3F3C22352F82330D840E8
:1094F00008BD00BF7C7001084FF0B043D3F8900066
:10950000C0F3400070474FF0B0410209D1F88830F5
:1095100002F47F22000123EA020300F47F200343C8
:10952000C1F8883070474FF0B041020CD1F8883054
:10953000120423EA020343EA0040C1F8880070479E
:1095400070B5066816F48036044638D0FFF7C2FAC4
:10955000F9F73CFD614E05463368DB0529D54FF030
:10956000B043616BD3F8902002F44072914214D062
:10957000D3F89010D3F8902042F48032C3F89020B2
:10958000D3F8902021F4407022F480328D07C3F884
:109590009020C3F8900000F190804FF0B042616BD2
:1095A000D2F8903023F440730B43C2F89030002679
:1095B00005E0F9F70BFD401B0228CDD903262568ED
:1095C000E8070AD54FF0B0416268D1F8883023EA45
:1095D000124392B21343C1F88830A9070AD54FF05D
:1095E000B041A268D1F8883023EA124392B2134303
:1095F000C1F88830AA0609D54FF0B0422169D2F8E7
:10960000883023F440630B43C2F88830AB0502D5A1
:10961000206AFFF788FF680502D5606AFFF783FFBD
:10962000290502D5A06AFFF77EFF6A0602D56069A8
:10963000FFF769FF2B0602D5A069FFF764FFE80575
:1096400002D5E069FFF75FFFE90610D54FF0B042A1
:10965000E168D2F8883023F440730B43C2F88830B5
:10966000B1F5807F02BFD36843F08073D3602A04D2
:109670000ED54FF0B042216BD2F8883023F0404332
:109680000B43C2F8883019B9D36843F08073D360B4
:109690006B0410D54FF0B042E16AD2F8883023F065
:1096A00040530B43B1F1005FC2F8883003D1D36857
:1096B00043F48033D360304670BDF9F787FC41F244
:1096C00088360546FFF718FF01283FF466AFF9F723
:1096D0007DFC401BB042F5D970E700BF0004005884
:1096E00030B590F82C30012B02464FF0020022D00A
:1096F000174B82F82D00CA24012582F82C505C6299
:1097000053245C62B1F5807F146B996914D121F404
:1097100088519961596C24F0010421F00041596489
:109720001463DD650A4BFF2159620020012382F892
:109730002D3082F82C0030BD21F408519961D96C8C
:1097400024F0020421F00041D9641463D865E9E7EC
:109750000028004070B50B4E036B756D1D40EA0785
:10976000044603D50123F365F9F7F9FDAB0704D5EA
:109770000223F365204600F0CBF9012384F82D3055
:1097800070BD00BF0028004038B50A4CE36823F0E4
:109790002003E360F9F71AFC0546E3689B0601D550
:1097A000002038BDF9F712FC401BB0F57A7FF4D9E0
:1097B0000320F6E7002800402DE9F041114DEC6848
:1097C00014F0400407461AD1EB6843F08003EB60C5
:1097D000F9F7FCFB4FF003080646EB685B0601D483
:1097E000032C02D12046BDE8F081F9F7EFFB801B86
:1097F000B0F57A7F84BF87F82D800324EDE700243D
:10980000F0E700BF0028004038B50F4CE36823F0B4
:109810008003E360A3699B06054606D4FFF7B4FF07
:1098200010B1032085F82D0038BDA36923F0200373
:10983000A361FFF7A9FF10B1032085F82D00A369EC
:1098400043F02003A361EFE70028004038B5044649
:1098500000284BD090F82D3003F0FF021BB980F8A0
:109860002C20F9F7C1F90223214D84F82D30EB6843
:10987000DB0632D4CA236B6253236B622046FFF7A8
:109880009BFF78BBAB6923F08E6323F04003AB6191
:1098900021696368AA690B431343A2691343AB614F
:1098A000D4E9022343EA02432B61D4E90931EA688F
:1098B0000B4322F4F8521343EB602046FFF7A4FF5A
:1098C00080B9D4E90713AA690B4322F0604213431D
:1098D00062691343AB61FF236B62012384F82D306F
:1098E000002002E0024BFF225A6238BD0120FCE753
:1098F000002800400023092803D840EA0310C0B222
:1099000070470A380133C0B2F5E700002DE9F0478F
:1099100090F82C30012B05464FF0020069D001234E
:1099200085F82C304E4B85F82D00DE6806F4407625
:10993000B6F5807F78D04C69087891F8019091F85D
:1099400002A091F82470002A55D19B6913F04003BE
:1099500008BFCB70FFF7CEFF80464846FFF7CAFF2F
:1099600002465046FFF7C6FF81463846FFF7C2FF62
:109970000B6ACF78234343EA875343EA090343EA58
:10998000084343EA022343EA0063354ACA2050628F
:10999000532050628C6A8869B4F5807F946945D100
:1099A00024F4885494610124D465B6F5807F09BFFE
:1099B000CB6913640343536418BF5064284B4A684F
:1099C0001A672A6B42F001022A639A6942F48852AC
:1099D0009A61244AD2F8803043F40033C2F88030D0
:1099E0001F4BFF225A620020012385F82D3085F895
:1099F0002C00BDE8F087B4F1803F07D0B4F5000F2C
:109A000004D09B6913F0400308BFCB700B6ACA787F
:109A10001C4344EA0A0444EA004343EA092343EAB4
:109A2000825343EA0763B0E70023AEE724F4085407
:109A300094610224D465B6F5807F09BFCB69936435
:109A40000343D36418BFD064054B4A685A672A6B36
:109A500042F002022A639A6942F40852B8E700BF52
:109A6000002800400008005890F82C20012A0346E6
:109A70004FF0020012D00A4A83F82D00CA21516229
:109A800053215162916941F020019161FF2151629E
:109A90000020012283F82D2083F82C00704700BF9E
:109AA0000028004090F82C20012A03464FF00200C5
:109AB00019D00D4A83F82D00CA21516253215162F9
:109AC00091690A4841F080019161D0F8801041F419
:109AD0008021C0F88010FF2151620020012283F80C
:109AE0002D2083F82C007047002800400008005803
:109AF000064B5A6D520610B5044603D54022DA656E
:109B0000F9F730FC012384F82D3010BD0028004007
:109B10007047890001F1804101F531410A607047C9
:109B2000890001F1804101F531410868704700006A
:109B3000034AD2F8903043F40043C2F890307047A3
:109B400000040058034AD2F8903023F40043C2F8CE
:109B50009030704700040058074B1A6822F040020A
:109B60001A6040F441704FF4B85218605A601A6895
:109B700042F040021A6070470000015837B50546B0
:109B800000284ED0837903F0FF046BB1032C0BD077
:109B9000254B4FF400629A612868FFF7DDFF00242F
:109BA00001232B71AC602FE000236B712846F9F77D
:109BB00025F91E4AD2F8903043F48053C2F8903011
:109BC000002CE5D102234FF0B042AB71D2F89430B3
:109BD00023F40043C2F89430154B1B681C214B43FF
:109BE000DB0C64214B430193019B93B90124AC60CE
:109BF000FFF79EFF0C4B9A6842F400629A604FF4A4
:109C000000629A61002CC7D00123AB71204603B0DB
:109C100030BD019B013B0193D2F894305B04E3D447
:109C2000E6E70124F2E700BF0004005800080058EE
:109C30002808002037B5174D2B6802461C204343E7
:109C4000DB0C6420434314480193019B93B901202A
:109C50009060114C21732B681C214B43DB0C642159
:109C60004B430193019B6BB9012090600A4BDB6869
:109C700003B030BD019B013B019383689C07E4D591
:109C80000020E6E7019B013B0193A368DB07E9D5D0
:109C9000ECE700BF280800200000015837B5184D38
:109CA0002B6802461C204343DB0C642043431548C9
:109CB0000193019BA3B901209060124CFF232373F1
:109CC0002B681C256B43DB0C64256B430193019BC4
:109CD00073B9012090600B4BDB680B7003B030BD93
:109CE000019B013B019383689C07E2D50020E4E7D8
:109CF000019B013B0193A368DB07E8D5EBE700BFBD
:109D000028080020000001580F4B13B51B680F4CAA
:109D1000182253431B0D6422534301460193626989
:109D2000019B02F0040223B902238B60012002B0E0
:109D300010BD019B013B0193606910F00200F6D059
:109D4000002AECD11046F2E7280800200004005851
:109D500007B50379012B0FD10A4B1B681822534317
:109D60001B0C0193FFF7EEFE019B013B0193019B4E
:109D7000002BF9D1FFF7DCFE03B05DF804EBFFF731
:109D8000C3BF00BF28080020F8B51E468379012B09
:109D9000154604460F46DAB22DD14379012B2AD05D
:109DA000022342718371FFF7D3FF0D212046FFF795
:109DB000C9FEFFF73FFF390A2046FFF73BFFF9B224
:109DC0002046FFF737FF2E44B5420ED12046FFF75D
:109DD000AFFEFFF799FFA06801230038A3714FF091
:109DE000000318BF01206371F8BD15F8011B204660
:109DF000FFF720FFE8E70220F6E7F8B51E46837973
:109E0000012B154604460F46DAB22FD14379012BB8
:109E10002CD04271FFF79CFF1D212046FFF792FED8
:109E2000FFF708FF390A2046FFF704FFF9B2204682
:109E3000FFF700FF00212046FFF7FCFE2E44B5424D
:109E40000ED12046FFF774FEFFF75EFFA0680123E6
:109E50000038A3714FF0000318BF01206371F8BDF3
:109E600029462046FFF71AFF0135E8E70220F6E70A
:109E7000F8B51F468379012B154604460E46DAB223
:109E80002CD14379012B29D04271FFF761FF06F0F5
:109E9000EF03A3F18402534253412371314620461C
:109EA000FFF750FEFFF7C6FE2F44AF4210D1FFF779
:109EB0003FFE842E02D02046FFF726FFA068012334
:109EC0000038A3714FF0000318BF01206371F8BD83
:109ED00015F8011B2046FFF7ADFEE6E70220F6E786
:109EE000F8B51E468379012B154604460F46DAB2B3
:109EF00027D14379012B24D04271FFF729FF39463E
:109F00002046FFF71FFEFFF795FE00212046FFF7D2
:109F100091FE2E44B5420ED12046FFF709FEFFF711
:109F2000F3FEA06801230038A3714FF0000318BFAF
:109F300001206371F8BD29462046FFF7AFFE0135C9
:109F4000E8E70220F6E737B50023ADF8043001AAB0
:109F5000022312210546FFF7C3FFBDF80440022388
:109F600064BA01AAA4B219462846FFF781FFE207A6
:109F700002D5284609F0DAFBA30702D5284609F0E6
:109F8000DBFB600702D5284609F000FC210702D55B
:109F9000284609F001FCE20602D5284609F002FC39
:109FA000A30602D5284609F0EBFB600602D5284639
:109FB00009F0C8FB210606D514F4807118BF0121F1
:109FC000284609F0C5FBA20502D5284609F0D0FBBA
:109FD000630402D5284609F0EBFB03B030BDF8B5A9
:109FE0001E468379012B154604460F46DAB227D167
:109FF0004379012B24D04271FFF7AAFE0E2120469F
:10A00000FFF7A0FDFFF716FE39462046FFF712FEC8
:10A010002E44B5420ED12046FFF78AFDFFF774FEAD
:10A02000A06801230038A3714FF0000318BF01207E
:10A030006371F8BD15F8011B2046FFF7FBFDE8E74B
:10A040000220F6E7F8B51E468379012B1546044633
:10A050000F46DAB22BD14379012B28D04271FFF79A
:10A0600077FE1E212046FFF76DFDFFF7E3FD394621
:10A070002046FFF7DFFD00212046FFF7DBFD2E44E1
:10A08000B5420ED12046FFF753FDFFF73DFEA06815
:10A0900001230038A3714FF0000318BF0120637142
:10A0A000F8BD29462046FFF7F9FD0135E8E7022013
:10A0B000F6E7026852E8003F23F0C00342E80031AF
:10A0C00002680029F5D102F1080353E8003F23F4A8
:10A0D000000302F1080C4CE800310029F3D12023E1
:10A0E000C0F888307047000010B5026852E8003FA1
:10A0F00023F4907342E8003102680029F5D10F4C37
:10A1000002F1080353E8003F234002F1080C4CE839
:10A1100000310029F4D1C36E012B07D152E8003F72
:10A1200023F0100342E800310029F7D12023C0F8C2
:10A130008C300023C366436710BD00BFFEFFFFEFF6
:10A14000F8B504461346D4F88850202D32D1F1B129
:10A15000EAB1E06FA4F85620A4F85420002621228A
:10A16000C4F890602165C4F88820226888B1124F35
:10A17000C762124F0763124F2832C0E90D76FDF710
:10A1800045FE30B11023C4F89030C4F88850012047
:10A190000FE0236840221A62226802F1080353E8A4
:10A1A000003F43F0800302F1080141E8003000283D
:10A1B000F3D1F8BD0220FCE7C5A100080DA20008FC
:10A1C00019A2000808B50346806A1B681B6813F0D3
:10A1D000200317D1A0F85630026802F1080353E8B3
:10A1E000003F23F08003083242E800310268002972
:10A1F000F2D152E8003F43F0400342E80031002929
:10A20000F7D108BDF9F7E4F9FBE7704708B5806AB4
:10A21000FFF7FBFF08BD7047806A38B50468D0F8C7
:10A220008830D0F88C50A268120606D5212B04D1B4
:10A230000023A0F85630FFF73CFFA3685B0606D565
:10A24000222D04D10023A0F85E30FFF74DFFD0F897
:10A25000903043F01003C0F89030FFF7DCFF38BDBA
:10A2600008B5806A0023A0F85E30A0F85630FFF7EA
:10A27000D2FF08BD704700000368D9691A682DE94C
:10A28000F04140F60F0631429D68044610D18E061B
:10A2900040F1978002F0200605F080573E4300F021
:10A2A0009080436F002B00F08580BDE8F041184797
:10A2B000AB4EAC482E401040304300F08280CF07B8
:10A2C00009D5D00507D501201862D4F8900040F0D8
:10A2D0000100C4F890008F0709D5E80707D50220D0
:10A2E0001862D4F8900040F00400C4F890004F07C2
:10A2F00009D5E80707D504201862D4F8900040F08B
:10A300000200C4F890000F070BD502F02000304384
:10A3100007D008201862D4F8900040F00800C4F874
:10A3200090000E050AD5500108D54FF40060186260
:10A33000D4F8903043F02003C4F89030D4F8903033
:10A34000002B37D08B0609D502F0200205F080558E
:10A350002A4303D0636F0BB1204698472668D4F890
:10A360009020B36802F0280203F0400353EA02058C
:10A37000204621D0FFF7B8FEB3685F0617D52268E4
:10A3800002F1080353E8003F23F04003083242E89B
:10A3900000310029F3D1D4F8800040B1724B8363BF
:10A3A000FDF7ADFD30B1D4F88000836B7DE720462A
:10A3B000FFF731FFBDE8F081FFF72DFFC4F89050A3
:10A3C000F8E7E06E012840F08980CE0640F18680F3
:10A3D000D00640F1838010221A629A6851064BD54C
:10A3E000D4F8802011684A6892B2002AE2D0B4F80A
:10A3F0005C009042DED9A4F85E200A6892062FD451
:10A4000053E8002F22F4807243E800210029F7D19D
:10A4100003F1080252E8002F22F0010203F10800C4
:10A4200040E800210029F3D103F1080252E8002F8F
:10A4300022F0400203F1080040E800210029F3D196
:10A440002022C4F88C20E16653E8002F22F010028D
:10A4500043E800210029F7D1D4F88000FDF71AFD68
:10A4600002232367B4F85E30B4F85C10C91A89B2CD
:10A470002046FFF7FFFE9DE7B4F85E20B4F85E00CB
:10A48000B4F85C1080B292B2002893D0891A89B2D5
:10A4900000298FD053E8002F22F4907243E8002067
:10A4A0000028F7D1314D03F1080252E8002F2A406D
:10A4B00003F1080646E800200028F4D12022C4F861
:10A4C0008C206067E06653E8002F22F0100243E81A
:10A4D00000200028F7D102232367C9E7CF0209D55E
:10A4E0006E0207D54FF4801220461A62BDE8F04193
:10A4F00000F0F2BD08060BD502F0800005F400055F
:10A50000284305D0A36F002B3FF454AF2046CCE680
:10A510004F0611D556060FD553E8002F22F0400202
:10A5200043E800210029F7D12023C4F88830A1672F
:10A530002046F9F74DF83DE70D0206D5500004D549
:10A540002046BDE8F04100F0C9BDCB017FF532AF38
:10A55000002ABFF62FAF2046BDE8F04100F0BDBD98
:10A56000010000102001000461A20008FEFFFFEFBF
:10A57000D0F88C20B0F86010222A08B5036855D1B5
:10A580005B6A826D0B401370836D01338365B0F895
:10A590005E30013B9BB2A0F85E30B0F85E309BB2FB
:10A5A000002B42D1026852E8003F23F4907342E846
:10A5B000003103680029F5D103F1080252E8002FA9
:10A5C00022F0010203F1080C4CE800210029F3D12C
:10A5D0002022C0F88C20184A41679342016705D1B8
:10A5E000C26E012A0ED0F9F701F81EE05A68110276
:10A5F000F6D553E8002F22F0806243E800210029BD
:10A60000F7D1EDE70022C26653E8002F22F01002D6
:10A6100043E800210029F7D1DA69B0F85C10D206CE
:10A6200044BF10221A62FFF725FE08BD9A6942F066
:10A6300008029A61F9E700BF00800040D0F88C2042
:10A64000B0F86010222A08B5036852D15A6A114046
:10A65000826D22F8021B8265B0F85E20013A92B248
:10A66000A0F85E20B0F85E2092B2002A40D153E8F4
:10A67000002F22F4907243E800210029F7D103F162
:10A68000080252E8002F22F0010203F1080C4CE806
:10A6900000210029F3D12022C0F88C20174A4167FD
:10A6A0009342016705D1C26E012A0ED0F8F79EFFD2
:10A6B0001EE05A681102F6D553E8002F22F080629E
:10A6C00043E800210029F7D1EDE70022C26653E8F4
:10A6D000002F22F0100243E800210029F7D1DA69A7
:10A6E000B0F85C10D20644BF10221A62FFF7C2FD18
:10A6F00008BD9A6942F008029A61F9E700800040BB
:10A700002DE9F74F0368B0F86080DF691A689D682B
:10A71000D0F88C1001922229044640F0B480B0F8A1
:10A720006890DFF86CA1DFF86CB10026B9F1000F7A
:10A7300001D0BB0621D4B4F85E309BB2D3B1B4F8DB
:10A7400068209A4216D9226802F1080353E8003FB4
:10A7500023F08053083242E8003122680029F2D108
:10A760004D4B636752E8003F43F0200342E800315D
:10A770000029F7D103B0BDE8F08F2368A26D5B6AB2
:10A7800003EA08031370A36D0133A365B4F85E30C8
:10A79000013B9BB2A4F85E302368DF6978072CD0B8
:10A7A000F9070AD5019AD20507D501211962D4F813
:10A7B000901041F00101C4F89010B80709D5E907DD
:10A7C00007D502211962D4F8901041F00401C4F8B1
:10A7D00090107A0709D5E80707D504211962D4F843
:10A7E000903043F00203C4F89030D4F8903023B195
:10A7F0002046FFF710FDC4F89060B4F85E309BB2BD
:10A80000002B93D1216851E8003F23F4807341E885
:10A81000003023680028F5D103F1080252E8001F38
:10A8200001EA0A0142E800100028F5D120215B4529
:10A83000C4F88C10606720670AD05968090207D5F0
:10A8400053E8001F21F0806143E800100028F7D191
:10A85000E16E012913D1E66653E8001F21F01001D3
:10A8600043E800100028F7D1D969CA0644BF102177
:10A8700019622046B4F85C10FFF7FCFC56E720464E
:10A88000F8F7B4FE52E79A6942F008029A6171E75C
:10A89000FEFFFFEF0080004071A500082DE9F74F93
:10A8A0000368B0F86080DF691A689D68D0F88C1082
:10A8B00001922229044640F0B280B0F86890DFF897
:10A8C00068A1DFF868B10026B9F1000F01D0BB061E
:10A8D00021D4B4F85E309BB2D3B1B4F868209A4268
:10A8E00016D9226802F1080353E8003F23F0805391
:10A8F000083242E8003122680029F2D14C4B6367EC
:10A9000052E8003F43F0200342E800310029F7D12C
:10A9100003B0BDE8F08F2368A26D596A08EA01010F
:10A9200022F8021BA265B4F85E20013A92B2A4F8A4
:10A930005E20DF6978072CD0F9070AD5019AD20585
:10A9400007D501211962D4F8901041F00101C4F833
:10A950009010B80709D5E90707D502211962D4F884
:10A96000901041F00401C4F890107A0709D5E80767
:10A9700007D504211962D4F8903043F00203C4F8DB
:10A980009030D4F8903023B12046FFF744FCC4F84F
:10A990009060B4F85E309BB2002B95D1216851E8ED
:10A9A000003F23F4807341E8003023680028F5D18C
:10A9B00003F1080252E8001F01EA0A0142E8001010
:10A9C0000028F5D120215B45C4F88C106067206712
:10A9D0000AD05968090207D553E8001F21F08061A9
:10A9E00043E800100028F7D1E16E012913D1E66693
:10A9F00053E8001F21F0100143E800100028F7D1B0
:10AA0000D969CA0644BF102119622046B4F85C1007
:10AA1000FFF730FC58E72046F8F7E8FD54E79A695D
:10AA200042F008029A6173E7FEFFFFEF00800040EA
:10AA30003DA6000838B5044603682169A2681D6870
:10AA4000C0690A4361690A437D49024329400A43B8
:10AA50001A605A68E16822F440520A435A60794AFF
:10AA6000A16993421CBF226A11439A6822F06E4288
:10AA700022F430620A439A60DA6A616A22F00F02B5
:10AA80000A43DA62704A93421CD14FF0B043D3F8C4
:10AA9000883003F0030343F44033A3F54033013B14
:10AAA000022B00F2C780694A9B5CB0F5004F40F072
:10AAB0008980082B24D8DFE803F061C0832380233A
:10AAC00023236500624A934209D14FF0B043614AA3
:10AAD000D3F8883003F00C0343F44023E4E7594AE9
:10AAE00093420DD14FF0B043D3F8883003F4406364
:10AAF000B3F5006F1AD005D853B1B3F5806F12D0FB
:10AB0000012009E0B3F5406FFAD14FF400400EE0A8
:10AB1000FEF7D2FC58B900204FF00113A3660023C2
:10AB2000C4E91D3338BDFEF7CFF8F3E74A4865683E
:10AB30004A4B626A05EB450133F81220B0FBF2F391
:10AB40009942DDD8B3EB053FDAD800231946F7F771
:10AB50005FFA090241EA10616B080002C0182A4638
:10AB60004FF0000341F10001F7F752FA3C4BA0F51A
:10AB700040729A42C4D82368D860CCE7FEF79CFCA8
:10AB80000028C8D06168354B626A33F81220B0FBE8
:10AB9000F2F24B0803EB42034FF6EF72B3FBF1F313
:10ABA000A3F110019142ABD823F00F02216892B2B9
:10ABB000C3F342031343CB60ADE7FEF785F8DFE74D
:10ABC0002548DFE7082B9BD801A252F823F000BFED
:10ABD00019AC000825AC000831AC000801AB000836
:10ABE0002BAC000801AB000801AB000801AB00086A
:10ABF000F5AB00084FF400406368616A174A32F809
:10AC00001120B0FBF2F000EB5300B0FBF3F04FF675
:10AC1000EF73A0F11002ACE7FEF74EFC00283FF402
:10AC20007AAFE9E7FEF758FCF8E7FEF74DF8F5E7ED
:10AC30000948E1E7B0F5004FF4D1FEF74DFC9FE77E
:10AC4000F369FFCF0080004000380140DC7001084C
:10AC500000440040DF70F5070024F400EC700108A8
:10AC6000FFFC0F00836ADA0710B506D50168C46AD5
:10AC70004A6822F4003222434A609C0706D50168E4
:10AC8000046B4A6822F4803222434A60590706D591
:10AC90000168446B4A6822F4802222434A601A0702
:10ACA00006D50168846B4A6822F4004222434A6058
:10ACB000DC0606D50168C46B8A6822F48052224300
:10ACC0008A60990606D50168046C8A6822F40052ED
:10ACD00022438A605A060FD50168446C4A6822F400
:10ACE00080122243B4F5801F4A6005D14A68846C03
:10ACF00022F4C00222434A601B0606D50268C16CDA
:10AD0000536823F400230B43536010BD2DE9F04139
:10AD1000DDF8188004460E4615461F462268D369A2
:10AD200036EA03030CBF01230023AB4201D000200D
:10AD300027E0B8F1FF3FF2D0F8F748F9C01B4045D3
:10AD4000206802D8B8F1000F1DD150E8003F23F46D
:10AD5000D07340E80032002AF7D100F1080353E82D
:10AD6000003F23F0010300F1080141E80032002A0E
:10AD7000F3D12023C4F88830C4F88C3084F88420C0
:10AD80000320BDE8F08103685A07C7D5C3691B05D6
:10AD9000C4D54FF40063036250E8003F23F4D0733E
:10ADA00040E80032002AF7D100F1080353E8003FE1
:10ADB00023F0010300F1080141E80032002AF3D139
:10ADC0002023C4F88830C4F88C30C4F89030D5E71C
:10ADD0002DE9F7439846D0F88830202B04460E46DC
:10ADE000174643D1002943D0002A41D02123002512
:10ADF000C0F89050C0F88830F8F7E8F8A368A4F8D5
:10AE00005470B3F5805F8146A4F8567003D123696E
:10AE10000BB935461E46B4F85620CDF8008092B2E4
:10AE20004B4642B940212046FFF770FF48B9202326
:10AE3000C4F8883006E0002280212046FFF766FF34
:10AE400018B1032003B0BDE8F08322685EB935F87D
:10AE5000023BC3F308039362B4F85620013A92B25E
:10AE6000A4F85620D7E716F8013BF4E70220E9E7FB
:10AE70000120E7E773B504460026C0F89060F8F7B4
:10AE8000A5F823681B681A07054619D423681B68B0
:10AE90005B070AD56FF07E43009300222B464FF4E8
:10AEA00080012046FFF732FFB0B900202023C4F80C
:10AEB000883084F88400C4F88C30E06620670CE0A9
:10AEC0006FF07E430093324603464FF40011204654
:10AED000FFF71CFF0028D9D0032002B070BD10B5C9
:10AEE000044650B3D0F888301BB980F88430F8F7A6
:10AEF0007BFA22682423C4F88830136823F0010306
:10AF000013602046FFF796FD012816D0A36A13B1FF
:10AF10002046FFF7A7FE23685A6822F490425A6041
:10AF20009A6822F02A029A601A6842F001022046CA
:10AF30001A60BDE81040FFF79DBF012010BD000062
:10AF400030B581658168A0F85C200023B1F5805F91
:10AF5000A0F85E20436735D10369002B40F2FF1350
:10AF600018BFFF23A0F860300023C0F890302223E0
:10AF7000C0F88C30016801F1080353E8003F43F04A
:10AF80000103083141E800340368002CF2D1456E1A
:10AF900084680169B5F1005F34D1B0F8685095421A
:10AFA00030D8B4F5805F1DD1254A264C002918BF42
:10AFB00022464267C1B153E8002F42F4807243E851
:10AFC0000021F7E729B90369002B14BF7F23FF2372
:10AFD000C8E7B1F1805FC5D10369002B0CBF7F23A7
:10AFE0003F23BFE7174AE4E703F1080252E8002FC6
:10AFF00042F0805203F1080040E800210029F3D11B
:10B00000002030BDB4F5805F0FD10F4A0F4C0029EE
:10B0100018BF2246426751B153E8002F42F49072A4
:10B0200043E800210029F7D1EAE7084AF2E753E8AC
:10B03000002F42F0200243E800210029F7D1DFE78A
:10B040009DA8000801A700083DA6000871A50008FA
:10B05000D0F88C30202B30B415D1B9B1B2B1002367
:10B060000468C3660A4B9C420AD063681B0207D57A
:10B0700054E8003F43F0806344E80035002DF7D1E9
:10B0800030BCFFF75DBF022030BC70470120FBE7FA
:10B0900000800040436E30B52BB90123A0F86A3020
:10B0A000A0F8683030BD0368094D9A689968094C6A
:10B0B000490FC2F342626B5C615CDB00B3FBF1F3EE
:10B0C000A0F86A30AB5CA25CDB00B3FBF2F3E7E70D
:10B0D0000C710108047101087047704770471FB573
:10B0E00004AB03E9060090F88430012B04463AD003
:10B0F000012380F884302423C0F8883003681A685C
:10B1000022F001021A609A6822F440120A439A60FF
:10B1100071B95A68BDF80C009DF80E1022F01002AB
:10B1200002435A605A6822F07F4242EA01625A6042
:10B130001A6842F001021A60F7F748FF6FF07E428A
:10B14000034600924FF4800100222046FFF7DEFD07
:10B1500038B92023C4F88830002384F8843004B040
:10B1600010BD0320F8E70220F9E790F88430012BA6
:10B170000FD0012380F88430016851E8002F42F09D
:10B18000020241E80023002BF6D180F884301846F3
:10B1900070470220704710B590F88430012B0446A8
:10B1A00017D02423C0F8883003681A68196821F082
:10B1B0000101196042F000524FF0005141661A60DF
:10B1C000FFF768FF2023C0F88830002084F884004F
:10B1D00010BD0220FCE770B590F88430012B0446C6
:10B1E00017D005682423C0F888302E682B6823F018
:10B1F00001032B60AB6823F060431943A960FFF79C
:10B2000049FF20232E60C0F88830002084F8840095
:10B2100070BD0220FCE770B590F88430012B044625
:10B2200017D005682423C0F888302E682B6823F0D7
:10B2300001032B60AB6823F060631943A960FFF73B
:10B2400029FF20232E60C0F88830002084F8840075
:10B2500070BD0220FCE7000038B5084D052455F804
:10B26000043B2BB9013C14F0FF04F8D1204638BD53
:10B27000DB6898470028F5D0F9E700BF6C12002082
:10B28000034BD870034B1B681B6C03B11847704706
:10B290008012002068120020034B1874034B1B68B7
:10B2A0005B6C03B1184770478012002068120020C1
:10B2B000F0B5314D314B95F90420314E91B00C462B
:10B2C000012795F905108DF8047002288DF80920E2
:10B2D0008DF80A1010D18DF80800D8711C7202F098
:10B2E0009FFD337803B114B101A803F003FA254B95
:10B2F000059A1A6011B0F0BD59714FF480711A713E
:10B30000D9801C7233788DF8087053BB1F2306A8B0
:10B310008DF81C208DF8183002F064FF20238DF882
:10B32000183006A82B798DF81C3002F05BFF222321
:10B330008DF8183006A86B798DF81C3002F052FF9A
:10B3400021238DF8183006A86B798DF81C3002F097
:10B3500049FF29238DF8183006A80B4B079302F0FC
:10B3600041FF02F05DFD012306A88DF818308DF82D
:10B370001C3002F037FFB4E78012002030080020B4
:10B380005C12002060120020000400017FB5092338
:10B3900001A88DF8043003F0ADF90038044B059A8C
:10B3A0001A6018BF0120404207B05DF804FB00BFDF
:10B3B0006012002070B504460B46134962784A704B
:10B3C0000020A2780A7208701A884A729A788A72E3
:10B3D000DB780B746368CB600C4B1B68DA6A2AB1AC
:10B3E000237803F0FB030A2B00D09047084E052575
:10B3F00056F8043B1BB15B6A0BB120469847013DF0
:10B4000015F0FF05F4D170BD3C0800206812002043
:10B410006C12002070B50446104801230370637855
:10B420004370A3788372E368C360E378037623698B
:10B430004376237943720A4B1B689B6A03B1984792
:10B44000084E052556F8043B1BB19B690BB12046FD
:10B450009847013D15F0FF05F4D170BD500800205C
:10B46000681200206C120020014B1868704700BF62
:10B470006012002000B58BB0012368468DF80030C3
:10B4800002F088FD38B99DF80400003818BF01208B
:10B490000BB05DF804FB0020FAE7000008B501F0EE
:10B4A00073FE48B9FFF7E6FF012806D0054BD879AF
:10B4B000197AFFF7FDFE012008BDBDE80840FFF73F
:10B4C000CBBE00BF300800202DE9F04186B0054614
:10B4D0000E46174601F058FE00287FD101F06CFEA1
:10B4E000044640B9FFF7C6FF012807D03D4B197A43
:10B4F000D879FFF7DDFE6FF0020462E0DFF8E88044
:10B5000088F80860003E18BF01268DF80460374EA9
:10B51000687833798DF81230694602F0D9FC00283A
:10B520003ED08DF804400394ADF810406FF006044F
:10B5300095E803002E4B83E80300337988F80A303E
:10B54000394601A803F0DAF92A4B059A1A60112846
:10B5500041D801A353F820F0B7B50008DDB50008C5
:10B56000D7B50008D7B50008D7B50008D7B500088B
:10B57000D7B50008F7B40008D7B50008D7B500085C
:10B58000D7B50008D1B50008D7B50008D7B5000871
:10B59000DDB50008DDB50008DDB50008CBB5000855
:10B5A0002B788DF808306B78ADF810306B6803930A
:10B5B0004FF0FF34BCE7104B00221A70E31D18BF98
:10B5C0001446204606B0BDE8F0816FF00404F8E7A9
:10B5D0006FF00504F5E74FF0FF34F2E76FF0010478
:10B5E000EFE700BF30080020500800208012002044
:10B5F00060080020601200206412002037B501F0BE
:10B60000E5FD144D052455F8043B5BB11B694BB1B6
:10B6100055F8043C9B682BB1984718B155F8043C89
:10B620001B699847013C14F0FF04ECD1FFF714FEAE
:10B6300068B9094D2B7853B1084BADF80040D97863
:10B64000019422466846FFF73FFF00B92C7003B013
:10B6500030BD00BF6C120020641200208012002058
:10B6600030B58BB0054601F08FFD0446002839D176
:10B67000FFF700FF012838D168468DF8004002F03E
:10B6800089FC10B14FF0FF3004E09DF80430AB426C
:10B6900002D100200BB030BD012DF3D0022D11D00E
:10B6A000002DF7D1002BF4D068468DF8045002F03D
:10B6B00099FD0028E6D10E4B1B681B6B002BE8D0D0
:10B6C0009847E6E7002BDDD168468DF8045002F07C
:10B6D00089FD0028D6D1064B1B681B6B002BD8D0E8
:10B6E0002846EDE76FF00100D4E76FF00200D1E7E4
:10B6F0006812002010B504468AB018B94FF0FF3028
:10B700000AB010BD002368468DF8003002F042FCFC
:10B710000028F3D19DF804302370F1E77FB50022B3
:10B720000B4620498DF8072001220A7042784A70A2
:10B730000446002A33D102790A721A884A729A782A
:10B740008A72DB780B740369CB60C378164D8DF871
:10B750000830037B8DF80930836803932B68DB6A1C
:10B760000BB102A898472B689B6B13B1227E02B1E4
:10B7700098470E4E052556F8043B1BB1DB690BB10B
:10B7800020469847013D15F0FF05F4D10DF1070063
:10B79000FFF7B0FF637913B1054B01221A7004B0B3
:10B7A00070BD00BF3C080020681200206C12002011
:10B7B0006412002010B504468AB018B94FF0FF306B
:10B7C0000AB010BD202368468DF8003002F0E2FB7D
:10B7D0000028F3D1024A9DF9043023701371EFE77A
:10B7E0008012002000B58BB02323019068468DF8AD
:10B7F000003002F0F7FC003818BF012040420BB0C7
:10B800005DF804FB70B5654C01468EB018222046E9
:10B8100006F0FEF8624B00221A70F8F7C9FE237892
:10B820004068012202FA03F1014004D15D4B084651
:10B8300008F0E4F8FEE75C495C481A4602F032F989
:10B8400018B14FF0FF300EB070BD272304A88DF85B
:10B85000103002F0C7FC564E564D002870D101231F
:10B8600033702B68DB690BB100209847272304A8AD
:10B870008DF8103002F08EFB059B93F84820227063
:10B8800093F8182193F81A316270A370464BD3E9EC
:10B89000020105F0AFFF05460028D2D1464E06232F
:10B8A00004A88DF8103002F075FB059B736104A8A5
:10B8B00002F098FC022304A88DF81030059602F0DF
:10B8C00069FB0836032304A88DF81030059602F0B2
:10B8D00061FB0F2606F052F8012304A88DF81430FE
:10B8E0008DF8106002F07EFC10230DEB03008DF844
:10B8F00010308DF8145002F075FC04238DF81030D0
:10B9000004A8A3788DF8143002F06CFC3A238DF86B
:10B91000103004A86369059302F064FC02A9207842
:10B920008DF8086004F0E8F8003818BF0120E071D5
:10B930001420FFF757FFE07903F0A4F9284682E7C7
:10B9400028238DF810302B681B6943B104A802F03E
:10B9500021FB2B6805981B6940F2C45198472723A7
:10B9600004A88DF8103002F03DFC50B9012304A862
:10B970008DF8103002F00EFB9DF81430002B7FF490
:10B980006EAF3378002B7FF46CAF052204A88DF8DE
:10B990001020059302F026FC78E700BF80120020FB
:10B9A0006412002014710108A8120020C0120020A7
:10B9B0005C120020681200204412002037B50023DA
:10B9C0000D4601930446D0B900F0A8FB0190019BFD
:10B9D000D3B10F4A42F824300E4A9A620E4A1268D6
:10B9E000916B1963916C596392690C49D9625A61E0
:10B9F00028465B680A49F2229847002006E001A920
:10BA000000F092FB0028E2D04FF0FF3003B030BDD1
:10BA10006C120020B1B20008681200208DB300083B
:10BA200050110020194B07B51860194B194A1A60BC
:10BA3000194A5A60194A9A60194ADA60194B026821
:10BA40001A6042685A6082689A60C268DA60164A70
:10BA50001A6182695A61154BC26B5A60144A01918E
:10BA600019609A601946134ADA600020FFF7A6FFB2
:10BA700048B901A800F056FB003818BF0120404229
:10BA800003B05DF804FB4FF0FF30F9E768120020C7
:10BA9000C012002015B400081DB7000835BB00080F
:10BAA000B5B30008A8120020A9FA000898120020D7
:10BAB00081B2000899B2000851B118B1012804D030
:10BAC00000207047044B0B607047044B0B60F7E796
:10BAD0004FF0FF30704700BF000400010100010279
:10BAE00008B503F0EBF8002814BF6FF00100002048
:10BAF00008BD08B502F0BCF9002814BF6FF00100C2
:10BB0000002008BD10B504468AB018B94FF0FF30C8
:10BB10000AB010BD212368468DF8003002F03AFAD1
:10BB20000028F3D1024A9DF9043023705371EFE7E6
:10BB3000801200202DE9F0412E4D2F4F00232B7055
:10BB400043786B703B689B6A8AB004460BB1284609
:10BB50009847DFF8A880052658F8043B1BB11B6AFC
:10BB60000BB120469847013E16F0FF06F4D123782A
:10BB7000052B2FD00B2B35D0012B25D1204C0623A4
:10BB800068468DF8003002F005FA0199E07905F079
:10BB900077FE10B91B4B019A5A611B48FFF70AFE4A
:10BBA0001A48FFF7AFFF6B788BB9A371184B587821
:10BBB000FFF756FD3B685B6A0BB1114898476B78FD
:10BBC00013B9E07905F0ECFE0AB0BDE8F081FF237F
:10BBD000A371EFE70F4B01225A74227A9A74627AAA
:10BBE000DA74F1E76378002BEED00AB0BDE8F041DB
:10BBF000FFF7CCBB50080020681200206C12002018
:10BC000030080020441200203408002035080020AD
:10BC1000801200203C08002030B58BB0FFF769FF90
:10BC20000446F0B903F048FF831C1DD0F8B9134D4A
:10BC30002B685B69DBB1272368468DF8003002F082
:10BC4000A9F92B6801985B694FF4B961984703F033
:10BC500045FF78B92CB9094B1B68DB690BB1012092
:10BC6000984720460BB030BD6FF00704EFE74FF068
:10BC7000FF34ECE74FF0FF34F3E700BF6812002019
:10BC8000014B1878704700BFD4120020014B587840
:10BC9000704700BFD412002070470000044B9A7A0E
:10BCA0000AB101225A70034B5B6903B11847704710
:10BCB000D41200206C08002073B5224C6378002B4E
:10BCC00033D008F085F966680546FFF7CDFB0644DA
:10BCD000AE4214D2A37A93B1E0228DF800208DF801
:10BCE0000130217AE368019301226846FFF7ECFBFB
:10BCF00008B1073010D100236370A372656094F817
:10BD00003430EBB1002384F834300F4B5B6BBBB1A4
:10BD100002B0BDE87040184740F2DC510B4808F013
:10BD200023FA0A4808F0E6F9E8E794F83520002AF3
:10BD3000E5D094F8360084F83530FFF791FCDEE763
:10BD400002B070BDD41200206C0800200C1300203B
:10BD500037B5104D104CC8B1C1B101236272002239
:10BD60002860E16023700D480D4B00924FF0FF31C9
:10BD700008F014F900250B4825822022294605F0F9
:10BD80005BFE6570A574A58603B030BD00232B60F3
:10BD90002370EFE7D0120020D41200200C130020F3
:10BDA0009DBC0008E81200202DE9F0478E4C237856
:10BDB0008CB0002B56D0C2780AB9837B13B1238A8A
:10BDC00001332382437B002B4CD0E02A4AD100234D
:10BDD000A372876897F80080B8F1220F27D8B8F1CE
:10BDE000220F30D8DFE818F04100FB0052005A0063
:10BDF00061006E0075008E009D00B400C7002F002A
:10BE00002F002F002F002F002F002F002F002F00BA
:10BE10002F002F002F002F002F002F002F002F00AA
:10BE20002F002F002F002F00C900D000D400B8F140
:10BE30007E0F00F0CC80B8F17F0F00F0DF80B8F10A
:10BE40007D0F00F0AB80A57A002D00F05B81674C80
:10BE5000637A3BB94FF47A71204608F085F92046A1
:10BE600008F048F90CB0BDE8F087E3680122002132
:10BE7000A2721970A37AE1689818A0720620C854BB
:10BE8000A37AE1689818A072CA54DCE7584B9B6A01
:10BE9000002BD8D0012102209847D4E77B7884F882
:10BEA0003630012384F83530CDE704238DF8043093
:10BEB0007B78003B18BF012301A88DF8083002F001
:10BEC00091F9C0E77878003818BF012002F0DAFE57
:10BED000B9E7484E0FCE01AD0FC50FCE0FC596E89E
:10BEE000070085E807007B780A2BACD8424A126825
:10BEF0005268002AA7D00CA901EB830353F82C0C3D
:10BF00009047A0E77878431E012B9CD83A4B013824
:10BF10001B6818BF012020729B68002B93D09847A4
:10BF200091E7E26801230821A3721170627A057B10
:10BF3000A17AAA4228BF2A46934284D285685A1C15
:10BF4000EB5CE56801334E1CA6726B54D3B2EDE78F
:10BF5000E3680122A27209221A70A37AE268218A98
:10BF6000581CA072D154A27A238AE1681B0A501C83
:10BF7000A0728B5467E7238265E705238DF80430B0
:10BF800001A802F0B7FB5EE7194BDB6A98475AE756
:10BF9000194B78781B686075DB68BEE7037B072B5D
:10BFA0007FF451AF06238DF80430B7F80130ADF8B7
:10BFB00008307B793A791B0443EA0223FA78134369
:10BFC000642253430393BB798DF81030D8E73B22AA
:10BFD00001A88DF804208DF8083002F003F9012340
:10BFE00084F834302FE700BFD41200200C13002057
:10BFF0006C080020E46E0108D01200202A2301A85A
:10C000008DF8043001F0C6FF94F80A90E6689DF8B8
:10C0100008009DF809509DF80A709DF80BC09DF826
:10C020000D309DF80E209DF80F109DF80CE009F1E1
:10C03000010A84F80AA006F80980354E94F80A909F
:10C040003668D4F80C8009F1010A84F80AA096F841
:10C0500003A008F809A094F80A90D4F80C8009F11C
:10C06000010A84F80AA096F802A008F809A094F83A
:10C070000A90D4F80C8009F1010A84F80AA096F815
:10C0800001A008F809A094F80A9009F1010A84F8BF
:10C090000AA096F80080E66806F8098094F80A80FD
:10C0A000E66808F1010984F80A9006F808C094F8D7
:10C0B0000AC0E6680CF1010884F80A8006F80C70E2
:10C0C000A77AE66807F1010C84F80AC0F555A57A4D
:10C0D000E6686F1CA7727055A07AE568461CA672C8
:10C0E0002954A17AE0684D1CA5724254A27AE168F5
:10C0F000501CA0728B54A37AE268591CA17202F8FA
:10C1000003E0A0E6034807F0A7FF6570AAE600BFBA
:10C11000D01200200C130020704700000048704728
:10C120006C080020002070474FF0FF30704700007F
:10C13000044B054A93F81831022B18BF062382F8E6
:10C1400090347047E8180020B01E0020034BD3F84D
:10C15000483313B15B6903B118477047B01E002024
:10C16000034A137843F004031370FFF7EFBF00BFD7
:10C17000AC1E00201FB50A4B8DF8090093F87C20F7
:10C180008DF80A2093F88C2093F848000D3202A90C
:10C190008DF8082003F0B0FCC0B205B05DF804FBD8
:10C1A000E818002010B5074C04F5806007F054FF34
:10C1B00094F81A3413B1012384F81934BDE81040FF
:10C1C000FFF7C4BFB01E002010B50C4CD4F84033AC
:10C1D00043F08003C4F8403394F81A3413B10020BC
:10C1E000FFF7E0FF94F8913423F0120343F01203B9
:10C1F00084F89134BDE81040FFF79ABFB01E0020CC
:10C200002DE9F041DFF8AC8098F81831022B064692
:10C210000D4602D0284BDB6A984702F0E9FD044640
:10C2200028B1022002F0DAFD002002F0DCFD98F8CF
:10C230001831012B17D102F0DDFD074630B1002087
:10C2400002F0CDFD002002F0CFFD3C4602F0D4FD0F
:10C2500048B1002002F0C4FD002002F0C6FDBDE898
:10C26000F041FFF765BF002CF9D1144C94F89024ED
:10C2700094F81A34BAB90BB184F84164304602F02C
:10C2800065FFD8F82C0007F0ADFED4F8B43398421F
:10C29000E5D30B4807F0E0FE94F8913443F0100327
:10C2A00084F89134DBE70BB184F84154284602F05E
:10C2B0004DFFF1E7E818002098780108B01E002033
:10C2C0004822002073B5164C164D04F57A76EB6CB7
:10C2D00095F8502095F9781095F84800009603F0ED
:10C2E00031FC95F8303184F8FC3395F8480040F281
:10C2F000012304F224423146A4F8FA3303F02EFC61
:10C3000058B194F8243484F86A34074B00205B6BEE
:10C31000984794F8FB3384F8903402B070BD00BFA6
:10C32000B01E0020E818002098780108074A10B5D0
:10C33000137843F002031370FFF708FFBDE81040C5
:10C34000034B01220021022007F058BBAC1E002045
:10C350005D710108074A10B5137843F008031370A4
:10C36000FFF7F4FEBDE81040034B0122002102203C
:10C3700007F044BBAC1E00206D7101082DE9F041AF
:10C380000F4616461D46804607F022FE0B4A0C4C0F
:10C390001378278123F0110343F011031370C4E9CC
:10C3A000000866812573FFF7D1FEBDE8F041054B1B
:10C3B00001220021022007F021BB00BFAC1E00209B
:10C3C0005C2400207D71010813B507F001FE0D4BC0
:10C3D0006C461860204607F04FFD94E803000A4AB7
:10C3E0000A4B83E80300137843F020031370FFF730
:10C3F000ADFE074B01220021022002B0BDE8104033
:10C4000007F0FCBA6C240020AC1E0020E8210020BC
:10C410008A710108F8B5334D95F81841012C06468C
:10C420004BD0022C51D064B938B9D5E91B0105F1C4
:10C43000740383E803002046F8BD01283DD002289C
:10C4400001D00324F7E7284F85F8180107F5747E1B
:10C45000BEE80F0007F57A7CACE80F009EE8030009
:10C4600095F8E9308CE8030087F8FB63E3B195F8B1
:10C470000031022B18D1D5F804316B67C7F8EC33C3
:10C4800095F87D3095F8082187F8F83395F88C30C9
:10C4900085F8782087F8F93397F81B2487F8E82384
:10C4A00040F20133A7F8FA33002387F81A340F4B10
:10C4B000DB6A9847FFF706FFBDE702F0A4FC0446DD
:10C4C0000028B8D185F81861B5E70028B9D1064B26
:10C4D00085F81801062283F89024044BDB6A9847FC
:10C4E0003446A8E7E8180020B01E0020987801081C
:10C4F0002DE9F04192B0064602F07AFC002840F0A7
:10C500005981AD4D95F81831012B09D02B6BAB4CEF
:10C5100093B194F80431BBB1042B6FD0032003E036
:10C5200002F068FC18B10F2012B0BDE8F08102F0F3
:10C5300063FC0028EAD0F6E7B5F82031D4F81C24D3
:10C54000013B53432B63E4E79D4803F00CFA0028BA
:10C5500040F02C8194F80C3123802B6B0C930DF15F
:10C56000180895F839308DF83830404695F81C3168
:10C570008DF83A3007F0A6FCD5F82831009302AFC9
:10C5800098E80600D5F82431384607F032FC97E8E1
:10C5900003000FAB83E80300EB6A0D9300238DF8D3
:10C5A00044302388ADF8463095F8303101228DF8BB
:10C5B00039201BB98DF844208DF83930814B009318
:10C5C000814B95F84800A3F179020CA903F009FB0F
:10C5D000C0B10B28A8D1D4F8941499B1002EA3D0DF
:10C5E000D4F84033794843F02003C4F8403307F0CF
:10C5F000BBFD764807F07EFD002095E7704803F00C
:10C60000E6F9A4E795F8487095F9693095F939206D
:10C6100095F87D106E4E384603F0F0FA009641B260
:10C62000EB6C95F850203846183603F08BFA0096DC
:10C63000EB6C95F8502095F9701095F8480003F0D0
:10C6400081FAD4F8C413AB6DD4F8DC230B44C4F8DE
:10C65000B033EB6D1344C4F8B43394F80431042BB5
:10C6600007D02B6E0B44C4F8B0336B6E1344C4F880
:10C67000B4330023089395F8303183B108A802F051
:10C6800095FC00284ED195F9390094F837629DF851
:10C690002070FFF76FFD3E4480B2B04240D30023CC
:10C6A0008DF8133095F839308DF8213095F8383001
:10C6B0008DF82230D5F880300993D5F884300A936C
:10C6C0002388ADF82C3095F8303194F81B648DF840
:10C6D0002E3095F848003F4B8DF820600DF1130285
:10C6E00008A903F043FA012384F8413495F839305E
:10C6F00084F842349DF8133084F84334D4F81C3461
:10C70000C4F85064C4F84834C4F8583402F076FBD6
:10C7100050B1D4F81C0402F083FB28B1102003E7C9
:10C72000082001E71320FFE695F81831012B01D10D
:10C7300002F078FB02F065FB0023059394F80431C6
:10C7400095F9395094F81B649BB1042B7FF4E6AE45
:10C7500005A802F067FE58BB94F8183413B1059B86
:10C76000013B0593164B05983246E9B202F0C0FE34
:10C7700002E0134802F090FEC0B9D4F8403394F8B8
:10C780000C11218043F00203C4F8403394F81834AC
:10C7900011480133DBB284F8183484F845340F4B68
:10C7A00000259B6AC4F89854984725E71120BBE6FA
:10C7B0001220B9E60E20B7E6E8180020B01E0020CF
:10C7C000B81F002018190020442300201822002040
:10C7D00068220020CC220020B21E00209878010898
:10C7E000F0B5504C504EB4F8DC202287D4E92D012E
:10C7F00094F8B12084F8692004F16C0282E8030007
:10C80000D4E92F0104F1740282E80300B4F8C420D3
:10C81000A4F87C2091B0D4F8CC20D4F8C810C4F887
:10C8200084200025D4F8D020C4F888200123A4F85F
:10C830002031C4F8801084F83051A56284F81B516F
:10C8400084F83A5084F81D5184F81E51C4F83451CC
:10C85000C6F89854A6F8185486F81A54A4F8385113
:10C860008DF8183004F50973039304F50A7394F8EE
:10C870004800A4F84651049303A92C4B84F8455171
:10C88000C4E94F55059303F045F9E36EC6F8D43378
:10C8900094F87D3086F8E03394F88C3086F8E133F4
:10C8A0004FF48073A6F8E23386F8D05394F8303111
:10C8B00086F8E43306F574770FCF06F57A740FC463
:10C8C00097E8030040F2012384E80300A6F8FA3356
:10C8D000D6F8483386F81B54CDE901551BB15A6888
:10C8E0005B6901920293124B0793A3F148020892ED
:10C8F000A3F1140209920F4A0B9229330A93A2F171
:10C900009C030C93A2F198030D93131D0E9301A9A0
:10C9100002F14C0307A802F599620F9302F05DFA49
:10C9200011B0F0BDE8180020B01E0020CC2300207C
:10C9300018230020CC190020F8B50D4F0D4C0E4ED9
:10C940000D4607F089FB3B6B984796F8480004F2C8
:10C950002442294603F002F948B194F8243484F8BB
:10C960006A34706D7B6B9847EB7C84F89034F8BD2B
:10C9700098780108B01E0020E81800200F4890F8B1
:10C980001B3480F8B8330E4B93F8692080F8BB2332
:10C9900093F87D2080F8C82393F88C2080F8C92371
:10C9A00093F8303180F8CC330022A0F8CA2300F588
:10C9B0006E7100F56070FFF7BFBF00BFB01E0020B2
:10C9C000E8180020114890F89034EBB190F81B342F
:10C9D00080F8D0330E4BDA6EC0F8D42393F87D2064
:10C9E00080F8E02393F88C2080F8E12393F830312D
:10C9F00080F8E4334FF48072A0F8E22300F57471FC
:10CA000000F56670FFF798BF704700BFB01E0020AA
:10CA1000E818002070B5344C2421204605F00EF8AB
:10CA2000636A984218BF60624FF01C012F4814BF20
:10CA30000125002505F002F8636C984218BF606478
:10CA40004FF480712A4818BF45F0020504F0F6FF44
:10CA5000D4F84831984218BFC4F848014FF0D401C7
:10CA6000244818BF45F0040504F0E8FFD4F820324C
:10CA7000984218BFC4F820024FF000011E4818BFAA
:10CA800045F0080504F0DAFFD4F82432984218BFC4
:10CA9000C4F824024FF46071184818BF45F010051F
:10CAA00004F0CCFFD4F8A835984218BFC4F8A80504
:10CAB0004FF01401124818BF45F0200504F0BEFFE6
:10CAC000D4F8C03598420F4B18BFC4F8C005D3F84E
:10CAD000483318BF45F040052BB11B691BB12846F0
:10CAE000BDE87040184770BDE818002010190020FC
:10CAF00030190020341A00200C1B0020101B0020CD
:10CB0000941E0020B01E00202DE9F04F91B04FF090
:10CB10000008012B05460F4602928DF81580ADF8EE
:10CB2000188003D8C84EC146B94502D311B0BDE83C
:10CB3000F08F15F8090002F077FA4844B842F5DCA6
:10CB400015F8093009F10104023BE4B2112BEDD8CC
:10CB500001A252F823F000BFA1CB0008D3CB0008FC
:10CB6000D3CC0008FDCC000885CD0008ADCD000871
:10CB70001FCE000851CE0008CDCE00082DCB0008F6
:10CB80002DCB00082BCF00082DCB00082DCB0008A3
:10CB9000E9CF000811D0000855D0000893D0000854
:10CBA000052002F0EDFA90B10521002002F0ACFA68
:10CBB0002A5DA64B09F1030409F102095FFA89F91C
:10CBC00083F85C2415F8092083F85D24E4B2A146BB
:10CBD000AAE700238DF816308DF817308DF81C3039
:10CBE0008DF82030B8F1000F6CD14FF0050896F8A1
:10CBF0007C208DF83920631E96F839208DF83B2073
:10CC00002B4496F838200D938DF83C2096F81A3175
:10CC100096F868208DF83D20D6F82C218DF83A3012
:10CC20000C9273B37B1C1B1BDBB28DF8383008AB46
:10CC3000019307AB009396F848000DF117030DF12F
:10CC400016020CA902F09EFF8DF8150000F00700F7
:10CC5000072813D196F939209DF9163086F8393016
:10CC60009A429DF8173086F83830B8BF01229DF8F7
:10CC70001C30B8BF86F81D2186F868304FF00009D7
:10CC800009E00523D1E701220DF11501032002F08F
:10CC9000DBF809F101095FFA89F29DF82030B3FB56
:10CCA000F8F19142EFD82344DCB2631EDBB29F421D
:10CCB0000DD9EA5C032A9AD0A74288BF1C464FF0E0
:10CCC000010884E709F105095FFA89F4F7E71C46D2
:10CCD000F5E72B5D012203F00F0309F1020986F845
:10CCE0001B3102FA03F35FFA89F9A6F8203100221A
:10CCF00006A9042002F0A8F84C4668E707238DF83F
:10CD000015302B5D96F84800C3F3021203F00F03B1
:10CD10008DF8303009F10303DBB28DF83120EA5C85
:10CD200009F10403DBB209F10504EB5C09F1020926
:10CD30005FFA89F91B0443EA022315F8092013431B
:10CD4000642253430CA90D9302F02BFF00F007035C
:10CD5000072BE4B28DF815000CD19DF8303086F821
:10CD6000703086F878300D9BF36673679DF831302C
:10CD700086F869308DF81800012206A9052002F016
:10CD800063F824E7314BD3F848336BB11B685BB1D0
:10CD90009847029B8DF8180003F03F038DF8193077
:10CDA000022206A90620EAE7FF20F2E703238DF816
:10CDB00015302B5D8DF824300CAB089309F103037B
:10CDC000DBB209F10604EA5C96F8480009F10403B5
:10CDD000DBB208A9EB5C1B0443EA022309F102025F
:10CDE000D2B209F10509AA5C1343642253435FFAE6
:10CDF00089F90C9300230D9315F809308DF838301C
:10CE000002F0D5FEC3B20028E4B28DF81530FFF66B
:10CE1000DEAE8DF81830012206A90720AFE72B5DA2
:10CE200003F00F03012B4FF47A7238BF01235343F1
:10CE300009F10209B36513445FFA89F9F365002229
:10CE400006A9082056E700BFE8180020B01E002001
:10CE50002B5D96F84800C3F340128DF81D2007A9FA
:10CE6000C3F3001203F00F038DF81C208DF81E3061
:10CE700002F0A3FE09F1020901305FFA89F93FF4DB
:10CE80003BAFBDF81C30914AA6F87C309DF81E30AF
:10CE90009DF81C40D05CF5F73DF80223C6F88000F1
:10CEA0000CA996F848008DF830308DF8324002F029
:10CEB00023FE96F93930089040B29842B8BF184620
:10CEC00086F83900002206A9092013E703238DF80C
:10CED00015302B5D8DF8303009F10303DBB209F119
:10CEE0000504EA5C96F8480009F10403DBB209F195
:10CEF0000209EB5C5FFA89F91B0443EA022315F887
:10CF000009201343642253430CA90D9302F05BFEE6
:10CF1000C3B20028E4B28DF81530FFF658AE8DF894
:10CF20001830012206A90A2029E7092002F028F971
:10CF3000DFF89CA1002854D00921002002F0E4F879
:10CF40000023ADF8263009F10203DBB24FF47A7109
:10CF5000EA5C09F10303DBB20DF1300BEB5C1B045F
:10CF600043EA02232A5D134309F10402D2B209F114
:10CF7000060409F10509AA5C5FFA89F943EA02632C
:10CF800015F8092003934A4312125846ADF824209D
:10CF900006F072FF039B03F1965303F5A91303F503
:10CFA000EC530893DAF83C3300930DF1200999E82B
:10CFB0000600DAF838330AA806F01BFF0B9B009333
:10CFC0009BE806000A9B484606F0F8FE99E8030035
:10CFD00006F02AFF01F021FF0123E4B28AF8383479
:10CFE000F5E58AF83804F2E50C2002F0C9F80028CB
:10CFF0003FF4EDAD0C21002002F086F8344B93F89D
:10D000009034043B012B7FF6E2AD01F002FFDEE538
:10D0100009F10203DBB22A5DE95C09F10303DBB22B
:10D0200009F10504EB5C09F104095FFA89F91B04B5
:10D0300015F8090043EA012313436421594300F022
:10D040000F0001F0E7FEE4B28DF81800012206A9F6
:10D05000112094E60D2002F093F800283FF4B7ADBC
:10D060000D21002002F050F809F10203DBB2194A49
:10D07000E85C2B5D126809F1040409F103095FFA09
:10D0800089F943EA002015F80910E4B201F0C4FE62
:10D090009DE52A5D09F1020309F1040409F1030980
:10D0A000DBB25FFA89F9E95C15F809301B0443EA41
:10D0B000012313436420584301F0B0FEE4B28DF81D
:10D0C0001800012206A9132059E600BF9771010834
:10D0D000B01E00205C2400200E4B93F89124920790
:10D0E00003D593F88F24012A08D90B4991F81A2106
:10D0F00022B18A6A501C18BF01328A620022A3F84A
:10D10000182483F81A24D3F8402322F00202C3F82B
:10D1100040237047B01E0020E818002070B5184C5E
:10D12000184D04F55A7006F097FFD4F84033D4F840
:10D130009804D5F8906023F02003C4F8403338B148
:10D1400006F050FF864203D2002385F83A3070BDC6
:10D150000120FFF7CDF90028F9D00B28F7D095F87A
:10D16000393084F84234092094F8183484F845346E
:10D1700084F8410401F0EAFFBDE87040FFF7ACBF5E
:10D18000B01E0020E8180020094BD3F84023012AE4
:10D190000AD008490978C90708D43AB993F8920423
:10D1A000013818BF012070470020704701207047E8
:10D1B000B01E0020AC1E0020034BD3F84003431EDA
:10D1C00058425841704700BFB01E00202DE9F04F73
:10D1D000A9B0EFF3108272B6DFF8F4820021D8F81C
:10D1E0000030C8F8001082F31088BA4C002B00F011
:10D1F000E480DAB29B06039264D5B74D95F81831F6
:10D20000022B02D0B54BDB6A9847EFF3108972B658
:10D21000B34F06F0DDFE3E68D4F8B013361A314441
:10D22000B04806F0A1FFAF4806F064FFD4F8B4138D
:10D23000AD48314406F098FFAB4806F05BFF89F338
:10D24000108894F81A34002B00F06D81152312A970
:10D2500095F848008DF8483002F04EFCD4F8B4132D
:10D260000F900144A14806F07FFFA04806F042FF5E
:10D270003B6894F81B24EB620DAF38468DF87020A4
:10D280001D9306F01FFED5F82831009306AE97E8EF
:10D290000600D5F82431304606F0ABFD96E80300D1
:10D2A0001FAB83E80300D4F81C341E9395F830318B
:10D2B00095F84800003B18BF01231CA98DF8713078
:10D2C00002F023FC039BDF064BD5834DDFF820A241
:10D2D000D5F8E420BAF90A30059298F800200493B2
:10D2E000002363F300020A9388F8002084F8443492
:10D2F000049AA4F8223484F82534C4F82834A4F815
:10D300002C3484F82E34C4F8303484F82034C4F833
:10D31000343484F83834C4F83C34704B9AF90C90A7
:10D32000A4F88C2494F89024DB6A84F88E9484F812
:10D330008F24DAF80470BAF80860984794F88F34AC
:10D3400013B9694806F088FE3146384601F04EFDB3
:10D350008346002800F0EA80049BA4F87E3484F819
:10D360008094039B19071AD55B4B93F81831022B55
:10D3700002D05A4BDB6A98470220FEF7D9FE84F8A8
:10D38000410401F0E3FE94F81A3413B1012384F848
:10D39000193494F8913443F0100384F89134039BCA
:10D3A0005A0703D506210520FEF72AFF039B9B079A
:10D3B00003D504210320FEF723FF01F035FD94F887
:10D3C0009124D7065FD5002384F89234D4F84033F3
:10D3D0001E0644BF23F08203C4F8403312F0050F49
:10D3E00000F0FC820B2001F0CBFE002800F0F6825A
:10D3F00094F89134DD0700F1F182580740F1088379
:10D40000D4F8403323F00203C4F84033D4F8402367
:10D4100082BB94F8915415F001011EBF2B4662F3B4
:10D42000000384F8913494F891345E0744BF6FF39D
:10D43000820384F89134012384F8923421B1D4F822
:10D4400044332C481B6898476D070BD52A4801F0D8
:10D45000A3FE01F0D1FE28B194F8913443F0040307
:10D4600084F8913401F0CEFC94F891346FF30413F6
:10D4700084F89134012384F8923494F8913443F081
:10D48000200384F8913494F8913418070AD56FF387
:10D49000C3031A4984F89134D4F84433A1F1240029
:10D4A000DB68984794F8913499070AD56FF34103E4
:10D4B000124984F89134D4F84433A1F16C005B68CC
:10D4C000984794F89034022B1AD1FEF7FBFE17E030
:10D4D000AC1E0020B01E0020E8180020987801083B
:10D4E0006C2400203022002048220020B02200209E
:10D4F0005C240020F0220020042300203C23002094
:10D5000094F891349A0640F1C6826FF3451384F87B
:10D510009134D4F84033002B40F0BD8229B0BDE8EF
:10D52000F04FFFF777BA84F84134A1E695F8182157
:10D53000012A0CD101F05EFC804668B1584601F02A
:10D540004EFC584601F050FC042384F88F347EB919
:10D55000012384F8213450E101F04EFC0028F6D07C
:10D56000404601F03DFC404601F03FFC0523ECE75E
:10D570003B7804935B09013B062B00F21882DFE83D
:10D5800013F0070016029500160292001602070219
:10D59000102EDDD995F830311297F6B28DF84C6027
:10D5A000002BD5D11CA804F05DF912AA1CA9FF20FC
:10D5B00002F0B2F89DF85830C3F3030307468DF824
:10D5C0002C3095F8480095F87D308DF82D300722E5
:10D5D0000BA902F0A4FA002F5DD100285BD09DF8C2
:10D5E00053309DF852201599C5F8E4101B0443EA06
:10D5F00002239DF8512002201343C5F8E03004F0C7
:10D600003FF99DF8583095F8480085F82E71C3F31E
:10D610000212C3F3030385F8703085F878309DF863
:10D62000593085F86920012B38BF01234FF47A72F5
:10D630005343AB651344EB650DF15A034FF00108FA
:10D640001093113E94F81B348DF83C300FA985F8E7
:10D6500068808DF8446002F06AFA0223404685F83B
:10D66000303101F08DFD18B14146384601F04CFDD6
:10D6700094F88F34012B00F2A88194F81A34002B0F
:10D6800040F09B8194F8913443F0100384F8913476
:10D69000FEF74EFD65E6012001F072FD0028E7D09F
:10D6A00001210720E2E7012384F8203495F87D303A
:10D6B0008DF82E3094F824348DF82D3095F88C3078
:10D6C00095F848000D330BA98DF82C3002F014FAB0
:10D6D000A6F10D031BB2099023EAE37300B2834263
:10D6E0003FF736AF0B2E7FF633AFBB4B25931CA80D
:10D6F000FF231C978DF874608DF8983002F0D8F8ED
:10D70000074600287FF424AF95F81831012B13D178
:10D7100001F070FB002873D0384601F060FB3846FA
:10D7200001F062FB04239DF87C101E9884F88F346E
:10D73000C1F3001101F077FB9DF87C301E99C4F80D
:10D74000341413F00F0203D09DF89000002863D129
:10D750009DF89800002862D0002A7FF4F9AE9DF869
:10D760009020002A0CBF4FF002084FF0030800225F
:10D770000A92D5F8EC20914254D195F8E91000298D
:10D7800050D0D5F80C1195F8EAB009680A9195F8CF
:10D790001811022902D1032184F88F14B8F1030F64
:10D7A0007FF4D6AE13F0600F7FF4D2AE059201275E
:10D7B00095F82E31BBF1000F37D0BBF1010F38D1F6
:10D7C000012B34D16FF0090646FA08F606F001067F
:10D7D000C6F10206F6B2BDF87E100AAA304601F084
:10D7E0002DFE40B307280CBF0823012384F8213401
:10D7F0000A9BC4F83034C4F86C34FEF7E5FCB0E59D
:10D8000001F0FAFA002897D0384601F0E9FA3846D4
:10D8100001F0EBFA052386E74FF00008A7E74FF089
:10D820000108A4E74FF0010BC2E70426D3E7032663
:10D83000D1E70123DAE71CAB009305990A9B324636
:10D84000584601F0BBFE20B102280CBF0A230B236F
:10D850007FE60A9BC4F83034C4F86C349DF87C3001
:10D8600084F82104C3F3401384F82E3484F844343C
:10D8700094F88F3484F82274012B9EBF0122A86291
:10D8800085F81E21012FC4F8280484F82C0484F89C
:10D89000410438D1022284F8202495F83A20002A45
:10D8A0004AD19DF87C20D60646D4012B94F840142A
:10D8B0009DF87C2005D8012901D1900601D501F001
:10D8C0005FFBB8F1020F94F88F3443D0B8F1030F27
:10D8D0000AD09DF87C10B8F1010F4A4601F00F0103
:10D8E00020A83BD0FFF710F99DF8903084F823343E
:10D8F000259BC4F828349DF8983084F82C340123F3
:10D9000084F82D3430E0049A02F0E002A02A1BD102
:10D9100095F82E11012285F83A2009B927996963F3
:10D92000012B84F8202407D9D5F89020C4F83C2492
:10D93000DAF80020C4F8982495F81821002AB4D108
:10D94000012284F82524B0E7002285F83A2084F8E3
:10D950002024A6E79DF8981025984A46FFF7D4F8AA
:10D960009DF8903084F823349DF89020E02A08D167
:10D9700095F81F312BB984F82324C4F82834A4F86F
:10D980002C3494F8913443F0020384F891346FE618
:10D99000114D013EB2B2791C284604F039F8032338
:10D9A000A4F82034C4F8285484F82C64E9E701234F
:10D9B00084F82134FEF708FC5AE694F84434002B2E
:10D9C0003FF460AE0020FEF7EDFB94F88F34022B9D
:10D9D0003FF45EAE56E600BFE820002094F8913494
:10D9E000590715D5012001F0CBFB60B1012001F0F2
:10D9F0009DFB08B984F81804D4F8403323F00203DF
:10DA0000C4F8403304E0062001F0BAFB0028F3D14B
:10DA100094F89134DA077FF5F9AC94F840240AB110
:10DA2000032A18D11D4A94F8181492F868209142DC
:10DA300005D29B0723D594F88F34012B1FD81848A3
:10DA400006F00AFBD4F8403323F02003C4F8403337
:10DA5000FFF742FBDAE4012A11D194F81924002AD5
:10DA60003FF4D4AC0D4A94F8181492F8682091420F
:10DA7000E5D29F0703D594F84434002BDFD194F806
:10DA8000913400206FF3041384F8913484F819045E
:10DA9000FFF744FBBAE429B0BDE8F08FE818002096
:10DAA000182200202DE9F04F89468DB09046074698
:10DAB000002800F08F81002900F08C810368002B82
:10DAC00000F088814368002B00F084818368002B7C
:10DAD00000F08081C368002B00F07C81104602F0CA
:10DAE00007F8002800F07881BD4CBE4D384601F0A3
:10DAF000C1FA40F2C4520021204603F09DFF40F2DB
:10DB00001C520021284603F097FFB74BC4F82C3174
:10DB100004F50973089304F50A7300264046099337
:10DB200008A9B24B84F848800A9384F8186184F8F5
:10DB30008C608DF82C6001F0EDFF0F2306A994F89E
:10DB400048008DF8183001F0D7FF801B18BF012066
:10DB50004FF00A0B84F81C0106A994F848008DF8D0
:10DB600018B001F0C9FF4FF0060A84F8DC0006A9DE
:10DB700094F848008DF818A001F0BEFF102384F837
:10DB8000DD0006A994F848008DF8183001F0B4FFC4
:10DB90001123C4F89C0006A994F848008DF81830A9
:10DBA00001F0AAFF1223C4F8A00006A994F84800C7
:10DBB0008DF8183001F0A0FF1323C4F8A40006A9C3
:10DBC00094F848008DF8183001F096FF1423C4F83B
:10DBD000A80006A994F848008DF8183001F08CFFD1
:10DBE0001623C4F8AC0006A994F848008DF8183044
:10DBF00001F082FF172384F8B10006A994F84800C9
:10DC00008DF8183001F078FF18230DEB0301C4F8EC
:10DC1000B400C4F8BC0094F848008DF8183001F046
:10DC20006BFFC0B21D2384F8B80084F8C00006A9B9
:10DC300094F848008DF8183001F05EFF1E2384F838
:10DC4000C40006A994F848008DF8183001F054FF7C
:10DC50001F2384F8C50006A994F848008DF81830F1
:10DC600001F04AFF2023C4F8C80006A994F8480030
:10DC70008DF8183001F040FF0B23C4F8CC0006A942
:10DC800094F848008DF8183001F036FF0C2306A9EF
:10DC9000A4F8D00094F848008DF8183001F02CFF5B
:10DCA000D4F89C306365D4F8A030A365D4F8A430D0
:10DCB000E365D4F8A83023664FF00108D4F8AC30FF
:10DCC0000590A4F8D200636684F8B080C4F894B0DC
:10DCD00084F898A0C4F84CB084F850A084F8688008
:10DCE00084F81F81C5F84893FEF77AFD404B0096F3
:10DCF00032464FF0FF3105F55A70C5F84473C4E958
:10DD00000B6684F8198185F89164C5F8408306F0A4
:10DD100045F9384B009632464FF0FF3105F56070FB
:10DD200006F03CF9344B009632464FF0FF3105F5D2
:10DD3000667006F033F902AF304B009632464FF072
:10DD4000FF3105F5806006F029F9384606F0BAF88B
:10DD500097E8030004F5927383E80300284B294FEA
:10DD60001E60294BC5F84C33284BC5F85433284B5B
:10DD7000C5F85C33274BC5F85033274BC5F85833EB
:10DD800005F553703B68984704F5A67003F088FBCF
:10DD900020B1112630460DB0BDE8F08F204601F0CD
:10DDA0001DFB0028F5D101F041F8B8B91B4801F07E
:10DDB00067FB06460028ECD17B69984703F006FE16
:10DDC000BB6D94F819019847FB6A9847012385F8C1
:10DDD0009234DFE70326DDE70926DBE71326D9E7E0
:10DDE000E8180020B01E002000040001CC23002011
:10DDF0001DD100087DC90008C5C90008A5C10008DB
:10DE0000AC1E002098780108C9C300087DC3000833
:10DE100061C1000855C300082DC30008D0190020B7
:10DE200008B5034B0020C3F84003FEF781F908BD95
:10DE3000B01E002010B5FFF7A7F90A4C60B90A4BD5
:10DE400093F81831022B02D1084BDB6A9847012363
:10DE5000C4F84033002010BDD4F84003013818BF87
:10DE60000120F8E7B01E0020E8180020987801088B
:10DE700038B5134C04F55A7006F0EEF804F56070EE
:10DE800006F0EAF804F5667006F0E6F804F580603E
:10DE900006F0E2F800F0B5FF0A4B0025DB6A984770
:10DEA000C4F84053FEF7B6FD0749084840F2C45293
:10DEB00003F0AEFD0123C4F84033284638BD00BF4F
:10DEC000B01E002098780108E818002024130020D4
:10DED00070B52E4B8AB0054693F8DD008DF8090029
:10DEE00093F8DC008DF80A0029489A6A90F8180423
:10DEF000039200268DF80B0004960C46002940D0B2
:10DF00000692D3F8882007921A8F93F81A118DF889
:10DF1000151052BAADF8202093F87C2093F84830C1
:10DF20008DF8243003AB8DF822008DF82320009368
:10DF30000DF10A020DF10B030DF1090105A88DF891
:10DF4000146000F0DDFE9DF90900FEF713F9607022
:10DF500004A801F02BF8B0B9049A0F2A0DD8637801
:10DF60009A420AD81544AB42A3EB02012CBF002011
:10DF700001202170C0000AB070BD0023237008206A
:10DF8000F9E70320F7E71320F5E700BFE8180020C2
:10DF9000B01E00201FB50446002800F01281007852
:10DFA000412800F20881DFE810F0420048004D00EF
:10DFB000520056005A005F000601060106010601E4
:10DFC000060106010601060166006A006E0079007E
:10DFD0008000830086008B0089008D0091009400F2
:10DFE00097009A009D00A000AF00B300BB00B700EF
:10DFF000BF00C200C600CF00CB00CD000601D30099
:10E0000006010601060106010601060106010601D8
:10E010000601060106010601060106010601DB00F4
:10E02000DF00E300E800EC00F000F400FD00674BC7
:10E0300093F81831237104B010BD644B93F830315C
:10E04000237102E0606803F0C7FB0020F3E760681B
:10E0500003F008FCF9E75D4B93F81A31F0E75B4BEE
:10E06000D3F8E0306360F0E7584B211D93F830019E
:10E0700003F010FCE9E7554B93F81931E0E7534BF7
:10E0800093F88C30DCE71C238DF808304F4B02A945
:10E0900093F8480001F030FD6060D6E74C4B043443
:10E0A00093E8030084E80300CFE74A4B0434F7E722
:10E0B000494B0434F4E7494B0434F1E71A23E3E70E
:10E0C0001923E1E7414B93F86830B9E73F4B5B6DAB
:10E0D000C8E73E4B9B6DC5E73C4BDB6DC2E73B4B56
:10E0E0001B6EBFE7394B5B6EBCE702238DF808302F
:10E0F000364B02A993F87C2093F848008DF80A204B
:10E1000001F0FAFC2071A0E7304B93F8DD3097E77F
:10E110002E4B93F8393093E72C4B93F8DC308FE794
:10E120002A4B93F838308BE7284BDB6C9AE7274B68
:10E1300093F8503084E7254BD3F88430636084E74C
:10E14000224B8FE7264B8DE7204BD3F8CC30F5E7F9
:10E150001E4BD3F82C31636001F05CFDA06074E7C6
:10E160001A4BD3F890307DE7184B93F81F3167E7CF
:10E17000164BB3F88830A38067E7144BB3F88A30A6
:10E18000F9E7124BB3F8D030F5E7104BB3F8D230C3
:10E19000F1E70E4B93F848200AB1062A13D1B3F8E1
:10E1A000A035E8E7094B93F848200AB1062A0AD1BE
:10E1B000D3F8A43556E7204604B0BDE8104000F07F
:10E1C00024BE032037E7182035E700BFE8180020F9
:10E1D000541900209C1900205C190020A41900206B
:10E1E000241300207FB5044610B9032004B070BD8D
:10E1F000A44DD5F840339A0700F171820278412A84
:10E2000000F26A82DFE812F04200480056005C002B
:10E21000600065006A007700820088008E0094002C
:10E220009A00A000A600AC00B6006802BB00DD00AA
:10E23000F000170139012A0144014D015101550136
:10E2400059015D016802610173019B018901AD0102
:10E25000B301BA01BF01C40168022A026802680260
:10E26000680268026802680268026802680268025E
:10E2700068026802680268026802680236023B02AD
:10E28000400245024A024F0254025E020079FEF744
:10E29000C1F80028AAD105E00379022BA5D07A4A5B
:10E2A00082F8303195F8913443F0200385F89134A9
:10E2B00000209BE7406803F081FA0028F2D094E741
:10E2C000406803F0BFFAF8E76F4B027983F81A2130
:10E2D000E8E76D4B4268C3F8E020E3E76A4E416827
:10E2E00096F8300103F0CCFA00287FF47EAF636823
:10E2F000C6F8E430D6E7416800293FF476AF002045
:10E3000001F0EEF90028CDD011206FE74168002917
:10E310003FF46BAF0120F3E7416800293FF465AF9C
:10E320000820EDE7416800293FF45FAF0920E7E7E7
:10E33000416800293FF459AF0C20E1E7416800290A
:10E340003FF453AF0D20DBE7416800293FF44DAFA8
:10E350000E20D5E7416800293FF447AF0F20CFE7F3
:10E360004A4C494B007983F81901A36D9847E36A39
:10E37000984797E7444B027983F88C2092E7424E06
:10E38000037A8DF8043096F8480096F87D308DF8C1
:10E390000530072201A901F0C2FB00283FF425AF98
:10E3A000636896F848000193002201A901F0B7FBC9
:10E3B00000283FF41AAF6C36D4E9010186E8030067
:10E3C00070E7314E037A8DF8043096F8480096F8DD
:10E3D0007D308DF80530072201A901F0A0FB00284F
:10E3E0003FF403AFB436E7E7274E037A8DF80430E5
:10E3F00096F8480096F87D308DF80530072201A97F
:10E4000001F08DFB00283FF4F0AED4E9010106F1E4
:10E41000740383E8030096F81831022B7FF442AFAF
:10E4200096F83031002B3FF43DAF184BDB6A98472C
:10E43000FDF748FF36E7144E037A8DF8043096F85E
:10E44000480096F87D308DF80530072201A901F0CB
:10E4500066FB00283FF4C9AEBC36ADE743680293C3
:10E4600001238DF80C30084B02A993F8480001F005
:10E4700063FB00287FF416AFB7E6436802930023DE
:10E48000EFE700BFB01E0020E818002098780108D0
:10E4900003795A1E0E2A3FF6A8AE934A82F86830D6
:10E4A00000E7914B42685A65FCE68F4B42689A65DB
:10E4B000F8E68D4B4268DA65F4E68B4B42681A66E3
:10E4C000F0E6894B42685A66ECE6874C037994F88B
:10E4D00048008DF80430062201A901F020FB002835
:10E4E0003FF483AE9DF8043084F8DD30DAE67E4CEC
:10E4F00003798DF8043094F8480094F87C308DF856
:10E500000630052201A901F00AFB00283FF46DAE98
:10E510009DF8043084F83930C4E6734C037994F8DC
:10E5200048008DF804300A2201A901F0F8FA002809
:10E530003FF45BAE9DF8043084F8DC30B2E66A4C00
:10E54000037994F848008DF80430092201A901F0FC
:10E55000E6FA00283FF449AE9DF8043084F83830DC
:10E56000A0E6614B4268C3F89420DA649AE65E4BF9
:10E57000027983F8982083F8502093E65A4B42683A
:10E58000C3F884208EE6584B4268C3F8CC2089E655
:10E59000012B40F0A480554C2421204603F04EFA74
:10E5A000636A984201D0172020E61C2104F128005C
:10E5B00003F044FA636C9842F5D14FF4807104F192
:10E5C000480003F03BFAD4F848319842EBD1D4210B
:10E5D00004F5A67003F032FAD4F820329842E2D162
:10E5E000002104F5097003F029FAD4F82432984286
:10E5F000D9D14FF4607104F50A7003F01FFAD4F812
:10E60000A8359842CFD1142104F2AC5003F016FA89
:10E61000D4F8C0359842C6D1334E2146304640F238
:10E62000C45203F0F5F9204640F2C452002103F031
:10E6300003FA95F81B3485F8E833736FC5F8EC33AB
:10E6400096F87D3085F8F83340F20123A5F8FA33C7
:10E65000274B96F819019B6D984723E68379012B88
:10E660003FF6C3AD204B42684068C3F82C2100F050
:10E67000D1FE47E61C4B4268C3F8902012E61A4BC5
:10E68000027983F81F210DE6174B8288A3F88820B2
:10E6900008E6154B8288A3F88A2003E6124B82888D
:10E6A000A3F8D020FEE5104B8288A3F8D220F9E52C
:10E6B0000D4B93F848200AB1062A12D1A288A3F87C
:10E6C000A025EFE5084B93F848200AB1062A08D1A7
:10E6D0006268C3F8A425E5E500F099FBD9E50120BF
:10E6E00084E5182082E500BFE818002024130020EC
:10E6F000987801082DE9F04387B00023ADF8003089
:10E700000646002800F0ED800361FEF73DFD20B1D4
:10E710000124204607B0BDE8F08300F073FD002817
:10E72000F6D100F069FD014618B96F48142203F0D4
:10E7300083F96E4D95F89134012243F0040385F876
:10E74000552485F8913433788DF804300021013B4D
:10E750008DF80520ADF806100C2B00F2BA80DFE82A
:10E7600003F007B8B8B87881B8B88FB8AC99A800EA
:10E77000D5F8407317F02007CAD196F80480B8F195
:10E78000020F45D1DFF868815A4CFEF729F896F957
:10E79000051098F848003A4601F01BFA88F839004D
:10E7A000B37988F83830384607238DF80530FDF7FF
:10E7B00031FEFF2304F58670A5F80C31C5F8084139
:10E7C00085F8047103F04EF804F58A7003F004F83C
:10E7D0003846FDF78DFE044640B196F9051098F8CD
:10E7E0004800012201F0F5F988F83900D5F8943491
:10E7F0003361002C71D000F0FFFC002889D195F81E
:10E80000913485F81A0460F3820385F8913480E727
:10E81000B8F1010F4FF00204E8D1DFF8D4908DF881
:10E82000144099F8480089F81D7102A901F072F9A5
:10E83000337989F830318DF805708DF80680FDF751
:10E8400085FC95F8913443F0100385F89134002449
:10E85000CCE700226946022000F0F6FA0028F6D044
:10E860001324C3E7244BB288DB6B96F90C10B06815
:10E870009847D5F8403343F00203C5F84033E6E744
:10E8800002A90D2000F060FB0028E0D000226946BC
:10E890000D20E1E7164B93F81831D3B9347904F021
:10E8A000070000F0ADFA8DF8004001226946102003
:10E8B000D2E7002269461220CEE78DF8072000F04B
:10E8C00090FA044638B900F089FA204600F08BFA35
:10E8D0008CE702248AE7012488E701A800F0DEFB28
:10E8E00017E7032415E700BF04230020B01E002013
:10E8F000E8180020B21E0020987801082DE9F04F9A
:10E9000099B08046059118B9032019B0BDE8F08F81
:10E9100000230361FEF738FC0646002840F0AB8078
:10E9200045460FCD0EAC0FC45A4C98F800A0B8F86D
:10E930000C7098F90EB0142204F58860314603F08B
:10E940007BF8012284F84124534C94F83021022AA8
:10E9500035460BD194F81821022A07D194F81E21CC
:10E9600022B9BAF1010F38BF4FF0010ABAF1010F15
:10E970002DD0BAF1030F2CD0BAF1000F35D10222FD
:10E980009DF83C30DDF84090029362F34715012674
:10E9900094F87C108DF8321002220CA994F84800EB
:10E9A0008DF8302001F0A8F894F81A3194F830C1AD
:10E9B00094F81D1140B20222002B6FD0BCF1010F60
:10E9C00065D1002963D1002E6DD1104627E00422C5
:10E9D000D6E70023DDF83C90BDF840709DF942B0C9
:10E9E000029365F01F050126D2E74FF0000BD946D0
:10E9F000CDF808B0CCE74FF0010084F81A04DDE050
:10EA000005F29A420BA900F0DDFA002800F02081FF
:10EA10001320049B33871F4B002283F81A241D4BBD
:10EA2000D3F89434C8F810306FE705F29A452A46B7
:10EA30000BA900F0C7FA0028EAD10B9B84F8280143
:10EA4000C4F82C5184F8303102E1B9F1000F00F024
:10EA5000FF80002A00F0FC804946E01C02F0D8FF4D
:10EA600094F8373201332380F2E01220D1E70220FC
:10EA7000CFE70720CFE7012047E7064B93F8912423
:10EA800083F840A442F0010283F89124C7E7EEB96D
:10EA90000220C4E7B01E0020E8180020002E94D009
:10EAA0005845B8BF584694F87C308DF820000522B0
:10EAB00094F848008DF8223008A901F030F80028B9
:10EAC0003FF422AF9DF8203084F83930694A6A4B10
:10EAD000D2F89804D3F8904038B105F083FA664B29
:10EAE00084423CBF002283F83A20198F1A8F93F892
:10EAF00030010491996A099152BA0028B9D093F86B
:10EB00001B0100B9186393F81801ADF858200138BB
:10EB100093F87C2093F81A411491D0F1000BD3F8AC
:10EB200088108DF85B204BEB000B93F8482093F88E
:10EB30003A0093F868308DF85A3009AB00934F4B88
:10EB400003904FF001008DF84C0015918DF85C207A
:10EB5000A3F12F01A3F1300213A88DF84D4000F06E
:10EB6000CFF8039B4FEA0B1B4BEA431B00264BEAF3
:10EB7000801B4BEAC413B1453E4C039308BF374694
:10EB80003A46494604F59C70CDE90A669B462680C4
:10EB900084F81A6402F03CFFE9B2A570C5F342158F
:10EBA000FAB2042D344E039B84F837223FF423AF8E
:10EBB000072D3FF44AAF022D7FF459AF304D84F852
:10EBC0000D110420029984F80401FF2084F80C013F
:10EBD00084F8281184F81431D6F8E410C4F80851E8
:10EBE00005F59B730AA8C4F8101184F83021C4F805
:10EBF0002C3100F017FC00287FF437AF0A9BA4F8F3
:10EC000044040BA8A4F81631C4F84C3400F0CEF933
:10EC100000287FF4FDAE0B9BD3B196F93900FDF7C8
:10EC2000A9FA94F83732002B3FF4FFAE0B9B0F2B61
:10EC30003FF6E6AE05F58B720BA90F2000F0C2F986
:10EC400000287FF4E5AE0B9B63F3030B84F814B14B
:10EC50000598FDF74DFC00287FF4DBAE099B86F894
:10EC60003A00B36200F07EF900283FF406AF1320AB
:10EC7000D1E600BFB01E0020E81800205019002087
:10EC8000B21E002037B50B4D8DF8040004460F224C
:10EC900095F8480001A900F042FF40B1064A85F806
:10ECA0001C4192F8913443F0200382F8913403B070
:10ECB00030BD00BFE8180020B01E002010B5FFF7DF
:10ECC000B9F8044688B90A4805F0C6F9094805F0BC
:10ECD000C3F9094805F0C0F900F093F8FDF780FD8D
:10ECE000064BDB6A9847204610BD0124FBE700BFB6
:10ECF00018220020302200204822002098780108A5
:10ED00002DE9F04F8BB047780093149B90F90C805D
:10ED100090F90D6090F80E908B464168196004469A
:10ED20009246002F57D002238DF8103004A9C37BE0
:10ED3000007C8DF8123000F0DFFEB4F808C0618965
:10ED400043B26068984545466144B8BF1D4660457A
:10ED500034BF00270127884209D30A218DF81010FB
:10ED6000207C019304A900F0C7FE019B46B2B4F8D1
:10ED700008C0608961680CEB400E714520D3A1EB9F
:10ED80000C01B1FBF0FC00FB1C11C9B998450ADC71
:10ED9000237833B10223207C8DF8243006A900F0BB
:10EDA000B9FE4FF0010921238DF81030207CE37B60
:10EDB0008DF8115004A98DF8123000F09DFE45B277
:10EDC000009B8BF8005038468AF8006083F800906A
:10EDD0000BB0BDE8F08F4546F2E7704770477047CB
:10EDE0007047002070477047704770470020704799
:10EDF00000207047002070470020704700207047B7
:10EE00007047704770470220704702207047022009
:10EE10007047704700207047704770470020704768
:10EE200000207047704770477047000010B5054CD0
:10EE30004FF403722046002102F0FEFD0020C4E9D9
:10EE4000000010BD702400202DE9F84381461746CC
:10EE500000293FD0244B002503F1010C1A4628015C
:10EE6000103312F8018FB8F1000F36D19A42F8D161
:10EE70001E4E33680BB9C6F800C073680BB1C3F8F7
:10EE800000C03318002401359C6083F80C900D30CD
:10EE90002B01BAB206EB05153044F750C6F804C092
:10EEA00002F0B6FDB9F1110F4FF0000398BF104CFE
:10EEB0006B71D6F8083298BF24FA09F403F1010304
:10EEC00098BF04F001043B442C71C6F80832404658
:10EED000BDE8F8834FF00108F9E70135202DBBD1DB
:10EEE0004FF00208F3E700BF7724002070240020D1
:10EEF0002007020010B510B3124A1368984204D1DB
:10EF000003681360002304E00B4613B119688842BC
:10EF1000FAD15168884208BF53600BB1016819608B
:10EF2000D2F808328168013B00245B1A0460214654
:10EF3000C2F80832102202F07FFD204610BD0120E9
:10EF4000FCE700BF70240020054B1B6813B11A7941
:10EF50008242FAD1002B0B600CBF032000207047C7
:10EF60007024002010B5054B186800B910BD037B54
:10EF700004680BB9FFF7BEFF2046F6E770240020B7
:10EF800038B5084B084C186800B938BD03790568D6
:10EF9000112B05D824FA03F3DB0701D5FFF7AAFFED
:10EFA0002846F1E7702400202007020028B1044B16
:10EFB000D3F808320360002070470120704700BF7B
:10EFC000702400202DE9F04107460E4615463AB35D
:10EFD00031B3144B1C6800232CB93046FFF7E6FF11
:10EFE0000020BDE8F081A268F91A0132914210D3E5
:10EFF0002279EA54581C22895FFA80F8611D55FA7B
:10F0000080F002F005FDA368246898445FFA88F355
:10F01000E2E720462468FFF76DFF002CF9D1DCE71A
:10F020000120DEE7702400200238C0B211289ABF08
:10F03000014B185C00207047A771010830B50B4BDD
:10F0400093F820200446084672B100211C3305784D
:10F05000A54208D001319842CDB20CBF044804301B
:10F06000AA42F4D8002030BD1046FCE77C260020E0
:10F070008826002010B5084C00232060142204F1DB
:10F080000C00FF2184F82030C4E9010002F0D4FC18
:10F09000012384F8213010BD7C26002010B50E4AD3
:10F0A00092F82010042915D8936804781C704478CD
:10F0B0005C70C478807898700131DC7082F8201020
:10F0C00002F11C018B4214BF043302F10C03936064
:10F0D000012010BD0020FCE77C260020094B93F89E
:10F0E000200068B15A6803F11C018A4200F1FF3028
:10F0F00014BF043203F10C0283F820005A6001208F
:10F10000704700BF7C26002010B5074B93F82020E5
:10F110000446084632B15968FFF790FF10B1012349
:10F120004470837010BD00BF7C26002008B5064BDC
:10F1300093F820202AB15968FFF780FF08B1407882
:10F1400008BD0120FCE700BF7C26002030B50A4A3C
:10F1500092F82010536882F8210061B1916801246F
:10F160001C32DD78587005B99C7093420CBF034B7C
:10F1700004339942F5D130BD7C260020882600203A
:10F1800008B5044B5968FFF759FF003818BF012034
:10F1900008BD00BF7C2600202DE9F3410422154E56
:10F1A000044600210DEB020096F8208002F044FC9A
:10F1B0000025EBB2984502D802B0BDE8F081736833
:10F1C000197821705A7862709F785FB13368204651
:10F1D0009B689847FFF782FF17B901A8FFF75EFF0A
:10F1E0000135E6E7DB788DF804108DF805208DF801
:10F1F0000730EFE77C260020014B93F82000704792
:10F200007C260020034B93F82000042894BF0020A4
:10F21000012070477C2600201FB50024CDE9024460
:10F22000C41F8DF800408DF801100C0AADF80420C1
:10F23000090C120C8DF803108DF806208DF807309C
:10F2400002461B0A012168468DF802408DF80830FD
:10F2500002F04FFA002818BF0E2004B010BD2DE9AF
:10F26000F04188B017460D460F9A064600284DD04B
:10F2700000240121CDE904448DF810109DF83810C8
:10F280008DF81510ADF81630190CCDE900441B0EA1
:10F29000CDE902448DF81930ADF81A20130C120E86
:10F2A00007948DF818108DF81C308DF81D20E3B2EE
:10F2B0004FEA0318002D5FFA88F803DC002008B03D
:10F2C000BDE8F081013310218DF81F303A466B46BE
:10F2D0000DEB010002F0A3F90346C8B9102DAC46AE
:10F2E000A8BF4FF0100CDAB2624503F1010303DB53
:10F2F000103D2DB20134DAE708EB020020326A44F7
:10F30000315C12F8202C4A403254ECE70920D6E751
:10F310000E20D4E70138032815D8DFE800F00208F2
:10F320000C100A4B1B681B690B6000207047074BD1
:10F330001B685B69F8E7054B1B689B69F4E7034BA7
:10F340001B68DB69F0E70520704700BFA02600209E
:10F350002DE9F041C4B00C464A9E17461D46804632
:10F36000B8B3B1F5807F36D84FF488720021684673
:10F3700002F062FB492300934FF48073ADF8043030
:10F380002B0C8DF80830330CADF80650ADF80A6040
:10F390008DF80C3022460023414604A82D0E360E6F
:10F3A0008DF80E308DF809508DF80D608DF80F40F6
:10F3B00002F02EFB04F110014B9A3B4689B26846DD
:10F3C00002F017F910B1012818BF0E2044B0BDE8B3
:10F3D000F0810920FAE70D20F8E7000010B590B1A0
:10F3E0000A4C28220021206002F026FB2368084AEC
:10F3F0001A6000204FF0FF32C3E90302C3E905227F
:10F40000C3E9072210BD0820FCE700BFA0260020AA
:10F4100000010101024B1B6818600020704700BF0B
:10F42000A026002030B1044B1B68DB680133036069
:10F430000020704709207047A026002013B5002344
:10F440000C460193D2B101A9FFF764FF18B9019BE3
:10F45000591C02D1146002B010BD99B2611A002982
:10F4600002DD0B441360F6E702D113600720F2E7D8
:10F470001B0C1B0403F580332344F3E70920EAE760
:10F4800028B1044B1B681C334362002070470920DD
:10F49000704700BFA02600201FB5044600B300231C
:10F4A00003A8039302F07CF9104ABDF80C301268EF
:10F4B00020469380E38200F056FA98B904F11803CD
:10F4C000009321680123132202F08AF860B92046D4
:10F4D00000F049FA003818BF0120000104B010BD47
:10F4E0000920FBE71020F9E70E20F7E7A02600200F
:10F4F000F0B5054687B01C463BB32F4E3368DB683A
:10F50000834257D894F82020002A14BF09220822E9
:10F51000834205D3204600F05AFA70B110200AE069
:10F52000002301900093A36894F82810606AFFF705
:10F5300096FE0028EED007B0F0BD23792168B4F81C
:10F5400008C0A768043B9AB209B90920F3E7B2F5ED
:10F55000807F2DD8ADF80EC08DF817304FEA174CCC
:10F5600004F12C033F0E8DF8117000932F0C08232B
:10F570004FF0490EADF80C008DF814708DF81600A0
:10F580002F0E0DEB0300CDF808E08DF810C0ADF89C
:10F5900012508DF8157002F023F808B10E20CAE75A
:10F5A000204600F014FA0028B8D13368DD60C2E7C5
:10F5B0000D20C0E70620BEE7A02600202DE9FF4170
:10F5C0000A9D80460F4616461C46002D5AD0002341
:10F5D00003A910460393FFF79DFE18B1062004B05F
:10F5E000BDE8F081039B9C4201D80133F6D1284647
:10F5F00000F05EF9002847D1264B1A78424503D027
:10F600001A79424542D10120AA68BA4240D103EB9F
:10F610008002EB6A92F801802979CDE90043043930
:10F62000927828683B4689B2FFF792FE0028D6D12F
:10F6300095F820300194002B4FF00103009314BF84
:10F640004246082295F82810686A3B46FFF707FEF5
:10F650000028C4D1013E032EC1D8DFE806F002071E
:10F660000B0F0D4B1B681C611C62B8E70A4B1B6833
:10F670005C61F9E7084B1B689C61F5E7064B1B686A
:10F68000DC61ACE70920AAE70F20A8E70B20A6E77A
:10F690000220A4E7A4080020A02600201FB50A46E7
:10F6A0000B2A4FF00001CDE90011CDE9021107D07E
:10F6B0000C2A13D00A2A0FD00A2005B05DF804FBEB
:10F6C000012802D120238DF80030684602F011F89D
:10F6D000002818BF0E20F0E73023F4E70B21F4E7F1
:10F6E00038B5054602F000F8044678B97DB9094BF3
:10F6F0001B680B219878FFF7D1FF38B90C21FFF771
:10F70000CDFF18B90A21FFF7C9FF00B10E2420462A
:10F7100038BD00BFA02600202DE9F04380468FB001
:10F720000C461746002A6BD0002969D000252946CF
:10F730001D2206A8059505F000FC8DF81350344DE8
:10F740002B680DF114099E88CDF804900DF1130378
:10F7500002933B7900933B6832462146404601F0D4
:10F76000E4FF00284ED138683A79494602F050F952
:10F77000384600F04FF8002846D13C7AFA79BB7938
:10F78000240444EA02241C432B689A6894423DD91D
:10F790009C609DF813000B21FFF780FF034658BBC8
:10F7A0000C21FFF77BFF034630BB0A21FFF776FFF2
:10F7B000034608BB7B7ABA7AFF7A3F0447EA0227FE
:10F7C0001F433A46334621460920FFF725FD0346ED
:10F7D00090B933463A4621460820FFF71DFD0346FF
:10F7E00050B92A689DF8131091700021D1604FF034
:10F7F000FF31C2E90411916118460FB0BDE8F083F2
:10F800000923F9E70E23F7E70F23F5E70323F3E7CF
:10F81000A026002010B50446002845D00168002924
:10F8200042D011F8013B43710322063002F0F0F898
:10F830002046032250F8091B043102F0E9F8216840
:10F84000CB79E3600A7A43EA0223E3604A7A43EA27
:10F850000243E3608A7A43EA0263E360CB7A23746B
:10F860000B7B63742379212B1AD110220D3104F103
:10F87000120002F0CDF81D222168501C8B5C6362DF
:10F88000085C43EA0023901C6362085C033243EA8D
:10F89000004363628A5C43EA02636362002010BD36
:10F8A000112B03DC0D22E7E70220F8E70120F6E741
:10F8B00010B50446002854D00168002951D00B78B7
:10F8C00043714B7883608A7843EA02238360CA7865
:10F8D00043EA024383600A7943EA026383604B7917
:10F8E00003738B79C381CA7943EA0223027BC38104
:10F8F00002F00F020831103002F08AF8237B002258
:10F9000003F00F0384F8202084F82820227903F1E3
:10F910000800111A04290DDD21680933043AD21AAE
:10F92000085C84F82000D2B2606A84F82820194468
:10F9300002F06EF8237922681A44002012F8043C81
:10F94000E36212F8031C43EA0123E36212F8021C8B
:10F9500043EA0143E36212F8012C43EA0263E362E3
:10F9600010BD0220FCE710B5044660B3036853B332
:10F970000279162A29D942791A700146082251F8CB
:10F98000060B013002F04EF82146082251F80E0B0A
:10F99000093002F047F82368E28A5A74E38A226841
:10F9A0001B0A93742368A269DA74A36922681B0A8C
:10F9B00013752368628B5A752368E27E9A75172344
:10F9C0002371002010BD0120FCE70220FAE738B5C2
:10F9D0000446002863D00168002960D0037B90F8BA
:10F9E000282003F00F03002A57D10833207904326E
:10F9F0001344984255D363790B702368A2685A70F8
:10FA0000A36822681B0A937023686289DA702368EE
:10FA1000E27A1A712368227B5A712368E2899A710B
:10FA2000E38922681B0A2146D371227B51F8100B0F
:10FA300002F00F02083001F0EBFF237B94F828203E
:10FA400003F00F0303F108052AB1226894F820108F
:10FA5000515503F10905206894F82820616A28446B
:10FA600001F0D6FF94F828302268E16A2B44D15483
:10FA70005A1CE16A206892B2090A81549A1C2168D2
:10FA8000E08D92B28854DA1C216894F82F0092B26B
:10FA9000043388542371002038BD0933A6E70120C0
:10FAA000FAE70220F8E70000024B1A88104318809A
:10FAB000704700BFA426002008B5074B1B883BB148
:10FAC000FEF7B8F900280CBF00206FF0020008BD57
:10FAD0006FF00100FBE700BFA426002010B5034B28
:10FAE00000241C80FEF79CF9204610BDA4260020AF
:10FAF000B0FA80F04009704782B018B9084602B0E9
:10FB000000F0CAB8002002B0704710B9084600F0F3
:10FB100077B9704710B9084600F08EB970470346B0
:10FB2000084611460BB900F0E5B90020704710B93E
:10FB3000084600F071BD704710B9084600F006BADB
:10FB40000020704710B40446084611461A46019B2F
:10FB500014B910BC00F018BA10BC70470346084630
:10FB600011460BB900F042BA0020704710B40446A9
:10FB7000084611461A4614B910BC00F0AFBA00206E
:10FB800010BC704730B40546084611461A46DDE9F8
:10FB900002341DB9029430BC00F02EBB002030BCF2
:10FBA000704710B9084600F0DFBB0020704710B95D
:10FBB000084600F06FBD0020704710B9084600F0FD
:10FBC000EEBB0020704710B9084600F0EBBB0020E8
:10FBD00070470346084611460BB900F005BC0020EB
:10FBE000704710B40446084611461A46019B14B9E2
:10FBF00010BC00F0FBBB092010BC704710B40446D9
:10FC0000084611461A4614B910BC00F063BDC8B2CC
:10FC100010BC70470048704701000102064B10B548
:10FC20001B6A0446984730B10448054B204498426B
:10FC30008CBF0020012010BD9878010840C220C967
:10FC400080B92A00F0B5114B85B00C4610491F56FB
:10FC5000054601F049F80F4BE4B25E6A072D4FF0FC
:10FC60000103CDE9024301460AD105220023CDE973
:10FC700000234FF47A727A431846B04705B0F0BDBE
:10FC800008220020CDE900203A46F5E7E37101089B
:10FC9000BC710108987801081FB500230093037810
:10FCA000013B372B21D8DFE803F01C242020201E45
:10FCB000202020204143454E2055585B5E61642042
:10FCC0006C1E6E73787A20207D81262020202020D3
:10FCD000202020202020202083858A2020838A2025
:10FCE0008C90C3780BB102230093009805B05DF8A7
:10FCF00004FB8378F6E743788DF8043005238DF80C
:10FD000005308378003B18BF01235B008DF8063077
:10FD100010238DF80730304B1B6801A803F558728B
:10FD2000CDE9022300F0C0FF0090DEE74023DBE7CF
:10FD30002023D9E7827890F9013012B9274AD35CA1
:10FD4000D2E7274AFBE7827890F90130002AF8D100
:10FD5000244AF4E740F6B833C6E74FF47A73C3E7B2
:10FD60004FF4FA63C0E741F28833BDE741F27073A4
:10FD7000BAE71D484FF47A7101F02EFE00F5FA60E3
:10FD8000D2E71A4BB0E7144B1B6803F55873ABE787
:10FD9000114B1B6803F55B73A6E71023A4E70E4B1A
:10FDA0001B68A1E74FF0834300939EE7104BFBE7EE
:10FDB000104B99E740F21113ADF8003095E703239B
:10FDC00092E790F901300C4AB9E70C4990F901002B
:10FDD00000F08AFFA8E700BFAC2600206B72010884
:10FDE000737201087B72010818FCFFFF00EA0637F6
:10FDF0009A99094040F70937E3710108BC7101087D
:10FE000037B50B4B02781B680C2101FB02335B7A80
:10FE100003EB4304074B1D6803690093C3684278F2
:10FE2000816805EBC40000F0DFFC03B030BD00BF0B
:10FE3000AC260020A826002070B586B0027B642383
:10FE4000ADF80030012A4FF00003CDE90133CDE9D0
:10FE500003338DF802308DF8143030D0022A39D0B7
:10FE60005ABB03684BB343683BB31F4D80682B609C
:10FE70001E4B18226946186001F0CAFD1C4B2C6805
:10FE800093E807000C3384E8070093E8070004F1C7
:10FE90000C06032386E80700A4F86C33012204F55E
:10FEA0005B7104F5587000F090FC2B684FF6B0724F
:10FEB000A3F878230522C3F87C2306B070BD0A4955
:10FEC00008684360036100F55B7100F5587000F04D
:10FED0007CFCF2E7044B1B68B3F86023B3F86C13A7
:10FEE0000A43A3F86023E8E7AC260020A8260020F8
:10FEF000106F010808B503460A2924D8DFE801F08D
:10FF000006232323230B161B23212100BDE80840D1
:10FF10000068FFF783BE90F900009978052271B957
:10FF200000F013FC003818BF012008BD052293F92A
:10FF300000000021F4E790F900005978EEE7022173
:10FF4000EEE70722F3E70020EFE7000010B50479A1
:10FF50001CB1012C0BD0002010BD0A4B01681B689E
:10FF6000012203F5587000F030FC0120F4E7054B46
:10FF700001681B68224603F55B7000F026FC2046F2
:10FF8000EAE700BFAC260020F7B50528144D1C4653
:10FF9000A8BF052058700E462946174600F0A4FE5B
:10FFA00094F90130A070072B13D1322000F09CFD92
:10FFB0000C4BDB6D0546984704F10C0208340346F0
:10FFC000019200943A463146284600F092FD03B073
:10FFD000F0BD054A55F82310D05C00F07DFDE7E741
:10FFE000BC71010898780108E37101082DE9F04F10
:10FFF000344F90F901607B68D0F804908BB00446D0
:020000040801F1
:10000000884698470546002859D1E37C73B92E4AA3
:100010002378126803EB4303990002EB8303D3F8C0
:100020000490B9F1000F01D152F80190274B4846D6
:1000300013F906B0FB689847A37CD7F818A022896B
:100040000993072E28D100230121CDE90223204A5C
:100050000693CDE90431CDE907330521CDE900212F
:100060004FF47A7202FB0BF24CF250311846D04733
:10007000637C13B3174B995D7B6D0D31C9B2284674
:100080009847E07C3246494600F040FE88F8006020
:1000900001200BB0BDE8F08F002101250823CDE938
:1000A0000013CDE90715CDE90511CDE90311029241
:1000B000A1782B465A462846D9E7074BDBE70020B4
:1000C000E7E700BF98780108AC260020E37101083B
:1000D000854501007B7201086B7201082DE9F04F24
:1000E0008DB090F90130DFF8FCA0DFF8FC90CDE98D
:1000F0000A123E4A12F903B00278DAF800300C25F1
:1001000005FB02333A4A5B7A126803EB430302EBC6
:10011000C303044693F9021090F9020000F0DFFDDA
:100120003449064694F9010000F0DEFDA2686168DA
:100130008046304600F005FD2178DAF80020D9F835
:100140000C306943074650589847D9F81C309C46F4
:1001500094F901300025072B4FF47A63CDE907535A
:10016000CDE905552DD10123CDE903530523CDE973
:1001700001534FF47A7303FB0BF300933946434664
:1001800046F2A81228466746B8472378DAF80020D6
:100190000C214B4394F90110D05800F0D9FDA189EE
:1001A00094F90100FFF74EFD0B9B217B1860D9F8F5
:1001B0005430284698470A9B01201E700DB0BDE8B8
:1001C000F08F01200823CDE90350CDE901032A4631
:1001D000CDF800B0654643463946A847012005469C
:1001E000D3E700BFAC26002098780108E37101082E
:1001F000A8260020BC7101082DE9F04F8FB0002423
:1002000005468A46914698460494ADF81440ADF8E8
:10021000024007264FF0010B2B7AA34206D96868EB
:1002200004A9204400F0F2FB00285ED102238DF8DF
:10023000083002A86B7A8DF80A30FFF72DFDAB7AF3
:100240008DF81D309DF811308DF81E309DF812305C
:100250008DF81F309DF810308DF82030EB7A8DF836
:1002600021302B7B8DF822306B7B8DF823301023CF
:100270008DF81C608DF824303A4E8DF82C000DF16D
:1002800002030A9305238DF82D3033680C9307235E
:10029000ADF834302B6806930DF1120204AB0DF16A
:1002A000110106A800F0CCFB072805460BD13068E9
:1002B0000C22002100F5587001F0BEFB3368BDF838
:1002C0000220A3F860239DF811308AF800309DF8D1
:1002D000123089F800309DF8103088F80030189BF3
:1002E00028461C700FB0BDE8F08F9DF81330BDF8A4
:1002F0001470ADF802702044C4B2F3B917B3194AB0
:1003000000201168072602464FF00C0C062B1BD16B
:100310000CFB00FE51F80EE0BEF1000F04D00BFA0A
:1003200000F23A4397B2012201301028EED1002AA0
:100330003FF472AFADF802706EE75A1E042A01D97D
:10034000062BDCD0062667E747FA00FE1EF0010FF9
:10035000EAD00CFB00FE51F80EE0BEF1000F08BF22
:100360000626E1E7AC26002038B505464068FFF7D1
:1003700055FC0522841D002195F90000E4B200F02F
:10038000E4F908B904F0FD0495F901000722002101
:1003900000F0DBF908B904F0FB04204638BD00206A
:1003A0007047000010B503780F2B044618D840683A
:1003B000FFF734FC22780B4902EB42020968831CE8
:1003C00001EB820051F82220DBB21AB903F0FD03E1
:1003D00058B210BD032B06BF626842600223F7E7E4
:1003E0000020F6E7AC260020022070472DE9F04FF0
:1003F000DFF838810446D8F8000099B089461746DE
:1004000000211E460122032300F55870CDE9061194
:10041000CDE908118DF814108DF81510ADF81630CF
:1004200000F0B5F938B9D8F80020B2F8603343F0DD
:100430000303A2F86033D8F80020637A8DF82830DF
:1004400002F55871CDE90B12394A94F90830126857
:100450000D920DF116020F922268109262681192AD
:10046000D4E90301A27A8DF8482001228DF84920B1
:1004700013AA82E803001025227DE18A8DF8293035
:1004800018468DF85420ADF83850FFF7DBFB0AAB67
:1004900017930DF11503169000933146019705ABA4
:1004A00006AA10A800F0BCFB064698BB9DF81410E5
:1004B000204F013901F090FA1F4B1B690393C4B21E
:1004C0004FF00C0B04F160036B44D8F8000013F8F4
:1004D00048AC9DF814300BFB0AFC01343946B4FBE0
:1004E000F3F203FB1244D0F87C33B0F9782350F8D0
:1004F0000C00DDF80CC0E4B2E04728B189F800A098
:10050000304619B0BDE8F08F013D15F0FF05D9D197
:100510000D26F5E70C2801BFD8F80020B2F86033AB
:1005200043F00303A2F86033EAE700BFAC260020E3
:10053000A8260020400D030098780108F8B5067938
:10054000012E054601D80620F8BD0F2E2BD80368D2
:10055000187A40F303000522002140B200F0F5F8BC
:100560002B680446187A40F303100522002140B29C
:1005700000F0EBF8A8B1B4FA84F4640929680B7AA6
:10058000086843F3030243F3031352B25BB29A4287
:10059000C8BF0124FFF742FB48B9002CD3D1042087
:1005A000D2E70124EAE70320CEE70520CCE7002CC0
:1005B000FBD10C4F29683B6806EB460003EB80003B
:1005C0000C2201F025FA3A680C2303FB062320468F
:1005D0005C72B2F860130123B3400B43A2F860339E
:1005E000B2E700BFAC26002010B4017801290ED973
:1005F000084B18680C234B43C4180022C250C4E9AE
:10060000012200F5587010BC102200F0A7B800209D
:1006100010BC7047AC2600202DE9F04186B0502375
:100620008DF81430037A102B074630D14368DD7BF8
:100630006DBB0224A8466426062C14D87A68535D44
:1006400003932A44517843EA01230393927843EABF
:1006500002437343CDE9033863B968468DF800401F
:10066000FFF7C2FF0DE0CDF80C808DF81480CDF8B7
:100670001080F2E703AB01A801938DF80840FFF763
:100680005DFF0134E4B2102C05F10305D4D106B0AE
:10069000BDE8F0811FB502680379116851B901A85E
:1006A0008DF80430FFF7A0FF78B9002040B205B004
:1006B0005DF804FB02A802928DF80C30FFF73EFFB4
:1006C0000628F2D8024B185CF0E70320EEE700BFE3
:1006D000DC710108C90020B9034B0B449856C0B225
:1006E0007047024BF9E700BFEB7101082B7201085C
:1006F000F0B59A42069D03DB9DF914309A4220DD45
:100700000020F0BD03EB430331F814C005EB830375
:1007100000264CFA06F7FF0707D51F7A07F00F0EE1
:10072000724502DBB2EB171F0DDD0136102E03F10F
:100730000C03EED10134E4B22301DBB29842E1D8DC
:10074000DEE70024F8E70120DBE7884204DB904283
:10075000CCBF0020012070470020704710B514095D
:10076000B4EB111F03464FEA11100ED391420CD285
:1007700002B201F00F0133F81240012000FA01F13A
:1007800024EA010123F8121010BD0020FCE7F0B5A7
:1007900028B100EB410501270020914200D3F0BDB4
:1007A000002435F802CB234607FA04F636EA0C0695
:1007B00008BF013304F1010408BFDBB2102CF3D1F0
:1007C00018440131C0B2C9B2E7E710B500B149B968
:1007D00010BD31F8134020F813400133DCB2A242BF
:1007E000F7D8F5E70023F9E782B030B50488049321
:1007F0006AB9B3F5616F18D349F6AF2542F21072AA
:10080000AB4298BF4FF47A72944238BF1446012C21
:1008100038BF01246143BDE83040C3688B428CBFC0
:100820005B1A0023C36002B070476422ECE700004B
:100830002DE9F04F91B01546DDF86C8004939DF8DA
:10084000683009930C46064603F0C2FB684ADFF89D
:10085000A4B10590A8F5F633303BB3FBF2F3534354
:1008600003F5F63203F5A83303F5C0730393182399
:1008700013FB054330320692089300254FF0FF3AF0
:10088000089BA34207D1002D14BF50464FF0FF3004
:1008900011B0BDE8F08FBDF97030ADF82C300B9978
:1008A000CDF86C804046CDF8288003F021FBB4F8E9
:1008B00000906EB9B8F5616F5BD349F6AF2242F292
:1008C0001073904598BF4FF47A73994538BF994695
:1008D0004B46012B38BF01230793002E52D1B9F1AB
:1008E000640F48D1A0605F46A1680EA803F022FB08
:1008F0000F9B0093DDE90A120E9B0CA803F079FA16
:10090000049B0C9A0BB9099B2BB12369BB4202D102
:10091000394B9A420DD9394BE760984509D90023E4
:10092000ADF83430069B0D990C93184603F0E0FAAD
:10093000A060606800B9E760276126B103F052FB50
:10094000E3680344E360D4E903329342059B1D99B5
:100950006360079B88BFE2604B43E168994202D223
:100960000498A8B9A6B101231D442375EDB218342B
:1009700086E76423A9E7B9F57A7F0ABF204F214FA4
:10098000A060B1E7049B0BB9C4F80CB05F46D0E798
:1009900000209342207506D85B1A9A4505F101059F
:1009A00028BF9A46EDB2002EE1D1B9F1640F164A84
:1009B000ADF8346019D049F6B023B9F57A7F18BF85
:1009C0001346904584BF039A9B180C931C9B00937D
:1009D0000CAF97E806001B9B384603F00AFA97E82D
:1009E000030003F085FA8246C1E74FF46163E8E74C
:1009F0008051010040771B007F5101002FEC010066
:100A000080A81201002E930230EC01000378032B22
:100A100014D1437803F00F021B098A704B7083785E
:100A20008B80C27843EA02238B800379C3F30212DE
:100A300003F00F03CA700B70052070470020704749
:100A40002DE9F34798464379057990F90760914677
:100A5000044690F906208A4683B190F9087075B370
:100A60000F2A12D194F909200F2E1ED194F90A6091
:100A7000072D24D1002F08BF012720E090F90B702B
:100A800090F9092090F90A60E9E7A369019394F9C4
:100A900015300093216994F91430207BFFF728FE6C
:100AA0000028E1D105F0FD05DEE794F91D30B342E1
:100AB0000FDC94F91C30B342DADA05F0FB05284666
:100AC0008AF8002089F8006088F8007002B0BDE85C
:100AD000F0871E46CCE70000024B03FA00F0B0FBA3
:100AE000F1F0704740420F004FF4FA53B3FBF0F0BF
:100AF000704730B54FF47A750C1F6A4300FB04222F
:100B000052001EBF00F1FF341219B2FBF0F2914205
:100B100038BF1146039A1160820048431CBF013060
:100B200040084FF47A71121A01FB1323002BCABF3D
:100B300003F2E73393FBF1F1B3FBF1F1049B19608E
:100B400030BD38B5400014460D46F1F7E3F90146D3
:100B50002846F1F72DF92146F1F72AF9F0F7F4FDCF
:100B600006F02EF9F1F7F8F840B238BD2DE9F74F4D
:100B7000019300231F469C461C01058A5FFA84FEF0
:100B800004F0F004A54206D8019B82F800C01F7053
:100B900003B0BDE8F08F0EEB4E054FEA4309AD0000
:100BA0000024466836F809602641F60727D586688E
:100BB00006EB050A765916B3067836B9466926B1AA
:100BC00036F809602641F60719D59AF8086090F9B9
:100BD00001B046F303084FFA88F8D8450FDC46F316
:100BE000031676B25E450ADB9AF8096006EB460802
:100BF000C66806EBC806367D4EB90137FFB2013430
:100C0000102C05F10C05CCD10133DBB2B4E70CF1AB
:100C100001060EEB040801F80C805FFA86FCEEE793
:100C20002DE9FF4704464068DDE90C671D468A460A
:100C3000914603F0D7F923681B1A3B604FF0000878
:100C40000123337085F80080636813B12368834201
:100C500024D8CAF80080D4F81CC0A3699CF800E02E
:100C60000393D4E9030101AB83E80300237D0093E0
:100C7000DCF80C10237A627A7046FFF7D9FD334610
:100C800038602A46E0694946FFF770FF2B782BB1A0
:100C9000C7F80080002004B0BDE8F0873378002B4F
:100CA00014BF0B200C20F6E737B590F9002090F91F
:100CB0000250954204460FD0013A52B295420BD0F1
:100CC000A368019394F9013000936168E0782B46A2
:100CD000FFF70EFD0028EFD0104603B030BD88426C
:100CE000B8BF08467047000051F82000054B9842F5
:100CF00005D0054BC31A58425841400070470120A7
:100D0000704700BF90D0030020A1070005281FB541
:100D10000ED80C4B53F820300093CDE901120A4B4A
:100D200001220021022002F069FE05B05DF804FBFB
:100D3000CDE90012054B01220021022002F05EFEE7
:100D4000F3E700BFF072010883720108A272010884
:100D500007B5054BCDE9000101220021022002F078
:100D60004DFE03B05DF804FBBE72010810B5102201
:100D700004460021F13000F05FFE0021C4F8141198
:100D80002046F022BDE8104000F056BE024608465C
:100D9000102100F0A5B92DE9F0430446D0F8140164
:100DA00085B00E46154604F2011988B3C0F110084B
:100DB0009045474628BF1746BAB2484400F028FE7F
:100DC000D4F814313B440F2BC4F814312DD9A84565
:100DD0002BD204F1F00304F5807113F8012F187C75
:100DE0008B4282EA00021A70F7D104F1F108102256
:100DF0004146684600F00CFE22466946684600F00F
:100E0000E9F910226946404600F002FE3E44ED1B1F
:100E100004F5807804F1F107102D09D8AAB2314603
:100E2000484600F0F5FDC4F8145105B0BDE8F08364
:100E300004F1F003711E13F8012F11F8010F43455F
:100E400082EA00021A70F6D110223946684600F094
:100E5000DFFD22466946684600F0BCF9102269466B
:100E6000384600F0D5FD1036103DD5E7F0B589B015
:100E70000C46102200210546684600F0DDFD2246A2
:100E80006946684600F0A6F99DF90030002B6A46D5
:100E90004FF0000143DA137812F8010F01315B00C3
:100EA00043EAD0130F2902F8013CF4D19DF80F302A
:100EB0005B0083F08703D4F81401DBB210288DF8AF
:100EC0000F303BD104F58073694604F5887013F840
:100ED000016F11F8012B984282EA06021A70F6D1CE
:100EE00004F1F00304F5807113F8012F187C8B4294
:100EF00082EA00021A70F7D110220DEB020004F111
:100F0000F10100F085FD2246294604A800F062F9AF
:100F100010220021684600F08FFD09B0F0BD137863
:100F200012F8010F01315B0043EAD0130F2902F8D8
:100F3000013CF4D19DF80F305B00BCE79DF9003017
:100F4000002B6A464FF0000137DA137812F8016F70
:100F500001315B0043EAD6130F2902F8013CF4D1BA
:100F60009DF80F305B0083F08703471CDBB28DF8E0
:100F70000F30102F04EB0003C0F10F064FF080027A
:100F800088BF002600F5817083F8012100213246D8
:100F900020443E4403F0D1FFC4F8146104F580738B
:100FA000694604F5887013F8016F11F8012B984217
:100FB00082EA06021A70F6D192E7137812F8016FEE
:100FC00001315B0043EAD6130F2902F8013CF4D14A
:100FD0009DF80F305B00C8E70A7803785340037030
:100FE0004A784378534043708A78837853408370BB
:100FF000CA78C3785340C3700A79037953400371A8
:101000004A794379534043718A7983795340837194
:10101000CA79C3795340C3710A7A037A5340037281
:101020004A7A437A534043728A7A837A534083726E
:10103000CA7AC37A5340C3720A7B037B534003735B
:101040004A7B437B534043738A7B837B5340837348
:10105000CA7BC37B5340C373704710B50B781478B9
:101060006340037054784B786340437094788B7876
:1010700063408370D478CB786340C37014790B7964
:101080006340037154794B796340437194798B7950
:1010900063408371D479CB796340C371147A0B7A3E
:1010A00063400372547A4B7A634043728B7A947A2A
:1010B00063408372D47ACB7A6340C372147B0B7B18
:1010C00063400373547B4B7B63404373947B8B7B04
:1010D00063408373CB7BD27B5340C37310BD00004E
:1010E000A1F11003DBB2102B2DE9F04704D8374CE7
:1010F00024FA03F3DB0705D4002382F8F030FF2045
:10110000BDE8F087531E4418A0424ED101F11C03E4
:101110009B005FFA83F9C3F30313013B2C4D82F864
:10112000F03001240B46D618B3FBF1F001FB103070
:1011300010F0FF0016F804AC16F803EC16F802CC19
:1011400016F8017C36D115F80E8015F80CE015F86C
:1011500007C015F80A70E00900EB400084EA0808AF
:1011600000EBC0006400C0B2E4B24440C246581A6A
:10117000C0B212F800808AEA080A02F803A01044FC
:10118000043390F801808EEA080E86F801E090F8AA
:1011900002E08CEA0E0C86F802C0C078DBB2474051
:1011A0009945F770BFD80020AAE710F8015B03F853
:1011B000015FA9E71829DAD9102801BF15F80AA09C
:1011C00015F80EE015F80CC0EF5DD0E70101010045
:1011D000087501082DE9F04FA3B092F8F0301D9189
:1011E0001B920193002B00F0538101461EA8FFF7CC
:1011F00034FF1B9BA74CA84DA84E1033029300232D
:1012000003939DF87C0004909DF886000590205C77
:1012100006909DF87B000790205C089004989DF84C
:1012200081C0205C099014F80C000A909DF88000A1
:101230000B909DF885009DF878809DF87DE09DF8E5
:1012400082A09DF887900C909DF87A00029B1C93D9
:1012500014F80A2014F8093014F8081014F80E7065
:101260000D90205C0E909DF87F000F90205C1090F8
:101270000B98205C11900C98205C12909DF88400D3
:1012800013909DF8790014909DF87E001590205CD5
:1012900016909DF883001790205C18901398205C9E
:1012A00019901498205C1A900398013003900298CA
:1012B000DDF804B0103002909DF80C00834536D85C
:1012C0008DF878108DF87A2009990E9A8DF87C1097
:1012D0008DF882201199069A8DF880108DF87E2065
:1012E0001999169A8DF884108DF886200A99189A03
:1012F0008DF87D108DF887201299109A8DF87B302B
:101300001B9B8DF881108DF883201A99089A1D98DF
:101310008DF885108DF87F201EA903EB0B128DF838
:101320007970FFF79AFE002023B0BDE8F08F15F822
:1013300008B082EA03008BEA000016F80EB080EADB
:101340000B008DF8780015F80E004B40434016F85E
:101350000A0043408DF8793081EA070315F80A1036
:10136000594016F80930594016F808308DF87A10AF
:101370007A40534015F8092053408DF87B30089A85
:10138000069B5340049AAA5C534016F80C20534025
:101390008DF87C30DDE908325A4015F80C305340A6
:1013A000059AB25C53408DF87D30DDE909325A4030
:1013B000059BEB5C5340079AB25C53408DF87E303E
:1013C000069B0A9A5340049AB25C5A40079BEB5C16
:1013D0005A408DF87F200E9B109A53400B9AAA5CBE
:1013E00053400C9AB25C53408DF88030DDE91032E6
:1013F0005A400C9BEB5C53400D9AB25C53408DF805
:101400008130DDE911325A400D9BEB5C53400F9A5D
:10141000B25C53408DF88230129A0E9B53400B9A67
:10142000B25C5A400F9BEB5C1C995A408DF88320AC
:10143000169B189A5340139AAA5C5340149AB25CB4
:1014400053408DF88430DDE918325A40149BEB5C30
:101450005340159AB25C53408DF88530DDE919325E
:101460005A40159BEB5C5340179AB25C53408DF881
:1014700086301A9A169B5340139AB25C5340179ABF
:10148000AA5C1EA853408DF88730FFF7A5FDB8E68B
:10149000FF2049E70875010808730108087401086E
:1014A00008B538B1044A05491060D82200F0B0FAF6
:1014B000002008BD0220FCE7B0260020A47D010822
:1014C0000A4B1A6870B5002302F1180503EB0314E8
:1014D0002E5D864204D1183422440A60002070BD7B
:1014E00001330B2BF2D10320F9E700BFB026002017
:1014F0002DE9F041CCB00646DDF8488117461C4680
:101500000D4631B3B8F1000F23D006A8FFF72EFC2B
:10151000204601A9FFF7D4FF0446B0B9019906A8F7
:101520000131FFF733FC26B11022314606A8FFF740
:1015300032FC3A46294606A8FFF72DFC06A902A868
:10154000FFF794FC029BC8F8003020464CB0BDE881
:10155000F0810224F9E7000030B595B013A90446E4
:10156000FFF7AEFF002830D11B490C2303FB00F22C
:10157000555CA5422BD1139B187C1090D87B0F9003
:10158000987B0E90587B0D90187B0C90D87A0B901E
:10159000987A0A90587A0990187A0890D879079022
:1015A000987906905879059018790490D878039026
:1015B000987802900A445B78019393680093002224
:1015C000064B1146022002F019FA15B030BD013069
:1015D0000B28CBD1F9E700BF807701080876010816
:1015E0000B2B10B402D810BCFFF782BF032010BC35
:1015F000704730B50D4685B01446014668B103AA60
:10160000002000922A460390FFF772FF18B9039852
:10161000001B18BF012005B030BD0220FBE72DE9FB
:10162000F0430D46BFB014469946804620B31BB325
:1016300011F00F0122D1F02201A800F0FDF920469F
:101640006946FFF73DFF044648B9009801AA1021FA
:101650000130FFF745FD2E46AF1BFFB21EB92046F5
:101660003FB0BDE8F08301AA09EB070108EB0700D2
:10167000FFF7B0FD103EEFE70224F0E70524EEE7A8
:10168000F0B5184E3468024685B00846002304F1D0
:10169000180103EB03154F5D97421ED10D2A05F18A
:1016A000190513D10023CDE90033CDE902330C2213
:1016B00010216B46FFF7B3FF0446306810226946DD
:1016C000284400F0A5F9204605B0F0BD01461022DF
:1016D000601900F09DF90024F5E701330B2BD8D1F8
:1016E0000324F0E7B026002009B1FFF7C9BF0220AC
:1016F00070471FB51446A0B10C2A01D10B2912D195
:101700000023CDE90033CDE902330A466B461021B0
:10171000FFF785FF18B969462046FFF7B1FF04B00F
:1017200010BD0220FBE70320F9E7F8B51E46DDE90E
:1017300007479DF818505BB354B34FB3212D29D8F8
:1017400019462A46204600F063F90122631C691EEF
:10175000B018FFF764FFF8B9E37ADB093B70EBB927
:101760006319204613F8012C13F8021C120642EAF2
:10177000014213F8041C0A4313F8031C012342EA34
:101780000122291FFFF735FF003818BF0120F8BDDF
:101790000220FCE70520FAE70720F8E70420F6E737
:1017A00010B5044628B1044B5B69984720600020BF
:1017B00010BD0220FCE700BF9878010808B501467B
:1017C00030B1044B0822186800F022F9002008BD4F
:1017D0000220FCE7B026002008B530B1044B0822F7
:1017E000196800F015F9002008BD0220FCE700BFD1
:1017F000B02600207FB5124E0023044602A80193B4
:101800000D46FFF7E9FF33685B6901936CB102AAEB
:10181000082312F8011B41B9013B13F0FF03F8D173
:1018200002A8A04702A8FFF7C9FF35B1019B23B961
:1018300001A8A8473368019A5A61002004B070BD1E
:10184000B026002008B5014638B1054B18680822BB
:10185000104400F0DDF8002008BD0220FCE700BFC6
:10186000B026002008B538B1044B1968082211448D
:1018700000F0CEF8002008BD0220FCE7B0260020D2
:10188000034B1B6802280CBF196159610020704787
:10189000B026002041B1054B1B6802280CBF1B6914
:1018A0005B690B600020704702207047B026002063
:1018B00030B58FB0002405460CA80994FFF78CFFC3
:1018C0009DF8373007939DF8363006939DF83530F4
:1018D00005939DF8343004939DF8333003939DF8BD
:1018E000323002939DF8313001939DF830300093EF
:1018F000224621461E4B022002F080F80AA8FFF77C
:10190000B1FF9DF82F3007939DF82E3006939DF878
:101910002D3005939DF82C3004939DF82B300393C4
:101920009DF82A3002939DF8293001939DF82830C4
:10193000009322460F4B2146022002F05FF809A9CE
:101940002846FFF7A7FF9DF8243003939DF8253024
:1019500002939DF8263001939DF82730009322468C
:10196000054B2146022002F049F80FB030BD00BF00
:1019700064760108A2760108E076010808B5002027
:10198000FFF7EAFD0120FFF7E7FD0920FFF7E4FD7F
:101990000820FFF7E1FD0020FFF78AFF002008BDC7
:1019A00010B504460B20FFF7D7FD0C20FFF7D4FD40
:1019B0000920FFF7D1FD0820FFF7CEFD0A20FFF731
:1019C000CBFD2046FFF774FF002010BD014B1860CF
:1019D000704700BFAC0800200B4A30B514680B4DAF
:1019E00043F2390305FB04331360091A6FF0004218
:1019F000B3FBF2F2C2EBC27201319B1A93FBF1F21C
:101A000001FB1233184430BDAC0800206D4EC641B6
:101A100001380A44914200D1704711F8013B00F8A7
:101A2000013FF7E710440A44914200D1704711F892
:101A3000013B00F8013DF7E703F07FBA30B530B164
:101A40000A4D01444FF0FF33814201D1D84330BDEC
:101A500010F8012B5340082243F30004013A2C40B4
:101A600092B284EA5303002AF6D1EDE72083B8ED61
:101A700001207047054B4FF400529A62044B1B68DB
:101A800013B15B6803B11847704700BF00040048FA
:101A9000B4270020054B4FF480529A62044B1B6818
:101AA00013B1DB6803B11847704700BF000400485A
:101AB000B4270020012070470120704701F048B989
:101AC00001F036B910B501F019FE0E21044640F6BA
:101AD0001F1001F02DF92046012101F0F9FDBDE8AC
:101AE000104001F0D7BA000070B50C4E01EB400376
:101AF0000D46B3654FF6FF71002304461A460846AB
:101B000001F05EFB96F85600002101F0E1FD294648
:101B10002046BDE8704001F095BA00BFD0270020F4
:101B200010B5044601F0AAFE01281CD101F0AEFE5A
:101B300034B11248214602F017FB104802F0DAFADD
:101B40000F4C104B00214FF48052A1659A6194F81C
:101B5000560001F0BDFD63786BB16FF07F40BDE8CA
:101B6000104001F053BA002340F262211A460846A1
:101B700001F026FBDCE7A0688001F0E7B827002031
:101B8000D027002000040048002001F0BFB9000069
:101B900008B501F0C7F80438C0B2032896BF024B5D
:101BA0000020185C08BD00BF9478010808B501F05A
:101BB000BAFD033008BD01F049B901F009B908B513
:101BC00001F000FD00B208BD38B50D46144601F025
:101BD0005DFB284601F092FD0E21054640F61F10E0
:101BE00001F0A6F828460121074D01F071FD01F032
:101BF00051FA4FF47A716143284602F0B5FA28464B
:101C0000BDE8384002F076BA2C28002001F03EBB37
